S015000070756D705F626F6172645F76322E73726563DF
S3150802000000000A203DE203086D830308758303088E
S315080200107D830308858303088D8303088DE203081D
S315080200200000000000000000000000008DE2030846
S31508020030958303080000000035030208E10202085E
S315080200408DE203088DE203088DE203088DE20308B8
S315080200508DE203088DE203088DE203088DE20308A8
S315080200608DE203088DE203088DE203088DE2030898
S315080200708DE203088DE203088DE203088DE2030888
S315080200808DE203088DE203088DE203088DE2030878
S315080200908DE203088DE203088DE203088DE2030868
S315080200A08DE203088DE203088DE203088DE2030858
S315080200B08DE203088DE203088DE203088DE2030848
S315080200C08DE203088DE203088DE203088DE2030838
S315080200D0000000008DE203088DE20308A5830308E9
S315080200E08DE203088DE203088DE203088DE2030818
S315080200F08DE203088DE203088DE203088DE2030808
S315080201008DE20308B98303088DE203088DE203082A
S315080201108DE203088DE203088DE203088DE20308E7
S315080201208DE203088DE20308CD8303088DE20308F6
S31508020130E18303088DE203088DE203088DE20308D2
S315080201408DE203088DE203088DE203088DE20308B7
S315080201508DE203088DE203088DE203088DE20308A7
S315080201608DE203088DE203088DE203088DE2030897
S315080201708DE203088DE203088DE203088DE2030887
S315080201808DE203088DE203088DE203088DE2030877
S315080201908DE203088DE203088DE203088DE2030867
S315080201A08DE203088DE203088DE203088DE2030857
S315080201B08DE203088DE203088DE203088DE2030847
S315080201C08DE203088DE203088DE203088DE2030837
S315080201D08DE203088DE20308000000008DE20308A1
S315080201E08DE203088DE2030800000000000000000B
S315080201F08DE2030800000000000000008DE20308FB
S315080202008DE203088DE203088DE203080000000070
S31508020210000000008DE20308000000008DE20308DA
S315080202208DE203088DE203088DE203088DE20308D6
S315080202308DE203088DE203088DE203088DE20308C6
S315080202408DE203088DE203088DE203080000000030
S3150802025010B5054C237833B9044B13B10448AFF3F0
S3150802026000800123237010BD5414002000000000F2
S315080202700C69050808B5034B1BB103490348AFF3DC
S31508020280008008BD00000000581400200C6905080B
S3150802029072B64FF0E0201749C0F8081D16480168E3
S315080202A041F00101016015481249096801604FF0E1
S315080202B0E020134941614FF0070101614FF0000147
S315080202C0C0F8181D4FF07F41C0F81C1D0D49C0F833
S315080202D0201D7047FFF7FEBF01B5BDE80140704714
S315080202E001B500F097F8BDE801407047FFF7FEBF79
S315080202F0FFF7FEBF00000208001000E0FC560120CE
S315080203008FD003000000FF404FF000002D4A106016
S31508020310EFF3148020F0040080F3148862B64FF0DD
S3150802032080504FF0E021C1F8040DBFF34F8FBFF3A1
S315080203306F8FFEE72448254A4FF00003016891B102
S315080203400360EFF3098C2CE9F00F1EF0100F01D1B0
S315080203502CED108A1E4C4CF804EDC1F808C025682D
S315080203600DB18D61236072B61168D1B1016062B6B2
S315080203704F68174C8D6907F101074F602560D1F860
S315080203800CC08CF30B88D1F808C05CF804EB1EF09D
S31508020390100F01D1BCEC108ABCE8F00F8CF3098867
S315080203A0704772B61168016009B962B6F9E74FF08B
S315080203B000674FF0E028C8F8047D62B6D8E700BFA8
S315080203C07047000098570120005701200457012062
S315080203D0045D0120026922F00702A2F144026FF0CD
S315080203E0430313604FF0000353609360D3601361B5
S315080203F053619361D361136253629362D362136347
S3150802040053634FF0FF339363D1634FF080731364E2
S31508020410826070472249086800F101000860214B92
S315080204201A683AB1A2F101021A601AB91E4B4FF0C4
S31508020430010018601D490868026822B11C4B4FF07A
S3150802044001021A6008E000F104001A4B1A68904289
S3150802045001D1194B18680860134B1A6812B9144966
S315080204600868C8B101B51249086808B129F0D4FD6F
S315080204700D4B1A6872B129F041FD1048016849B955
S315080204800F4801680F4A13680F484FF08052994285
S3150802049000D00260BDE80140BFF34F8F70470000ED
S315080204A0A4570120045D0120A857012034580120D1
S315080204B038580120305801202C580120985701201D
S315080204C0005701200457012004ED00E0034613F803
S315080204D0012B002AFBD1181A0138704781F0004116
S315080204E002E000BF83F0004330B54FEA41044FEA09
S315080204F0430594EA050F08BF90EA020F1FBF54EAA4
S31508020500000C55EA020C7FEA645C7FEA655C00F03F
S31508020510E2804FEA5454D4EB5555B8BF6D420CDD10
S315080205202C4480EA020281EA030382EA000083EA93
S31508020530010180EA020281EA0303362D88BF30BD33
S3150802054011F0004F4FEA01314FF4801C4CEA113189
S3150802055002D0404261EB410113F0004F4FEA0333E8
S315080205604CEA133302D0524263EB430394EA050F73
S3150802057000F0A780A4F10104D5F1200E0DDB02FAE2
S315080205800EFC22FA05F2801841F1000103FA0EF276
S31508020590801843FA05F359410EE0A5F120050EF13C
S315080205A0200E012A03FA0EFC28BF4CF0020C43FA6D
S315080205B005F3C01851EBE37101F0004507D54FF07A
S315080205C0000EDCF1000C7EEB00006EEB0101B1F5CA
S315080205D0801F1BD3B1F5001F0CD349085FEA300010
S315080205E04FEA3C0C04F101044FEA445212F5800F1B
S315080205F080F09A80BCF1004F08BF5FEA500C50F1B8
S31508020600000041EB045141EA050130BD5FEA4C0C9A
S31508020610404141EB0101013C28BFB1F5801FE9D2F7
S3150802062091F0000F04BF01460020B1FA81F308BF1A
S315080206302033A3F10B03B3F120020CDA0C3208DDE6
S3150802064002F1140CC2F10C0201FA0CF021FA02F1C1
S315080206500CE002F11402D8BFC2F1200C01FA02F131
S3150802066020FA0CFCDCBF41EA0C019040E41AA2BF56
S3150802067001EB0451294330BD6FEA04041F3C1CDA1E
S315080206800C340EDC04F11404C4F1200220FA04F03E
S3150802069001FA02F340EA030021FA04F345EA0301E8
S315080206A030BDC4F10C04C4F1200220FA02F001FAAA
S315080206B004F340EA0300294630BD21FA04F029462C
S315080206C030BD94F0000F83F4801306BF81F48011C5
S315080206D00134013D4EE77FEA645C18BF7FEA655C38
S315080206E029D094EA050F08BF90EA020F05D054EA0A
S315080206F0000C04BF1946104630BD91EA030F1EBF0F
S315080207000021002030BD5FEA545C05D14000494112
S3150802071028BF41F0004130BD14F580043CBF01F505
S31508020720801130BD01F0004545F0FE4141F47001EB
S315080207304FF0000030BD7FEA645C1ABF19461046C6
S315080207407FEA655C1CBF0B46024650EA013406BFC7
S3150802075052EA033591EA030F41F4002130BD00BF86
S3150802076090F0000F04BF0021704730B54FF4806443
S3150802077004F132044FF000054FF0000150E700BFC4
S3150802078090F0000F04BF0021704730B54FF4806423
S3150802079004F1320410F0004548BF40424FF0000110
S315080207A03EE700BF42004FEAE2014FEA31014FEA53
S315080207B002701FBF12F07F4393F07F4F81F06051A2
S315080207C0704732F07F4208BF704793F07F4F04BFED
S315080207D041F40021704730B54FF4607401F00045CA
S315080207E021F000411CE700BF50EA010208BF70472A
S315080207F030B54FF000050AE050EA010208BF70471B
S3150802080030B511F0004502D5404261EB41014FF483
S31508020810806404F132045FEA915C3FF4D8AE4FF08B
S3150802082003025FEADC0C18BF03325FEADC0C18BF6E
S31508020830033202EBDC02C2F1200300FA03FC20FABF
S3150802084002F001FA03FE40EA0E0021FA02F114440C
S31508020850BDE600BF70B54FF0FF0C4CF4E06C1CEA25
S3150802086011541DBF1CEA135594EA0C0F95EA0C0F96
S3150802087000F0DEF82C4481EA030621EA4C5123EA09
S315080208804C5350EA013518BF52EA033541F4801138
S3150802089043F4801338D0A0FB02CE4FF00005E1FBEB
S315080208A002E506F00042E0FB03E54FF00006E1FB35
S315080208B003569CF0000F18BF4EF0010EA4F1FF0478
S315080208C0B6F5007F64F5407404D25FEA4E0E6D41B8
S315080208D046EB060642EAC62141EA55514FEAC520C9
S315080208E040EA5E504FEACE2EB4F1FD0C88BFBCF545
S315080208F0E06F1ED8BEF1004F08BF5FEA500E50F1F6
S31508020900000041EB045170BD06F0004646EA0101BB
S3150802091040EA020081EA0301B4EB5C04C2BFD4EBED
S315080209200C0541EA045170BD41F480114FF0000EE6
S31508020930013C00F3AB8014F1360FDEBF002001F054
S31508020940004170BDC4F10004203C35DA0C341BDCCE
S3150802095004F11404C4F1200500FA05F320FA04F0A0
S3150802096001FA05F240EA020001F0004221F00041D4
S3150802097010EBD37021FA04F642EB06015EEA430E47
S3150802098008BF20EAD37070BDC4F10C04C4F1200577
S3150802099000FA04F320FA05F001FA04F240EA02002A
S315080209A001F0004110EBD37041F100015EEA430EFB
S315080209B008BF20EAD37070BDC4F1200500FA05F21B
S315080209C04EEA020E20FA04F301FA05F243EA02039A
S315080209D021FA04F001F0004121FA04F220EA0200A9
S315080209E000EBD3705EEA430E08BF20EAD37070BDEF
S315080209F094F0000F0FD101F00046400041EB0101CF
S31508020A0011F4801F08BF013CF7D041EA060195F0B0
S31508020A10000F18BF704703F00046520043EB03036A
S31508020A2013F4801F08BF013DF7D043EA0603704757
S31508020A3094EA0C0F0CEA135518BF95EA0C0F0CD062
S31508020A4050EA410618BF52EA4306D1D181EA0301A8
S31508020A5001F000414FF0000070BD50EA410606BFA2
S31508020A601046194652EA430619D094EA0C0F02D1E7
S31508020A7050EA013613D195EA0C0F05D152EA03362C
S31508020A801CBF104619460AD181EA030101F000414A
S31508020A9041F0FE4141F470014FF0000070BD41F093
S31508020AA0FE4141F4780170BD70B54FF0FF0C4CF46D
S31508020AB0E06C1CEA11541DBF1CEA135594EA0C0F8C
S31508020AC095EA0C0F00F0A7F8A4EB050481EA030ED9
S31508020AD052EA03354FEA013100F088804FEA0333C0
S31508020AE04FF0805545EA131343EA12634FEA02228E
S31508020AF045EA111545EA10654FEA00260EF000414F
S31508020B009D4208BF964244F1FD0404F5407402D2A0
S31508020B105B084FEA3202B61A65EB03055B084FEA31
S31508020B2032024FF480104FF4002CB6EB020E75EB2E
S31508020B30030E22BFB61A754640EA0C005B084FEA56
S31508020B403202B6EB020E75EB030E22BFB61A7546D3
S31508020B5040EA5C005B084FEA3202B6EB020E75EB1E
S31508020B60030E22BFB61A754640EA9C005B084FEA96
S31508020B703202B6EB020E75EB030E22BFB61A7546A3
S31508020B8040EADC0055EA060E18D04FEA051545EA92
S31508020B9016754FEA06164FEAC30343EA52734FEA3B
S31508020BA0C2025FEA1C1CC0D111F4801F0BD141EAB4
S31508020BB000014FF000004FF0004CB6E711F4801F19
S31508020BC004BF01430020B4F1FD0C88BFBCF5E06FF9
S31508020BD03FF6AFAEB5EB030C04BFB6EB020C5FEA09
S31508020BE0500C50F1000041EB045170BD0EF0004E5E
S31508020BF04EEA113114EB5C04C2BFD4EB0C0541EA90
S31508020C00045170BD41F480114FF0000E013C90E68C
S31508020C1045EA060E8DE60CEA135594EA0C0F08BF50
S31508020C2095EA0C0F3FF43BAF94EA0C0F0AD150EA4F
S31508020C3001347FF434AF95EA0C0F7FF425AF1046E2
S31508020C4019462CE795EA0C0F06D152EA03353FF40A
S31508020C50FDAE1046194622E750EA410618BF52EA87
S31508020C6043067FF4C5AE50EA41047FF40DAF52EA5B
S31508020C7043057FF4EBAE12E74FF0FF3C06E000BFF8
S31508020C804FF0010C02E000BF4FF0010C4DF804CD05
S31508020C904FEA410C7FEA6C5C4FEA430C18BF7FEAC5
S31508020CA06C5C1BD001B050EA410C0CBF52EA430CF3
S31508020CB091EA030F02BF90EA020F0020704710F173
S31508020CC0000F91EA030F58BF994208BF90422CBF02
S31508020CD0D8176FEAE37040F0010070474FEA410CFB
S31508020CE07FEA6C5C02D150EA013C07D14FEA430C19
S31508020CF07FEA6C5CD6D152EA033CD3D05DF8040B8A
S31508020D00704700BF8446104662468C4619466346BB
S31508020D1000E000BF01B5FFF7B7FF002848BF10F192
S31508020D20000F01BD4DF808EDFFF7F4FF0CBF0120D7
S31508020D3000205DF808FB00BF4DF808EDFFF7EAFF53
S31508020D4034BF012000205DF808FB00BF4DF808ED0E
S31508020D50FFF7E0FF94BF012000205DF808FB00BF03
S31508020D604DF808EDFFF7CEFF94BF012000205DF88D
S31508020D7008FB00BF4DF808EDFFF7C4FF34BF01209A
S31508020D8000205DF808FB00BF4FEA410C7FEA6C5C65
S31508020D9002D150EA013C0AD14FEA430C7FEA6C5C65
S31508020DA002D152EA033C02D14FF0000070474FF0DD
S31508020DB0010070474FEA410212F5001215D211D509
S31508020DC06FF47873B3EB625212D94FEAC12343F038
S31508020DD0004343EA505311F0004F23FA02F018BFBA
S31508020DE0404270474FF00000704750EA013005D183
S31508020DF011F0004008BF6FF0004070474FF0000046
S31508020E00704700BF4A0011D212F5001211D20DD551
S31508020E106FF47873B3EB62520ED44FEAC12343F0F0
S31508020E20004343EA505323FA02F070474FF000009A
S31508020E30704750EA013002D14FF0FF3070474FF049
S31508020E40000070474FEA4102B2F1E04324BFB3F50E
S31508020E50001CDCF1FE5C0DD901F0004C4FEAC00221
S31508020E604CEA5070B2F1004F40EB830008BF20F005
S31508020E700100704711F0804F21D113F13872BCBFBF
S31508020E8001F00040704741F480114FEA5252C2F114
S31508020E901802C2F1200C10FA0CF320FA02F018BF5D
S31508020EA040F001004FEAC1234FEAD32303FA0CFCB0
S31508020EB040EA0C0023FA02F34FEA4303CCE77FEA3F
S31508020EC0625307D150EA01331EBF4FF0FE4040F489
S31508020ED04000704701F0004040F0FE4040F4000038
S31508020EE0704700BF53B94AB9002908BF00281CBF7A
S31508020EF04FF0FF314FF0FF3000F0B4B9ADF1080CF6
S31508020F006DE904CE00F03CF8DDF804E0DDE90223E1
S31508020F1004B0704738B50022002304460D46FFF791
S31508020F200BFF28B920462946BDE8384000F00AB822
S31508020F30204605F1004100F005F8404261EB410107
S31508020F4038BD00BFD0B500220B4B06460F46FFF749
S31508020F5081FCFFF757FF0446FFF702FC0022074B06
S31508020F60FFF778FC02460B4630463946FFF7BAFACF
S31508020F70FFF748FF2146D0BD0000F03D0000F041D2
S31508020F802DE9F04F099D0C46002B4DD18A420F469A
S31508020F9084469646B2FA82F360D94BB102FA03FE48
S31508020FA0C3F120029F4000FA03FC20FA02F217431B
S31508020FB04FEA1E461FFA8EF44FEA1C42B7FBF6F1B9
S31508020FC006FB117701FB04F042EA0742904208D970
S31508020FD01EEB020201F1FF3702D2904200F22D8186
S31508020FE03946121A1FFA8CFCB2FBF6F006FB1022DF
S31508020FF000FB04F44CEA024C644508D91EEB0C0CBF
S3150802100000F1FF3202D2644500F21A81104640EA24
S315080210100140ACEB040C002125B12CFA03F30022A3
S31508021020C5E90032BDE8F08F8B4205D90DB1C5E995
S31508021030000100210846F5E7B3FA83F100294DD1EC
S31508021040A342C0F0F280904280F0EF800646234623
S315080210500846002DE6D0C5E90063E3E7002B40F019
S31508021060A2808A1A4FEA1E471FFA8EF60121B2FBA0
S31508021070F7F407FB14204FEA1C4242EA004206FB39
S3150802108004F090420FD91EEB020204F1FF382CBF7E
S315080210904FF001094FF00009904203D9B9F1000F48
S315080210A000F0C8804446121A1FFA8CFCB2FBF7F00D
S315080210B007FB102200FB06F64CEA024C664508D9E5
S315080210C01EEB0C0C00F1FF3202D2664500F2BB8021
S315080210D01046ACEB060C40EA04409DE7C1F1200637
S315080210E08B4004FA01FE22FA06F720FA06FCF440BF
S315080210F08A401F434EEA0C0300FA01FE4FEA1748DC
S315080211004FEA13491FFA87FCB4FBF8F008FB1044B0
S3150802111049EA044400FB0CF9A1450ED93C1900F131
S31508021120FF3A2CBF4FF0010B4FF0000BA14503D934
S31508021130BBF1000F00F093805046A4EB09041FFA96
S3150802114083F9B4FBF8F308FB134403FB0CFC49EAE6
S315080211500444A44506D93C1903F1FF3801D2A44533
S315080211607AD8434643EA0040A4EB0C04A0FB029853
S315080211704445CC46434602D306D1CE4504D201386D
S31508021180B9EB020C68EB07035DB1BEEB0C0264EB2C
S31508021190030404FA06F622FA01F3CC401E43C5E913
S315080211A0006400213EE702FA03FEC3F1200104FAB5
S315080211B003F200FA03FCCC404FEA1E4720FA01F17B
S315080211C01FFA8EF6B4FBF7F00A4307FB1044110C1C
S315080211D041EA044100FB06F48C420ED91EEB0101DA
S315080211E000F1FF382CBF4FF001094FF000098C427D
S315080211F002D9B9F1000F2CD04046091B92B2B1FBB5
S31508021200F7F407FB141142EA014204FB06F1914284
S3150802121007D91EEB020204F1FF3801D2914215D812
S315080212204446521A44EA004121E7861A64EB03034C
S3150802123001200EE7023C724435E702397244D0E6D1
S31508021240F4440238E3E6F444023842E7023C7244C4
S31508021250E7E702387144D0E7023B3C4482E70238AA
S315080212603C446AE7704700BF80B586B002AF786033
S315080212700023FB60342300934FF448430B4A0C497E
S315080212800C4829F073F90346002B0AD1094BBB60B7
S31508021290B86803F049F9F860FB68002B01D000BF73
S315080212A0FDE700BF1037BD4680BD00BF70140020A1
S315080212B03069050870DC002080B483B000AF0346AD
S315080212C0FB71044AFB79137000BF0C37BD465DF803
S315080212D0047B704785F2002080B400AF034B1B786D
S315080212E01846BD465DF8047B704700BF85F20020AC
S315080212F080B500AF02481CF069FB00BF80BD00BF85
S315080213004469050880B586B000AFF8600B467A6076
S31508021310FB720023FB752D481CF058FB0023FB7556
S315080213204CE0FB7D2A4A4FF48E7101FB03F313440A
S315080213301B78012B3FD1FB7D4FF48E7202FB03F320
S31508021340234A13440233194622481CF03FFB22481B
S315080213501CF03CFBFB7D4FF48E7202FB03F3183341
S315080213601B4A1344043319461A481CF02FFB1B4820
S315080213701CF02CFBFB7D164A4FF48E7101FB03F31E
S3150802138013449C331B782D2B12D015481CF01EFBD8
S31508021390FB7D4FF48E7202FB03F398330C4A134417
S315080213A0043319460B481CF011FB0C481CF00EFBC3
S315080213B00A481CF00BFBFB7D0133FB75FB7D0E2BEC
S315080213C0AFD900BF00BF1837BD4680BD58690508AA
S315080213D000000020806905088469050888690508EF
S315080213E08C69050880B584B000AFF8600B467A6050
S315080213F0FB7217F09FFA0346184617F0F8FA00BF71
S315080214001037BD4680BD000080B586B000AFF860D3
S315080214100B467A60FB720023FB750023BB757B685B
S3150802142003F500730422CA49184631F0B3FF03468E
S31508021430002B08D17B6803F500731846FFF746F8B8
S315080214400346042B13D07B6803F500730322C149B4
S31508021450184631F09FFF0346002B23D17B6803F51C
S3150802146000731846FFF732F80346032B1AD1BA4817
S315080214701CF0ACFA06F010F92EF0ECFF03461846FB
S315080214802FF024F80346002118462CF027FF2EF0E9
S31508021490E1FF034618462FF019F8034618462CF0C2
S315080214A0E0FF9BE17B6803F500730222AB4918460D
S315080214B031F070FF0346002B40F08D817B6803F5FF
S315080214C000731846FFF702F80346022B40F08381A1
S315080214D0FB7A032B40F27F817B6803F5806318460B
S315080214E030F04EFE0346FB757B6803F5006318462B
S315080214F030F046FE0346BB75FB7D002B00F0668185
S31508021500FB7D0E2B00F26281FB7D194694481CF086
S315080215105DFA2EF09FFF034618462EF0D7FF0346C4
S31508021520032118462CF0DAFE7B6803F5C0631A78A5
S315080215308C4B1B78D31A002B40F096807B6803F5F8
S31508021540C0631846FEF7C2FF0346012B40F08C80A3
S3150802155085481CF03BFAFB7D013B0D2B00F282808D
S3150802156001A252F823F000BFA1150208AF1502081E
S31508021570BD150208CB150208D9150208E715020897
S31508021580F515020803160208111602081F160208A4
S315080215902D1602083B1602084916020857160208B3
S315080215A0BB7D1A460121332006F058F85BE0BB7D65
S315080215B01A460121342006F051F854E0BB7D1A463A
S315080215C00121352006F04AF84DE0BB7D1A46012175
S315080215D0362006F043F846E0BB7D1A46012137203D
S315080215E006F03CF83FE0BB7D1A460121382006F09A
S315080215F035F838E0BB7D1A460121392006F02EF867
S3150802160031E0BB7D1A4601213A2006F027F82AE086
S31508021610BB7D1A4601213B2006F020F823E0BB7D5C
S315080216201A4601213C2006F019F81CE0BB7D1A4631
S3150802163001213D2006F012F815E0BB7D1A4601216C
S315080216403E2006F00BF80EE0BB7D1A4601213F202C
S3150802165006F004F807E0BB7D1A460121402005F092
S31508021660FDFF00E000BFB0E07B6803F5C0631A78AF
S315080216703E4B1B78D31A002B40F0AB807B6803F5F0
S31508021680C0631846FEF722FF0346012B40F0A180ED
S3150802169037481CF09BF9FB7D013B0D2B00F2948029
S315080216A001A252F823F000BFE1160208EF1602085B
S315080216B0FD1602080B17020819170208271702084F
S315080216C03517020843170208751702088317020816
S315080216D0911702089F170208AD170208BB170208DE
S315080216E0BB7D1A460221332005F0B8FF6DE0BB7DAB
S315080216F01A460221342005F0B1FF66E0BB7D1A4680
S315080217000221352005F0AAFF5FE0BB7D1A460221B9
S31508021710362005F0A3FF58E0BB7D1A460221372082
S3150802172005F09CFF51E0BB7D1A460221382005F0E0
S3150802173095FF4AE0BB7D1A460221392005F08EFF45
S3150802174043E0BB7D1A4602213A2005F087FF3CE0BA
S3150802175098690508A0690508A4690508B86905080D
S31508021760BC690508C8690508CC690508DC69050865
S31508021770E0690508BB7D1A4602213B2005F06EFF8B
S3150802178023E0BB7D1A4602213C2005F067FF1CE0D8
S31508021790BB7D1A4602213D2005F060FF15E0BB7DA0
S315080217A01A4602213E2005F059FF0EE0BB7D1A4675
S315080217B002213F2005F052FF07E0BB7D1A460221AF
S315080217C0402005F04BFF00E000BF02E0FFF790FD66
S315080217D004E000BF02E0FFF78BFD00BF1837BD46E5
S315080217E080BD00BF80B588B002AFF8600B467A604C
S315080217F0FB7200237B750123FB7500233B750023CF
S31508021800BB75FB7A042B40F250817B6803F50073A3
S31508021810184630F0B5FC03467B757B6803F5C06352
S31508021820184630F0ADFC0346A24A82FB0312521157
S31508021830DB17D31A3B757B7D19469F481CF0C6F801
S315080218407B6803F580631A789C4B1B78D31A002BA6
S3150802185013D17B6803F580631846FEF737FE034605
S31508021860012B0AD13B7D642202FB03F319469448F5
S315080218701CF0ACF80123FB751BE07B6803F580635B
S315080218801A78904B1B78D31A002B12D17B6803F572
S3150802189080631846FEF71AFE0346012B09D13B7DE3
S315080218A0642202FB03F3194687481CF08FF80223C9
S315080218B0FB757B6803F500631A78844B1B78D31A89
S315080218C0002B0ED17B6803F500631846FEF7FEFD72
S315080218D00346012B05D17E481CF078F80123BB7517
S315080218E019E07B6803F500631A787A4B1B78D31ADA
S315080218F0002B0ED17B6803F500631846FEF7E6FD5A
S315080219000346012B05D174481CF060F80023BB7509
S3150802191001E00023BB752EF09DFD034618462EF006
S31508021920D5FD0346032118462CF0D8FC7B7D013BE6
S315080219300D2B00F2B98001A252F823F0751902089C
S315080219408B190208A1190208B7190208CD1902084B
S31508021950E3190208F91902080F1A0208251A0208D9
S315080219603B1A0208511A0208671A02087D1A020867
S31508021970931A0208594B1B78B87D3A7DF97D009374
S315080219800346332005F09EFE8FE0544B1B78B87D44
S315080219903A7DF97D00930346342005F093FE84E0F0
S315080219A04E4B1B78B87D3A7DF97D00930346352068
S315080219B005F088FE79E0494B1B78B87D3A7DF97DBA
S315080219C000930346362005F07DFE6EE0434B1B78F6
S315080219D0B87D3A7DF97D00930346372005F072FEFD
S315080219E063E03E4B1B78B87D3A7DF97D009303464A
S315080219F0382005F067FE58E0384B1B78B87D3A7DEB
S31508021A00F97D00930346392005F05CFE4DE0334B21
S31508021A101B78B87D3A7DF97D009303463A2005F096
S31508021A2051FE42E02D4B1B78B87D3A7DF97D009335
S31508021A3003463B2005F046FE37E0284B1B78B87D67
S31508021A403A7DF97D009303463C2005F03BFE2CE0E7
S31508021A50224B1B78B87D3A7DF97D009303463D20DB
S31508021A6005F030FE21E01D4B1B78B87D3A7DF97DE5
S31508021A70009303463E2005F025FE16E0174B1B7819
S31508021A80B87D3A7DF97D009303463F2005F01AFE9C
S31508021A900BE0124B1B78B87D3A7DF97D009303461D
S31508021AA0402005F00FFE00E000BF00BF1837BD4614
S31508021AB080BD00BF1F85EB51F0690508C869050896
S31508021AC0006A0508DC690508106A0508206A05081F
S31508021AD0246A0508306A0508346A050885F2002072
S31508021AE080B588B002AFF8600B467A60FB720023B5
S31508021AF0BB7500237B7500233B750023FB7400230B
S31508021B00FB757B6803F500730422B249184631F067
S31508021B1041FC0346002B08D17B6803F5007318467F
S31508021B20FEF7D4FC0346042B13D07B6803F5007337
S31508021B300322A949184631F02DFC0346002B23D16E
S31508021B407B6803F500731846FEF7C0FC0346032BB1
S31508021B501AD1A2481BF03AFF05F09EFD2EF07AFC38
S31508021B60034618462EF0B2FC0346002118462CF00E
S31508021B70B5FB2EF06FFC034618462EF0A7FC03466B
S31508021B8018462CF06EFC6EE1FB7A052B40F26B814F
S31508021B907B6803F58063184630F0F2FA0346BB7594
S31508021BA07B6803F5C063184630F0EAFA03467B758C
S31508021BB07B6803F50063184630F0E2FA03463B7584
S31508021BC07B6803F52063184630F0DAFA0346FB749D
S31508021BD0B97D7A7D387DFB7C0093034680481BF0ED
S31508021BE0F5FE7B6803F540631A787E4B1B78D31A99
S31508021BF0002B0ED17B6803F540631846FEF766FC98
S31508021C000346012B05D178481BF0E0FE0123FB753C
S31508021C1019E07B6803F540631A78744B1B78D31A6C
S31508021C20002B0ED17B6803F540631846FEF74EFC7F
S31508021C300346012B05D16E481BF0C8FE0023FB752F
S31508021C4001E00023FB757B6803F5007302226949EC
S31508021C50184631F09FFB0346002B40F004817B684F
S31508021C6003F500731846FEF731FC0346022B40F0D3
S31508021C70FA802EF0EFFB034618462EF027FC0346A1
S31508021C80032118462CF02AFBBB7D013B0D2B00F2E3
S31508021C90E98001A252F823F0D11C0208EB1C0208C3
S31508021CA0051D02081F1D0208391D0208531D0208D8
S31508021CB06D1D0208871D0208A11D0208BB1D020828
S31508021CC0FD1D0208171E0208311E02084B1E0208D5
S31508021CD0494B1B78F87C3A7D797D0193FB7D00930D
S31508021CE00346332006F078FABDE0434B1B78F87CAE
S31508021CF03A7D797D0193FB7D00930346342006F0F5
S31508021D006BFAB0E03C4B1B78F87C3A7D797D0193FF
S31508021D10FB7D00930346352006F05EFAA3E0364BB8
S31508021D201B78F87C3A7D797D0193FB7D0093034607
S31508021D30362006F051FA96E02F4B1B78F87C3A7D4E
S31508021D40797D0193FB7D00930346372006F044FA1A
S31508021D5089E0294B1B78F87C3A7D797D0193FB7DD6
S31508021D6000930346382006F037FA7CE0224B1B78AC
S31508021D70F87C3A7D797D0193FB7D009303463920F1
S31508021D8006F02AFA6FE01C4B1B78F87C3A7D797DBF
S31508021D900193FB7D009303463A2006F01DFA62E0A2
S31508021DA0154B1B78F87C3A7D797D0193FB7D009370
S31508021DB003463B2006F010FA55E00F4B1B78F87CD9
S31508021DC03A7D797D0193FB7D009303463C2006F01C
S31508021DD003FA48E098690508A0690508A469050890
S31508021DE0446A0508206A0508246A0508306A05084F
S31508021DF0346A0508B869050885F200201C4B1B7869
S31508021E00F87C3A7D797D0193FB7D009303463D205C
S31508021E1006F0E2F927E0164B1B78F87C3A7D797DC5
S31508021E200193FB7D009303463E2006F0D5F91AE09E
S31508021E300F4B1B78F87C3A7D797D0193FB7D0093E5
S31508021E4003463F2006F0C8F90DE0094B1B78F87CDB
S31508021E503A7D797D0193FB7D00930346402006F087
S31508021E60BBF900E000BF00BF1837BD4680BD00BF02
S31508021E7085F2002080B584B000AFF8600B467A6020
S31508021E80FB7243481BF0A2FD16F054FD03461846A2
S31508021E9016F0D4FD10EE103A1846FEF783FC0246F9
S31508021EA00B463C481BF092FD16F044FD03461846C5
S31508021EB016F0E2FD10EE103A1846FEF773FC0246DB
S31508021EC00B4635481BF082FD16F034FD03461846CC
S31508021ED016F0F0FD10EE103A1846FEF763FC0246BD
S31508021EE00B462E481BF072FD16F024FD03461846D3
S31508021EF016F0FEFD10EE103A1846FEF753FC02469F
S31508021F000B4627481BF062FD16F014FD03461846D9
S31508021F1016F00CFE10EE103A1846FEF743FC02467F
S31508021F200B4620481BF052FD16F004FD03461846E0
S31508021F3016F01AFE10EE103A1846FEF733FC024661
S31508021F400B4619481BF042FD16F0F4FC03461846E8
S31508021F5016F028FE10EE103A1846FEF723FC024643
S31508021F600B4612481BF032FD16F0E4FC03461846EF
S31508021F7016F036FE10EE103A1846FEF713FC024625
S31508021F800B460B481BF022FD00BF1037BD4680BD2D
S31508021F90786A05089C6A0508B86A0508D46A0508B5
S31508021FA0F06A05080C6B0508286B0508446B0508DA
S31508021FB0606B050880B5D6B002AF07F5A873A3F51E
S31508021FC0A273186007F5A873A3F5A6731A6007F536
S31508021FD0A873A3F245130A461A70002387F84F31ED
S31508021FE0002387F84E31002387F84D31002387F8FE
S31508021FF04C3107F5A873A3F245131B78012B41F25E
S31508022000508007F5A873A3F5A6731B6803F500733A
S315080220100622D249184631F0BDF90346002B18D1DB
S3150802202007F5A873A3F5A6731B6803F5007318468C
S31508022030FEF74CFA0346062B0BD1C9481BF0C6FC21
S31508022040FFF74AF903461946012009F055FD01F042
S3150802205028B807F5A873A3F5A6731B6803F50073DA
S315080220600322C049184631F095F90346002B16D1CA
S3150802207007F5A873A3F5A6731B6803F5007318463C
S31508022080FEF724FA0346032B09D1B7481BF09EFC38
S3150802209000220421B5481DF055FC01F002B807F5E7
S315080220A0A873A3F5A6731B6803F500730222B04949
S315080220B0184631F06FF90346002B16D107F5A873B7
S315080220C0A3F5A6731B6803F500731846FEF7FEF917
S315080220D00346022B09D1A7481BF078FC01220421EA
S315080220E0A2481DF02FFC00F0DCBF07F5A873A3F584
S315080220F0A6731B6803F5007304229F49184631F03C
S3150802210049F90346002B13D107F5A873A3F5A6735D
S315080221101B6803F500731846FEF7D8F90346042B25
S3150802212006D10AF045F995481BF050FC00F0B9BFF4
S3150802213007F5A873A3F5A6731B6803F500730622B1
S315080221408F49184631F026F90346002B0CD107F5BC
S31508022150A873A3F5A6731B6803F500731846FEF762
S31508022160B5F90346062B1BD007F5A873A3F5A67384
S315080221701B6803F5007303228249184631F00AF9EF
S315080221800346002B13D107F5A873A3F5A6731B689C
S3150802219003F500731846FEF799F90346032B06D191
S315080221A00AF0A6F878481BF011FC00F07ABF07F58A
S315080221B0A873A3F5A6731B6803F500730522734972
S315080221C0184631F0E7F80346002B40F0038107F57D
S315080221D0A873A3F5A6731B6803F500731846FEF7E2
S315080221E075F90346052B40F0F58007F5A873A3F2A7
S315080221F045131B78032B40F2E78007F5A873A3F56E
S31508022200A6731B6803F5806318462FF0B9FF0346C9
S3150802221087F84E3107F5A873A3F5A6731B6803F56D
S31508022220C06302225249184631F0B4F80346002B1D
S3150802223010D107F5A873A3F5A6731B6803F5C06347
S315080222401846FEF743F90346022B03D1012387F802
S315080222504F311EE007F5A873A3F5A6731B6803F5AD
S31508022260C06303223F49184631F094F80346002B0F
S315080222700FD107F5A873A3F5A6731B6803F5C06308
S315080222801846FEF723F90346032B02D1002387F8E3
S315080222904F3197F84E31013B062B00F2928001A28C
S315080222A052F823F0C1220208DB220208F5220208AC
S315080222B00F2302082923020843230208A923020836
S315080222C097F84F31194601200AF09CFA97F84F31D0
S315080222D019462F481BF07AFB7AE097F84F311946D0
S315080222E002200AF08FFA97F84F31194629481BF04F
S315080222F06DFB6DE097F84F31194603200AF082FA12
S3150802230097F84F31194624481BF060FB60E097F8AE
S315080223104F31194604200AF075FA97F84F311946D3
S315080223201E481BF053FB53E097F84F311946052018
S315080223300AF068FA97F84F31194619481BF046FB16
S3150802234046E097F84F31194606200AF05BFA97F8E5
S315080223504F31194613481BF039FB39E07C6B0508E7
S31508022360846B0508A0690508986B050800100242E7
S31508022370B8690508A86B050898690508B86B0508C1
S31508022380D06B0508D86B0508DC6B0508F86B0508E1
S31508022390006C0508146C0508286C05083C6C0508D1
S315080223A0546C05086C6C050897F84F3119460720D6
S315080223B00AF028FA97F84F311946AC481BF006FB83
S315080223C006E0FEF795FF03E0FEF792FF00F069BE0E
S315080223D000F067BE07F5A873A3F5A6731B6803F595
S315080223E000730622A249184630F0D4FF0346002B92
S315080223F07AD107F5A873A3F5A6731B6803F50073CC
S315080224001846FEF763F80346062B6DD107F5A8733F
S31508022410A3F245131B78032B60D907F5A873A3F516
S31508022420A6731B6803F5C06318462FF0A9FE034678
S3150802243087F84D3107F5A873A3F5A6731B6803F54C
S31508022440806304228B49184630F0A4FF0346002B0A
S3150802245018D107F5A873A3F5A6731B6803F580635D
S315080224601846FEF733F80346042B0BD197F84D317D
S31508022470184609F0E9FE97F84D3119467E481BF0D1
S31508022480A5FA2FE007F5A873A3F5A6731B6803F54B
S31508022490806303227949184630F07CFF0346002BF5
S315080224A018D107F5A873A3F5A6731B6803F580630D
S315080224B01846FEF70BF80346032B0BD197F84D3156
S315080224C0184609F0EBFE97F84D3119466C481BF091
S315080224D07DFA07E0FEF70CFF00F0E3BDFEF708FF02
S315080224E000F0DFBD00F0DDBD07F5A873A3F5A673FE
S315080224F01B6803F5007304226249184630F04AFF46
S315080225000346002B40F0C88007F5A873A3F5A67307
S315080225101B6803F500731846FDF7D8FF0346042B1C
S3150802252040F0BA8007F5A873A3F245131B78032B6C
S3150802253040F2958007F5A873A3F5A6731B6803F501
S31508022540C06302225049184630F024FF0346002B86
S3150802255010D107F5A873A3F5A6731B6803F5C06324
S315080225601846FDF7B3FF0346022B03D1012387F86A
S315080225704F311EE007F5A873A3F5A6731B6803F58A
S31508022580C06303224149184630F004FF0346002B74
S315080225900FD107F5A873A3F5A6731B6803F5C063E5
S315080225A01846FDF793FF0346032B02D1002387F84B
S315080225B04F3107F5A873A3F5A6731B6803F5806365
S315080225C004222C49184630F0E5FE0346002B19D1A1
S315080225D007F5A873A3F5A6731B6803F58063184667
S315080225E0FDF774FF0346042B0CD197F84F311946B1
S315080225F00B200AF007F997F84F31194624481BF0C1
S31508022600E5F930E007F5A873A3F5A6731B6803F589
S31508022610806303221949184630F0BCFE0346002B94
S3150802262019D107F5A873A3F5A6731B6803F580638A
S315080226301846FDF74BFF0346032B0CD197F84F318B
S3150802264019460C200AF0DEF897F84F311946114858
S315080226501BF0BCF907E0FEF74BFE00F022BDFEF7C1
S3150802266047FE00F01EBD00F01CBD00BF806C0508C9
S31508022670986C0508A06C0508A86C0508BC6C0508CA
S31508022680C06C0508D46C0508B8690508A069050870
S31508022690DC6C0508F06C050807F5A873A3F5A673A4
S315080226A01B6803F500730622C749184630F072FE06
S315080226B00346002B40F0F28407F5A873A3F5A67328
S315080226C01B6803F500731846FDF700FF0346062B41
S315080226D040F0E48407F5A873A3F245131B78042B8C
S315080226E040F2D78407F5A873A3F5A6731B6803F50A
S315080226F0206318462FF044FD034687F84C3197F8B5
S315080227004C31012B40F2C28497F84C31032B00F26C
S31508022710BD8407F5A873A3F5A6731B6803F5806342
S315080227200522AA49184630F035FE0346002B40F02A
S315080227308D8007F5A873A3F5A6731B6803F5806356
S315080227401846FDF7C3FE0346052B7FD107F5A87386
S31508022750A3F5A6731B6803F5C06305229C491846B0
S3150802276030F018FE0346002B17D107F5A873A3F518
S31508022770A6731B6803F5C0631846FDF7A7FE034652
S31508022780052B0AD197F84C3107F114000022009262
S315080227900022012109F036FE4CE007F5A873A3F5DD
S315080227A0A6731B6803F5C06305228A49184630F0EA
S315080227B0F1FD0346002B17D107F5A873A3F5A673F7
S315080227C01B6803F5C0631846FDF780FE0346052B12
S315080227D00AD197F84C3107F1140000220092002220
S315080227E0022109F00FFE25E007F5A873A3F5A673E3
S315080227F01B6803F5C06306227749184630F0CAFDFE
S315080228000346002B16D107F5A873A3F5A6731B6812
S3150802281003F5C0631846FDF759FE0346062B09D190
S3150802282097F84C3107F11400002200920022032186
S3150802283009F0E8FD97F84C3107F1140000220092DE
S315080228400022FF2109F0DEFD00F01FBC07F5A87380
S31508022850A3F5A6731B6803F5806304225F4918462D
S3150802286030F098FD0346002B40F0088207F5A8735E
S31508022870A3F5A6731B6803F580631846FDF726FEC3
S315080228800346042B40F0FA8107F5A873A3F5A6734D
S315080228901B6803F5C06304225149184630F07AFDD5
S315080228A00346002B40F0F18007F5A873A3F5A6733B
S315080228B01B6803F5C0631846FDF708FE0346042B9A
S315080228C040F0E38007F5A873A3F5A6731B6803F522
S315080228D0006305224349184630F05CFD0346002B87
S315080228E00CD107F5A873A3F5A6731B6803F5006355
S315080228F01846FDF7EBFD0346052B19D007F5A87315
S31508022900A3F5A6731B6803F500631A78364B1B7882
S31508022910D31A002B17D107F5A873A3F5A6731B685C
S3150802292003F500631846FDF7D1FD0346012B0AD1CC
S3150802293097F84C3107F11400002200920022042174
S3150802294009F060FD96E007F5A873A3F5A6731B6860
S3150802295003F5006306222549184630F01BFD034697
S31508022960002B0CD107F5A873A3F5A6731B6803F50C
S3150802297000631846FDF7AAFD0346062B19D007F58C
S31508022980A873A3F5A6731B6803F500631A78184B98
S315080229901B78D31A002B2DD107F5A873A3F5A673B6
S315080229A01B6803F500631846FDF790FD0346012BE5
S315080229B020D197F84C3107F1140000220092002228
S315080229C0052109F01FFD55E0006D0508086D05088B
S315080229D0106D0508186D0508206D0508286D05088F
S315080229E0306D0508386D0508406D0508446D050803
S315080229F04C6D050807F5A873A3F5A6731B6803F5BE
S31508022A00006305229649184630F0C4FC0346002B9B
S31508022A100CD107F5A873A3F5A6731B6803F5006323
S31508022A201846FDF753FD0346052B19D007F5A8737B
S31508022A30A3F5A6731B6803F500631A78894B1B78FE
S31508022A40D31A002B16D107F5A873A3F5A6731B682C
S31508022A5003F500631846FDF739FD0346012B09D134
S31508022A6097F84C3107F11400002200920022062141
S31508022A7009F0C8FC97F84C3107F1140000220092BD
S31508022A800022FF2109F0BEFCFEE207F5A873A3F5B2
S31508022A90A6731B6803F5C06303227349184630F010
S31508022AA079FC0346002B40F0EF8207F5A873A3F5DD
S31508022AB0A6731B6803F5C0631846FDF707FD0346B0
S31508022AC0032B40F0E18207F5A873A3F5A6731B68EA
S31508022AD003F5006305226549184630F05BFC034698
S31508022AE0002B0CD107F5A873A3F5A6731B6803F58B
S31508022AF000631846FDF7EAFC0346052B19D007F5CD
S31508022B00A873A3F5A6731B6803F500631A78584BD6
S31508022B101B78D31A002B17D107F5A873A3F5A6734A
S31508022B201B6803F500631846FDF7D0FC0346012B24
S31508022B300AD197F84C3107F11400002200920022BC
S31508022B40072109F05FFC80E007F5A873A3F5A673D1
S31508022B501B6803F5006306224649184630F01AFC3C
S31508022B600346002B0CD107F5A873A3F5A6731B68B9
S31508022B7003F500631846FDF7A9FC0346062B19D090
S31508022B8007F5A873A3F5A6731B6803F500631A78FD
S31508022B90394B1B78D31A002B17D107F5A873A3F55F
S31508022BA0A6731B6803F500631846FDF78FFC0346F8
S31508022BB0012B0AD197F84C3107F114000022009232
S31508022BC00022082109F01EFC3FE007F5A873A3F5C9
S31508022BD0A6731B6803F5006305222149184630F0DF
S31508022BE0D9FB0346002B0CD107F5A873A3F5A673E8
S31508022BF01B6803F500631846FDF768FC0346052BB8
S31508022C0019D007F5A873A3F5A6731B6803F5006325
S31508022C101A78144B1B78D31A002B16D107F5A8730A
S31508022C20A3F5A6731B6803F500631846FDF74EFC69
S31508022C300346012B09D197F84C3107F114000022FB
S31508022C4000920022092109F0DDFB97F84C3107F1C1
S31508022C501400002200920022FF2109F0D3FB13E29E
S31508022C60506D0508586D05085C6D0508386D050830
S31508022C70406D0508446D05084C6D050807F5A873EF
S31508022C80A3F5A6731B6803F580630422AF491846A9
S31508022C9030F080FB0346002B40F0FE8107F5A8734F
S31508022CA0A3F5A6731B6803F580631846FDF70EFCA9
S31508022CB00346042B40F0F08107F5A873A3F5A67323
S31508022CC01B6803F5C0630422A149184630F062FB6B
S31508022CD00346002B40F0DB8007F5A873A3F5A6731D
S31508022CE01B6803F5C0631846FDF7F0FB0346042B81
S31508022CF040F0CD8007F5A873A3F5A6731B6803F504
S31508022D00006305229349184630F044FB0346002B1C
S31508022D100CD107F5A873A3F5A6731B6803F5006320
S31508022D201846FDF7D3FB0346052B19D007F5A873FA
S31508022D30A3F5A6731B6803F500631A78864B1B78FE
S31508022D40D31A002B17D107F5A873A3F5A6731B6828
S31508022D5003F500631846FDF7B9FB0346012B0AD1B2
S31508022D6097F84C3107F114000022009200220A213A
S31508022D7009F048FB80E007F5A873A3F5A6731B685C
S31508022D8003F5006306227549184630F003FB03462D
S31508022D90002B0CD107F5A873A3F5A6731B6803F5D8
S31508022DA000631846FDF792FB0346062B19D007F572
S31508022DB0A873A3F5A6731B6803F500631A78684B14
S31508022DC01B78D31A002B17D107F5A873A3F5A67398
S31508022DD01B6803F500631846FDF778FB0346012BCB
S31508022DE00AD197F84C3107F114000022009200220A
S31508022DF00B2109F007FB3FE007F5A873A3F5A673B5
S31508022E001B6803F5006305225649184630F0C2FAD4
S31508022E100346002B0CD107F5A873A3F5A6731B6806
S31508022E2003F500631846FDF751FB0346052B19D037
S31508022E3007F5A873A3F5A6731B6803F500631A784A
S31508022E40494B1B78D31A002B16D107F5A873A3F59D
S31508022E50A6731B6803F500631846FDF737FB03469E
S31508022E60012B09D197F84C3107F114000022009280
S31508022E7000220C2109F0C6FA97F84C3107F1140022
S31508022E80002200920022FF2109F0BCFAFDE007F5B4
S31508022E90A873A3F5A6731B6803F5C0630322334917
S31508022EA0184630F077FA0346002B40F0F58007F50E
S31508022EB0A873A3F5A6731B6803F5C0631846FDF746
S31508022EC005FB0346032B40F0E78007F5A873A3F535
S31508022ED0A6731B6803F5006305221E49184630F0DF
S31508022EE059FA0346002B0CD107F5A873A3F5A67366
S31508022EF01B6803F500631846FDF7E8FA0346052B37
S31508022F0019D007F5A873A3F5A6731B6803F5006322
S31508022F101A78114B1B78D31A002B29D107F5A873F7
S31508022F20A3F5A6731B6803F500631846FDF7CEFAE8
S31508022F300346012B1CD197F84C3107F114000022E5
S31508022F40009200220D2109F05DFA92E0A06C0508B4
S31508022F50306D0508386D0508406D0508446D05088D
S31508022F604C6D0508506D0508586D05085C6D050819
S31508022F7007F5A873A3F5A6731B6803F50063062273
S31508022F804A49184630F006FA0346002B0CD107F5D3
S31508022F90A873A3F5A6731B6803F500631846FDF725
S31508022FA095FA0346062B19D007F5A873A3F5A67357
S31508022FB01B6803F500631A783D4B1B78D31A002B5E
S31508022FC017D107F5A873A3F5A6731B6803F5006363
S31508022FD01846FDF77BFA0346012B0AD197F84C31BE
S31508022FE007F114000022009200220E2109F00AFAC3
S31508022FF03FE007F5A873A3F5A6731B6803F50063FC
S3150802300005222C49184630F0C5F90346002B0CD187
S3150802301007F5A873A3F5A6731B6803F5006318469C
S31508023020FDF754FA0346052B19D007F5A873A3F53D
S31508023030A6731B6803F500631A781F4B1B78D31A0D
S31508023040002B16D107F5A873A3F5A6731B6803F51B
S3150802305000631846FDF73AFA0346012B09D197F899
S315080230604C3107F114000022009200220F2109F0C8
S31508023070C9F997F84C3107F1140000220092002290
S31508023080FF2109F0BFF907E000BF05E0FEF730F9B6
S3150802309007E0FEF72DF904E000BF02E0FEF728F983
S315080230A000BF07F5A877BD4680BD00BF446D050879
S315080230B04C6D0508506D0508586D050890B58BB01E
S315080230C000AFF8600B467A60FB7200237B6200232E
S315080230D03B620023FB610023BB6100237B617B68A3
S315080230E003F500731A78B64B1B78D31A002B10D146
S315080230F07B6803F500731846FDF7E8F90346012BCA
S3150802310007D1B0481AF062FCAF481AF05FFC00F02B
S3150802311086BD7B6803F500730322AC49184630F076
S3150802312039F90346002B08D17B6803F50073184664
S31508023130FDF7CCF90346032B15D07B6803F500731C
S315080231400722A349184630F025F90346002B40F01A
S3150802315063857B6803F500731846FDF7B7F90346DE
S31508023160072B40F059857B6803F580631A78944BE0
S315080231701B78D31A002B25D17B6803F58063184682
S31508023180FDF7A4F90346012B1CD192481AF01EFC3E
S3150802319091481AF01BFC91481AF018FC90481AF04C
S315080231A015FC90481AF012FC8F481AF00FFC8F484B
S315080231B01AF00CFC8E481AF009FC8E481AF006FC26
S315080231C000F02DBD7B6803F5806308228A491846FC
S315080231D030F0E0F80346002B08D17B6803F58063DC
S315080231E01846FDF773F90346082B11D07B6803F5D9
S315080231F080631A78814B1B78D31A002B33D17B68EC
S3150802320003F580631846FDF761F90346012B2AD1B7
S315080232107B6803F5C06318462EF0B2FF78627B6AB4
S31508023220002B02DB7B6A0A2B04DD75481AF0CEFBFB
S3150802323000F0F5BC27F0C0FC0346184627F004FD4B
S3150802324003460133DBB219466E4827F027FD7B6A2F
S31508023250DBB219466B4827F03CFD6B49694827F0F3
S3150802326099FD00F0CBBC7B6803F580630C226749A5
S31508023270184630F08FF80346002B08D17B6803F511
S3150802328080631846FDF722F903460C2B11D07B689A
S3150802329003F580631A785E4B1B78D31A002B1BD171
S315080232A07B6803F580631846FDF710F90346012B80
S315080232B012D127F081FC0346184627F0C5FC0346BF
S315080232C00133DBB21946534827F01EFD4E495148D1
S315080232D027F0C3FD00F092BC7B6803F580630C22DD
S315080232E04D49184630F056F80346002B08D17B683C
S315080232F003F580631846FDF7E9F803460C2B13D04D
S315080233007B6803F580631A78444B1B78D31A002B23
S3150802331040F0D1807B6803F580631846FDF7D6F83E
S315080233200346012B40F0C7807B6803F5C0631A7811
S31508023330234B1B78D31A002B16D17B6803F5C0637F
S315080233401846FDF7C3F80346012B0DD134481AF087
S315080233503DFB34481AF03AFB33481AF037FB334838
S315080233601AF034FB00F05BBCFB7A032B40F2A08018
S315080233707B6803F5C06318462EF002FF78627B6805
S3150802338003F5006318462EF0FBFE38627B6803F5E8
S31508023390206318462EF0F4FEF8617B6803F5406355
S315080233A018462EF0EDFEB8617B6A002B02DD7B6AB9
S315080233B00E2B3FDD1E481AF009FB00F030BC00BF99
S315080233C0606D0508646D0508786D0508906D050839
S315080233D0946D05089C6D0508AC6D0508CC6D05084D
S315080233E0E46D05081C6E0508586E05089C6E0508EE
S315080233F0CC6E0508FC6E0508386F0508446F05088B
S31508023400486F0508B4F20020BCF200206C6F05086C
S315080234107C6F0508B8F20020806F0508906F0508D2
S31508023420946F0508A86F0508B86F0508D86F0508D0
S31508023430EC6F0508FB69002B02DDFB69022B03DD35
S315080234409A481AF0C3FAEAE3BB69002B02DDBB69A4
S31508023450082B03DD96481AF0B9FAE0E327F0ACFB2D
S315080234600346184627F0F0FB03460133DBB219463A
S31508023470904813F00DFB7B6ADBB219468D4813F0B0
S3150802348022FB3B6A9BB219468A4813F037FBFB6953
S31508023490DBB21946874813F04CFBBB69DBB2194607
S315080234A0844813F061FB8449824814F0B1F8A5E315
S315080234B0FDF71EFFB3E37B6803F580630A227F49A3
S315080234C018462FF067FF0346002B08D17B6803F5E1
S315080234D080631846FCF7FAFF03460A2B13D07B686B
S315080234E003F580631A78764B1B78D31A002B40F0C3
S315080234F093807B6803F580631846FCF7E7FF03466B
S31508023500012B40F089807B6803F5C0631A786D4BFE
S315080235101B78D31A002B15D17B6803F5C0631846AE
S31508023520FCF7D4FF0346012B0CD167481AF04EFA72
S3150802353066481AF04BFA66481AF048FA65481AF0CD
S3150802354045FA6CE3FB7A032B63D97B6803F5C06300
S3150802355018462EF015FE78627B6803F50063184656
S315080235602EF00EFE38627B6803F5206318462EF0AD
S3150802357007FEF8617B6803F5406318462EF000FEE5
S31508023580B8617B6A002B02DD7B6A0E2B03DD52488B
S315080235901AF01CFA43E3FB69002B02DBFB69032BD7
S315080235A003DD4E481AF012FA39E3BB69002B02DD35
S315080235B0BB69082B03DD3E481AF008FA2FE327F009
S315080235C0FBFA0346184627F03FFB03460133DBB2F4
S315080235D01946434813F0FEFA7B6ADBB2194640489D
S315080235E013F013FB3B6A9BB219463D4813F028FBBE
S315080235F0FB69DBB219463A4813F03DFBBB69DBB2FD
S315080236001946374813F052FB2B49354814F0B1F8DE
S31508023610F4E2FDF76DFE02E37B6803F580630B2295
S31508023620304918462FF0B6FE0346002B08D17B68B0
S3150802363003F580631846FCF749FF03460B2B13D0A4
S315080236407B6803F580631A78274B1B78D31A002BFD
S3150802365040F0D7807B6803F580631846FCF736FF8F
S315080236600346012B40F0CD807B6803F5C0631A78C8
S31508023670144B1B78D31A002B42D17B6803F5C0631F
S315080236801846FCF723FF0346012B39D117481AF0CF
S315080236909DF917481AF09AF916481AF097F9164832
S315080236A01AF094F915481AF091F9B8E20C7005085F
S315080236B02C70050888F20020BCF200204C70050820
S315080236C058700508606D05085C7005086C70050879
S315080236D07C700508B4700508EC6F0508C870050803
S315080236E090F20020E4700508F0700508F4700508E9
S315080236F008710508287105084471050880710508CE
S31508023700FB7A042B7AD97B6803F5C06318462EF038
S3150802371037FD78627B6803F5006318462EF030FDA4
S3150802372038627B6803F5206318462EF029FDF86196
S315080237307B6803F5406318462EF022FDB8617B6864
S3150802374003F5606318462EF01BFD78617B6A002B31
S3150802375002DB7B6A012B03DDA6481AF037F95EE223
S31508023760FB69002B02DBFB69012B03DDA2481AF079
S315080237702DF954E2BB69002B02DDBB69042B03DD7C
S315080237809E481AF023F94AE27B69002B02DD7B691F
S31508023790032B03DD9A481AF019F940E227F00CFACE
S315080237A00346184627F050FA03460133DBB2194698
S315080237B0944813F0CCFA7B6ADBB21946914813F0A7
S315080237C0E1FA3B6A9BB219468E4813F0F6FAFB6990
S315080237D0DBB219468B4813F00BFBBB69DBB2194601
S315080237E0884813F020FB7B69DBB21946854813F03B
S315080237F035FB8549834814F08BF8FFE1FDF778FD20
S315080238000DE27B6803F580630D22804918462FF086
S31508023810C1FD0346002B08D17B6803F58063184671
S31508023820FCF754FE03460D2B11D07B6803F5806323
S315080238301A78774B1B78D31A002B6AD17B6803F563
S3150802384080631846FCF742FE0346012B61D17B686A
S3150802385003F5C0631A786F4B1B78D31A002B12D163
S315080238607B6803F5C0631846FCF730FE0346012B56
S3150802387009D169481AF0AAF868481AF0A7F86848F8
S315080238801AF0A4F8CBE1FB7A012B3FD97B6803F542
S31508023890C06318462EF074FC78627B6803F50063F1
S315080238A018462EF06DFC38627B6A0A2B02DD7B6AAB
S315080238B00D2B03DD51481AF089F8B0E13B6A002B5B
S315080238C002DD3B6A032B03DD4D481AF07FF8A6E1B9
S315080238D027F072F90346184627F0B6F9034601336C
S315080238E0DBB219464F4813F00AFB7B6ADBB219466C
S315080238F04C4813F01FFB3B6ADBB21946494813F0E2
S3150802390034FB4149474814F0E5F877E1FDF7F0FC46
S3150802391085E17B6803F580630922434918462FF03F
S3150802392039FD0346002B08D17B6803F580631846E8
S31508023930FCF7CCFD0346092B13D07B6803F580639D
S315080239401A783A4B1B78D31A002B40F0A2807B6870
S3150802395003F580631846FCF7B9FD0346012B40F0D0
S3150802396098807B6803F5C0631A782A4B1B78D31AAA
S31508023970002B12D17B6803F5C0631846FCF7A6FD37
S315080239800346012B09D12A481AF020F829481AF0C9
S315080239901DF829481AF01AF841E1FB7A022B75D963
S315080239A07B6803F5C06318462EF0EAFB78627B68EB
S315080239B003F5006318462EF0E3FB38627B6803F5CD
S315080239C0206318462EF0DCFBF8617B6A002B02DDC9
S315080239D07B6A072B03DD194819F0F8FF1FE13B6ADA
S315080239E0002B02DB3B6A012B2CDD154819F0EEFF92
S315080239F015E100BF90710508B0710508C870050881
S31508023A00CC71050898F20020BCF20020F071050876
S31508023A1000720508606D0508047205081872050823
S31508023A2080710508A0F20020447205085072050844
S31508023A305472050864720508B4720508CC72050842
S31508023A40E872050827F0B8F80346184627F0FCF886
S31508023A5003460133DBB21946724813F0D8FA7B6A79
S31508023A60DBB219466F4813F0EEFA3B6ADBB2194627
S31508023A706C4813F003FBFB699BB21946694813F0BD
S31508023A8018FB6949674814F0C2F8B7E0FDF730FC3D
S31508023A90C5E07B6803F580630822644918462FF05F
S31508023AA079FC0346002B08D17B6803F58063184628
S31508023AB0FCF70CFD0346082B13D07B6803F58063DD
S31508023AC01A785B4B1B78D31A002B40F093807B68DD
S31508023AD003F580631846FCF7F9FC0346012B40F010
S31508023AE089807B6803F5C0631A78524B1B78D31A10
S31508023AF0002B15D17B6803F5C0631846FCF7E6FC74
S31508023B000346012B0CD14C4819F060FF4B4819F0BB
S31508023B105DFF4B4819F05AFF4A4819F057FF7EE0F5
S31508023B20FB7A032B63D97B6803F5C06318462EF02C
S31508023B3027FB78627B6803F5006318462EF020FBA4
S31508023B4038627B6803F5206318462EF019FBF86184
S31508023B507B6803F5406318462EF012FBB8617B6A50
S31508023B60002B02DD7B6A072B03DD374819F02EFF8F
S31508023B7055E03B6A002B02DB3B6A012B03DD334827
S31508023B8019F024FF4BE0FB69002B02DBFB69642B6F
S31508023B9003DD2F4819F01AFF41E027F00DF8034616
S31508023BA0184627F051F803460133DBB2194629486D
S31508023BB013F09BFA7B6ADBB21946264813F0B1FA70
S31508023BC03B6ADBB21946234813F0C6FAFB69DBB235
S31508023BD01946204813F0DBFABB699BB219461D4801
S31508023BE013F0F0FA10491B4814F0A6F806E0FDF7A0
S31508023BF07FFB14E0184819F0E9FE10E00A482BF09A
S31508023C00A0FB044608482BF0A8FB0346DBB219467C
S31508023C10204606F04BF902E0104819F0D7FE2C3779
S31508023C20BD4690BDA4F20020BCF20020047305082C
S31508023C3010730508606D05081473050824730508D2
S31508023C40B472050840730508CC720508E8720508BF
S31508023C5054730508ACF200207073050884730508CE
S31508023C60F0B589B004AFF8600B467A60FB727D48FE
S31508023C7019F0ACFE7B6803F5007308227A491846E8
S31508023C802FF088FB0346002B40F0B7807B6803F5CC
S31508023C9000731846FCF71AFC0346082B40F0AD8061
S31508023CA0FB7A072B40F2A6807B6803F580631846E9
S31508023CB02EF066FA0346DAB26C4B1A707B6803F585
S31508023CC0C06318462EF05CFA0346DAB2684B1A70DD
S31508023CD07B6803F5006318462EF052FA0346DAB2F9
S31508023CE0644B1A707B6803F5206318462EF048FA6F
S31508023CF003469AB2604B1A807B6803F540631846FE
S31508023D002EF03EFA0346DAB25C4B1A707B6803F56C
S31508023D10606318462EF034FA0346DAB2584B1A7024
S31508023D207B6803F5805318462EF02AFA0346DAB260
S31508023D30544B1A704D4B1B781C464D4B1B781D462F
S31508023D404C4B1B781E464C4B1B881A464B4B1B7812
S31508023D5019464B4B1B7818464A4B1B78039302901D
S31508023D600191009233462A462146474819F02EFE0B
S31508023D703E4B1B781946454829F027FF2CF06AFB6B
S31508023D80034618462CF0F3FC0346013BDBB2194600
S31508023D903E4829F035FF364B1B7819463B4829F031
S31508023DA04AFF354B1B881946384829F05FFF334BC3
S31508023DB01B781946354829F074FF314B1B7819468A
S31508023DC0324829F089FF2F4B1B7819462F4829F0CC
S31508023DD09EFF2F492D482AF01CFE2D482AF0E0FCAA
S31508023DE004462B482AF0E8FC0346194620462DF0DD
S31508023DF037FB67E1FDF77CFA64E17B6803F500733C
S31508023E000522244918462FF0C5FA0346002B45D148
S31508023E107B6803F500731846FCF758FB0346052B27
S31508023E203CD12CF017FB034618462CF062FC0346DD
S31508023E301946194829F0E3FF0021174829F0C4FF5B
S31508023E40134915482AF0D2FE11482AF0A9FC04465D
S31508023E500F482AF0B1FC0346194620462DF000FB0E
S31508023E6030E100BF9C730508B8730508BEF300204D
S31508023E70BFF30020C0F30020C2F30020C4F30020E1
S31508023E80C5F30020C6F30020C4730508C8F3002052
S31508023E90D4F300201074050818F400207B6803F593
S31508023EA000730722894918462FF074FA0346002B35
S31508023EB040F0A4807B6803F500731846FCF706FBFE
S31508023EC00346072B40F09A80FB7A052B40F2938033
S31508023ED07B6803F5806318462EF052F90346DAB278
S31508023EE07B4B1A707B6803F5C06318462EF048F9B7
S31508023EF00346DAB2774B1A707B6803F500631846F5
S31508023F002EF03EF903469AB2734B1A807B6803F584
S31508023F10206318462EF034F90346DAB26F4B1A704C
S31508023F207B6803F5206318462EF02AF90346DAB2AF
S31508023F306B4B1A707B6803F5406318462EF020F91E
S31508023F400346DAB2674B1A70614B1B781946614B06
S31508023F501B781846604B1B881C46604B1B781A4612
S31508023F60604B1B7801930092234602465E4819F07D
S31508023F702DFD574B1B7819465C4829F076FF2CF025
S31508023F8069FA034618462CF0C5FC0346013BDBB228
S31508023F901946564829F084FF4E4B1B781946534852
S31508023FA029F099FF4C4B1B881946504829F0AEFF59
S31508023FB04A4B1B7819464D4829F0C3FF484B1B78D4
S31508023FC019464A4829F0D8FF464B1B7819464748EE
S31508023FD029F0EDFF464945482AF0DFFE44482AF013
S31508023FE0DFFB044642482AF0E7FB03461946204609
S31508023FF02DF0E8FC66E0FDF77BF963E07B6803F5E4
S31508024000007309223B4918462FF0C4F90346002BD0
S3150802401055D17B6803F500731846FCF757FA034631
S31508024020092B4CD1FB7A022B46D97B6803F58063B0
S3150802403018462EF0A5F80346DAB2284B1A707B68A2
S3150802404003F5C06318462EF09BF80346DAB2254BF1
S315080240501A70224B1B781946224B1B781A46264899
S3150802406019F0B4FC2CF0F6F9034618462CF052FC6B
S315080240700346013BDBB21946204829F0E9FF174BF4
S315080240801B7819461D4829F0FEFF164B1B78194660
S315080240901A482AF013F8164918482AF06BFF1448EA
S315080240A02AF07EFB044612482AF086FB0346194686
S315080240B020462DF087FC05E0FDF71AF902E0FDF728
S315080240C017F900BF1437BD46F0BD00BF18740508BE
S315080240D0BEF30020BFF30020C2F30020C4F3002081
S315080240E0C5F30020C6F30020207405081CF400203E
S315080240F0D4F300205C7405086874050828F40020C7
S3150802410080B584B000AFF8600B467A60FB727B68B4
S3150802411003F500730522254918462FF03BF9034695
S31508024120002B3FD17B6803F500731846FCF7CEF9DE
S315080241300346052B36D17B6803F5806302221C49A8
S3150802414018462FF027F90346002B10D17B6803F592
S3150802415080631846FCF7BAF90346022B07D114F016
S31508024160E9FB03460121184614F09FFD1AE07B6815
S3150802417003F5806303220F4918462FF00BF903460D
S31508024180002B0FD17B6803F580631846FCF79EF96E
S315080241900346032B06D114F0CDFB0346002118462D
S315080241A014F083FD00BF1037BD4680BD8C74050828
S315080241B0B8690508A069050890B585B000AF7860AA
S315080241C00023BB730023FB734FF4A052002120483F
S315080241D02FF0D8F807F10E030A221D49786827F04E
S315080241E081F80346012B2ED10023FB7328E0FB7BC3
S315080241F04FF48E7202FB03F3164A13449C1C1448AE
S31508024200FCF764F903461A46114920462FF0C2F80C
S315080242100346002B11D1FB7B0E4A4FF48E7101FB2C
S3150802422003F3134418331B68B97B094A00209847DD
S31508024230094819F0CBFB012306E0FB7B0133FB732C
S31508024240FB7B0E2BD3D9002318461437BD4690BDE7
S31508024250A4DC0020000000208869050880B582B029
S3150802426000AF0346FB71FB790D2B24D14F4B00227D
S315080242701A704F4819F0AAFB4E4B1B78002B16D022
S315080242804D48FFF799FF0346012B08D1F02200217A
S315080242904A482FF077F8484948482FF014F9454B11
S315080242A000221A70F022002143482FF06BF8444886
S315080242B019F08CFB76E0FB790A2B03D13B4B0022E3
S315080242C01A706FE0FB791B2B03D1384B01221A7047
S315080242D068E0FB795B2B07D1344B1B78012B03D1A2
S315080242E0324B02221A705DE0FB79412B1FD12F4B0C
S315080242F01B78022B1BD12D4B00221A702D4B1B78D3
S31508024300002B4FD12D492F4819F060FB2B48FCF79B
S31508024310DDF80346DAB2274B1A70F0220021264846
S315080243202FF030F8254924482FF0CDF83AE0FB79EA
S31508024330082B02D0FB797F2B16D11C4B00221A7050
S315080243401C4B1B78002B2DD01A4B1B78013BDAB27B
S31508024350184B1A70174B1B781A46174B002199549B
S31508024360194819F033FB1DE0124B1B785A1CD1B2BF
S31508024370104A11701946104AFB7953540D4B1A7894
S31508024380124BA3FB0213D9090B461B015B1A1B012D
S31508024390D31ADAB2074B1A70FB7919460C4819F088
S315080243A015FBFFE700BF0837BD4680BD2BF400208A
S315080243B08869050884F2002094F10020A4F0002000
S315080243C09474050880690508987405088988888898
S315080243D09C74050880B500AF342300223C493D4849
S315080243E026F064F90346002B01D01C236EE0342321
S315080243F000223949394826F059F90346002B01D0DB
S315080244001C2363E0342300223549364826F04EF948
S315080244100346002B01D01C2358E0342300223249DC
S31508024420324826F043F90346002B01D01C234DE0FF
S31508024430342300222E492F4826F038F90346002B4A
S3150802444001D01C2342E0342300222B492B4826F0B4
S315080244502DF90346002B01D01C2337E03423002212
S315080244602749284826F022F90346002B01D01C23A7
S315080244702CE0342300222449244826F017F903465F
S31508024480002B01D01C2321E0342300222049214895
S3150802449026F00CF90346002B01D01C2316E0342320
S315080244A000221D491D4826F001F90346002B01D0BA
S315080244B01C230BE03423002219491A4826F0F6F881
S315080244C00346002B01D01C2300E00023184680BDBA
S315080244D0A874050810F50020BC74050844F50020E8
S315080244E0D074050878F50020F0740508ACF50020AC
S315080244F014750508E0F500203475050814F6002041
S315080245004875050848F60020607505087CF60020FF
S3150802451074750508B0F6002090750508E4F60020C3
S31508024520A875050818F7002080B58EB008AF786020
S3150802453000237B617B683B6107F10C0100234FF482
S315080245408062386925F09EFF0346002B01D00223BC
S3150802455054E0FB68B02206920122059200220492D8
S315080245600A2203920A2202924FF48062019200936F
S315080245700023244A2449254826F0CAF90346002B73
S3150802458001D00E233AE0342300222149214826F09D
S315080245908DF80346002B01D01C232FE0FFF71AFFE4
S315080245A00346002B01D01C2328E0786818F0DAFFAE
S315080245B00346002B01D01C2320E0786818F074FF0C
S315080245C00346002B01D01C2318E0786816F0F8F889
S315080245D00346002B01D01C2310E0786816F0F4FA83
S315080245E00346002B01D01C2308E0786814F036FC39
S315080245F00346002B01D01C2300E07B6918461837B6
S31508024600BD4680BD19460208D07505082CF400205F
S31508024610E4750508DCF4002080B584B000AF786044
S3150802462001221021154819F0C9FC0346FB731448E8
S3150802463019F0CCF9134819F0C9F9134819F0C6F953
S31508024640104819F0C3F9114B1B780133DAB20F4B34
S315080246501A700E4B1B78092B08D90C4B00221A70BC
S3150802466020210B481BF086F919F080FDFB7B1846C2
S3150802467019F04EFD642025F06FF9E4E7D0750508B8
S31508024680F4750508F8750508187605084CF700202C
S315080246900010024280B500AF24F0FEF900BF80BDCB
S315080246A080B400AF034B1B681846BD465DF8047B11
S315080246B0704700BF50F7002080B500AF4FF4006284
S315080246C00E490F4826F078FE4FF400620D490E484F
S315080246D026F072FE4FF400720C490D4826F06CFE65
S315080246E04FF400620B490C4826F066FE4FF400624E
S315080246F00A490B4826F060FE00BF80BD64F7002019
S3150802470054F7002074FF002064FF0020A807012048
S3150802471098070120E8090120A8090120281201208A
S31508024720E811012080B483B000AF78607B68002B63
S3150802473001D1002346E07B68012B01D1012341E028
S315080247407B68022B01D102233CE07B68032B01D153
S31508024750032337E07B68042B01D1042332E07B680C
S31508024760052B01D105232DE07B68062B01D10623F3
S3150802477028E07B68072B01D1072323E07B68082BF7
S3150802478001D108231EE07B68092B01D80C2319E006
S315080247907B680A2B01D8102314E07B680B2B01D8FF
S315080247A014230FE07B680C2B01D818230AE07B68D8
S315080247B00D2B01D8202305E07B680E2B01D8302368
S315080247C000E0402318460C37BD465DF8047B704767
S315080247D080B483B000AF0346FB80FB88002B01D16F
S315080247E0002346E0FB88012B01D1012341E0FB8827
S315080247F0022B01D102233CE0FB88032B01D10323C0
S3150802480037E0FB88042B01D1042332E0FB88052B11
S3150802481001D105232DE0FB88062B01D1062328E0CA
S31508024820FB88072B01D1072323E0FB88082B01D13C
S3150802483008231EE0FB880C2B01D8092319E0FB8804
S31508024840102B01D80A2314E0FB88142B01D80B235A
S315080248500FE0FB88182B01D80C230AE0FB88202BD3
S3150802486001D80D2305E0FB88302B01D80E2300E082
S315080248700F2318460C37BD465DF8047B70470000C7
S3150802488084B0B0B400AF07F10C0484E80F00074BFC
S315080248901D4607F10C040FCC0FC50FCC0FC52368B4
S315080248A02B6000BFBD46B0BC04B070477407012038
S315080248B080B586B000AF78600B467B800023FB7517
S315080248C000233B610023FB600023BB6000F054FD1C
S315080248D00346002B0BD0444BD3F844323B61424B80
S315080248E0D3F8843AFB607B681B68BB600AE03E4BE0
S315080248F0D3F844323B613C4BD3F8843AFB607B687D
S315080249001B68BB603A69BB689A4227D1364B93F853
S315080249106832002B0AD1344BD3F850227B881344D1
S31508024920314AC2F850320123FB7558E02E4BB3F8D0
S315080249306C321A467B881344B3F5006F0BDA2A4B9E
S31508024940B3F86C227B8813449AB2274BA3F86C22DD
S315080249500123FB7543E00023FB7540E0FA68BB6858
S315080249609A4227D1204B93F8A83A002B0AD11E4B1C
S31508024970D3F850227B8813441B4AC2F850320223CA
S31508024980FB752CE0184BB3F8AC3A1A467B881344ED
S31508024990B3F5006F0BDA144BB3F8AC2A7B881344D1
S315080249A09AB2114BA3F8AC2A0223FB7517E000232F
S315080249B0FB7514E03B69002B07D1242279680B4862
S315080249C02EF097FD0123FB7509E0FB68002B06D143
S315080249D02422796806482EF08CFD0223FB75FB7D9E
S315080249E018461837BD4680BD74070120B80901204C
S315080249F0F811012080B584B000AF03463960FB7117
S31508024A001346BB800023FB81FB79012B12D10023BD
S31508024A10FB810AE0FB893A681344012219461248C7
S31508024A2026F070FDFB890133FB81FA89BB889A421D
S31508024A30F0D314E0FB79022B11D10023FB810AE0A3
S31508024A40FB893A68134401221946084826F05AFD9A
S31508024A50FB890133FB81FA89BB889A42F0D300BFEE
S31508024A601037BD4680BD00BFA8090120E811012004
S31508024A7080B582B000AF0346FB71FB1D01221946C1
S31508024A80034826F03FFD00BF0837BD4680BD00BF7C
S31508024A9098070120F0B5C3B008AFF861B9617A6129
S31508024AA0002387F8E730F8691AF041F8C7F8E000FA
S31508024AB0B34B00221A6084E0B14B1B685A1CB049FA
S31508024AC00A60B3F5FA7F7CD997F8E730013387F89D
S31508024AD0E73007F168031946F8691AF05BF9BB6E05
S31508024AE03B61FA6EFA60386FB8607B6FBA6FF96F1E
S31508024AF0D7F88000D7F884407C60D7F88850D7F872
S31508024B008C60D7F890400794069605957C680494BD
S31508024B100390029101920093BB68FA683969994831
S31508024B2018F054FFFB6F002B07D0FB691B689A69C4
S31508024B30FB691B6822F001029A61F86919F0F7FF0E
S31508024B40C7F8E000D7F8E010F86919F0FCFF8C4BBB
S31508024B5000221A6013F0EEFE03460121184614F0ED
S31508024B605DF80346002B02D0874818F02FFF874BC3
S31508024B701B78022B2ED0854B01221A7007F1D80317
S31508024B800221184627F0F9FD07F1940207F1D80326
S31508024B901146184628F0C1F827F0FAFA044607F132
S31508024BA09403184627F04FFE054607F19403184664
S31508024BB027F055FE03461A46294620462DF06EF87A
S31508024BC008E00721F8691AF035F90346002B7FF445
S31508024BD073AF00E000BF7A69B969F86919F063FF33
S31508024BE00346002B3AD097F8E730013387F8E730C7
S31508024BF013F0A0FE03460121184614F00FF80346E7
S31508024C00002B02D0624818F0E1FE604B1B78012B9C
S31508024C1024D05E4B01221A7007F1D80301211846E7
S31508024C2027F0ABFD07F1940207F1D803114618469F
S31508024C3028F073F827F0ACFA044607F194031846ED
S31508024C4027F001FE054607F19403184627F007FEEA
S31508024C5003461A46294620462DF020F897F8E730EB
S31508024C60002B28D1494B1B78002B24D0474B002216
S31508024C701A7007F1D8030021184627F07EFD07F1BE
S31508024C80940207F1D8031146184628F046F827F089
S31508024C907FFA044607F19403184627F0D4FD054621
S31508024CA007F19403184627F0DAFD03461A46294601
S31508024CB020462CF0F3FFF86900F002FB03461A4679
S31508024CC0344B9A60F86900F0C5FA0346314A136014
S31508024CD0F86900F0D7FA03462E4A53602D4B9B68B3
S31508024CE0002B04D02B4B9B68184600F031FB0C2294
S31508024CF0284929482EF036FB0346002B36D0254B89
S31508024D001B68DAB207F164031146184627F0E4FC79
S31508024D10204B5B68DAB207F164031146184627F09E
S31508024D20F6FC1C4B9B68DAB207F164031146184677
S31508024D3027F008FD07F1200207F164031146184619
S31508024D4027F0BCFF27F024FA044607F12003184689
S31508024D5027F079FD054607F12003184627F07FFD5F
S31508024D6003461A46294620462CF098FF0A4B094A5A
S31508024D7007CA83E8070000BFEC37BD46F0BD00BF8F
S31508024D80401A0120387605087C760508441A01205F
S31508024D90A0760508281A0120341A012080B592B097
S31508024DA000AF3B464022002118462EF0EBFA0023BC
S31508024DB0A7F8423000237B64B34826F087FB0346F4
S31508024DC083F00103DBB2002B00F0DB80AF4B93F8D4
S31508024DD06832002B5BD1AD4BD3F850329AB2AB4B4B
S31508024DE0A3F86C22A94B0F22C3F8502210233B705A
S31508024DF03B785AB2A54BB3F86C321B0A9BB25BB22C
S31508024E0003F00F035BB213435BB2DBB23B709F4BFB
S31508024E10B3F86C32DBB27B703B4602333E2219464C
S31508024E20994826F0AAFB0346002B00F029814FF485
S31508024E307A71974825F0D8FC0346002B09D1FFF76B
S31508024E402FFC3B461A469349FFF724FE904825F065
S31508024E5025FD8E4BB3F86C323E3B9AB28B4BA3F8C8
S31508024E606C228A4BB3F86A3201339AB2874BA3F89B
S31508024E706A22864B012283F86822844BFF2283F832
S31508024E806E22824B4FF4FA62C3F87022F8E07F4B27
S31508024E9093F86E32002B05D07C4B93F86E32012BB9
S31508024EA040F0EE80794BB3F86C323E2B02D94023A0
S31508024EB07B6404E0754BB3F86C3201337B642023C0
S31508024EC03B703B785AB2714BB3F86A325BB203F065
S31508024ED00F035BB213435BB2DBB23B707B6C5A1EA9
S31508024EE03B4601331946684826F047FB0346002B22
S31508024EF000F0C6804FF47A71654825F075FC0346C2
S31508024F00002B12D17B6C9BB21846FFF761FC034655
S31508024F105E4AC2F85032FFF7C3FB3B461A465D4962
S31508024F20FFF7B8FD5A4825F0B9FC584BB3F86C227E
S31508024F307B6C9BB2D31A9BB201339AB2534BA3F83A
S31508024F406C22524BB3F86A3201339AB24F4BA3F82A
S31508024F506A224E4BB3F86C32002B40F09180242221
S31508024F6000214C482EF00EFA484B002283F868229C
S31508024F70464B0022A3F86A22444BFF2283F86E228C
S31508024F807EE0454826F0A2FA034683F00103DBB227
S31508024F90002B75D03B46012219463F4826F0EDFA0A
S31508024FA00346002B69D03B781B09DBB2032B1FD1C2
S31508024FB03B46013302221946374826F0DEFA0346F3
S31508024FC0002B5DD0314B0322DA604FF47A713048F8
S31508024FD025F00AFC0346002B52D1FFF761FB3B463C
S31508024FE01A462A49FFF756FD294825F057FC47E095
S31508024FF03B781B09DBB2002B42D13B460133012227
S315080250001946254826F0B9FA0346002B37D03B78CD
S315080250101B029BB203F47063A7F842307B781A46E8
S31508025020B7F842301343A7F84230B7F842203B4656
S3150802503002331946184826F0A0FA0346002B1FD059
S31508025040B7F8423002339BB21846FFF7C1FB034654
S315080250500E4AD3604FF47A710D4825F0C5FB034614
S31508025060002B0DD1FFF71CFB3B461A460749FFF7F3
S3150802507011FD074825F012FC02E000BF00E000BF60
S315080250804837BD4680BD00BFA80901207407012024
S315080250907CF60020B80901209807012080B59AB04D
S315080250A000AF3B466822002118462EF06BF90E48DF
S315080250B026F00CFA034683F00103DBB2002B0ED06E
S315080250C004E03B466821184600F010F83B46682281
S315080250D01946054826F051FA0346002BF1D100BFBE
S315080250E06837BD4680BD00BF64FF002080B582B028
S315080250F000AF78600B467B80786800F099FB00BFAA
S315080251000837BD4680BD000080B500AF174B93F83F
S315080251106832002B28D0154B93F86E32FF2B23D119
S31508025120124BD3F87032002B07D0104BD3F87032DB
S31508025130013B0E4AC2F8703216E0242200210C48BE
S315080251402EF020F94FF400620A490B4826F034F98A
S31508025150064B002283F86822044B0022A3F86A222F
S31508025160024BFF2283F86E2200BF80BD740701201E
S31508025170B8090120E8090120A809012080B582B0F2
S3150802518000AF78600B467B80786800F079FA00BF3A
S315080251900837BD4680BD000080B582B000AF786092
S315080251A00B467B807B881A467968034826F0AAF95B
S315080251B000BF0837BD4680BD54F7002080B59AB0B7
S315080251C000AF3B466822002118462EF0DBF80E484F
S315080251D026F07CF9034683F00103DBB2002B0ED0DE
S315080251E004E03B4668211846FFF7C8FF3B4668229B
S315080251F01946054826F0C1F90346002BF1D100BF2E
S315080252006837BD4680BD00BF54F7002080B582B01E
S3150802521000AF78600B4A7B681360FFF74DFA2422C9
S31508025220002109482EF0AEF82422002107482EF064
S31508025230A9F82422002106482EF0A4F800BF083750
S31508025240BD4680BD50F7002074070120B809012029
S31508025250F811012080B485B000AF78607B681B68BE
S315080252601B6CBB600023FB60BB68DBB2002B02D061
S31508025270BB68DBB2FB60FB6818461437BD465DF8AF
S31508025280047B704780B485B000AF78607B681B6882
S315080252901B6CBB600023FB60BB6803F4FE43002B58
S315080252A006D0BB6803F4FE43FB60FB681B0AFB607F
S315080252B0FB6818461437BD465DF8047B7047000044
S315080252C080B485B000AF78607B681B685B6CBB6096
S315080252D00023FB60BB6803F00703002B2FD0BB68D3
S315080252E003F00703013B052B20D801A252F823F04D
S315080252F0095302080F530208155302081B530208E2
S3150802530021530208275302080123FB600FE00223F8
S31508025310FB600CE00323FB6009E00423FB6006E064
S315080253200523FB6003E00623FB6000E000BF7B6801
S315080253301B685A6C7B681B6822F007025A64FB6872
S31508025340DBB218461437BD465DF8047B704700BFCA
S3150802535080B582B000AF786013F0ECFA03460121FB
S31508025360184613F05BFC034683F00103DBB2002BFD
S315080253700837BD4680BD000080B400AF034B1B78DA
S315080253801846BD465DF8047B704700BFA41000208E
S3150802539080B500AFFFF7F0FF0346002B02D04FF4AB
S315080253A0807301E04FF48073184680BD80B500AF64
S315080253B0FFF7E2FF0346002B02D04FF4001300E08A
S315080253C00023184680BD80B500AFFFF7D5FF034618
S315080253D0002B02D040F20D1300E00023184680BDD0
S315080253E0B0B5A4B006AFF860B9601346FB800023D7
S315080253F0A7F87630FB683B65FFF7BEFF0346002B2E
S3150802540003D04FF080437B6501E000237B650023D0
S31508025410BB65FB8802339BB21846FFF7D9F90346E8
S31508025420FB6500233B664FF480137B664FF400133B
S31508025430BB660023FB6600233B6700233B743B7C69
S315080254405AB2FB881B0A9BB25BB203F00F035BB22C
S3150802545013435BB2DBB23B74FB88DBB27B74022379
S31508025460A7F8763010E0B7F87630023BBA681A44E5
S31508025470B7F87630127878333B4403F8682CB7F8D5
S3150802548076300133A7F87630B7F87620FB880133F1
S315080254909A42E8DD0023A7F876300DE0B7F87630B1
S315080254A078333B4413F8683C1846FFF7E1FAB7F835
S315080254B076300133A7F87630B7F87620FB880133C1
S315080254C09A42EBDD6D4607F160040FCC0FC52368DF
S315080254D02B6007F150030FCBFFF7D2F900BF7837DD
S315080254E0BD46B0BD80B58EB000AFF860B960134650
S315080254F0FB80002387F83730FB683B61FFF73CFFE8
S315080255000346002B03D04FF080437B6101E0002362
S315080255107B610023BB61FB88FB6100233B624FF47E
S3150802552080137B624FF40013BB620023FB620023E5
S315080255303B63FA8807F1100311461846FFF7B8F9D4
S31508025540034687F8373097F83730002B06D0FA88A3
S3150802555097F83730B9681846FFF74CFA00BF38375C
S31508025560BD4680BDB0B5A2B006AF78600846114602
S315080255701A460346FB700B46BB7013467B70002324
S3150802558087F86F307B68BB64FFF7F6FE0346002B8D
S3150802559003D04FF08043FB6401E00023FB64002341
S315080255A03B6503237B650023BB654FF48013FB65CC
S315080255B04FF400133B6600237B660023BB66302349
S315080255C03B723B7A5AB297F9033003F00F035BB288
S315080255D013435BB2DBB23B72BB787B727B78BB72DE
S315080255E0002387F86F300DE097F86F3070333B442D
S315080255F013F8683C1846FFF73BFA97F86F30013301
S3150802560087F86F3097F86F30022BEDD96D4607F1A0
S3150802561058040FCC0FC523682B6007F148030FCB3C
S31508025620FFF72EF900BF7037BD46B0BD80B582B010
S3150802563000AF78600023002200217868FFF792FF06
S3150802564000BF0837BD4680BD80B584B000AFF8609C
S31508025650B9601346FB80FB883E2B06D8FB881A46A0
S31508025660B968F868FFF7BCFE05E0FB881A46B96810
S31508025670F868FFF737FF00BF1037BD4680BD000048
S3150802568080B588B000AF7860FF23FB7600237B6184
S315080256900023FB6100237B827B68FB60FB6893F82F
S315080256A028301B09FB76FB681B687B617B69B3F5AF
S315080256B0001F02D140F20D13FB61FB7E032B00F2A1
S315080256C0A78001A252F823F0D95602081B570208EE
S315080256D065570208B3570208FB6893F8283003F0A7
S315080256E00F039AB24C4B1A804B4B1B881B029AB279
S315080256F0494B1A80FB6893F829301A46464B1B8891
S3150802570013439AB2444B1A80FB682A33424A1288D8
S315080257101146184604F0A6FB7AE0FB6893F828308F
S3150802572003F00F039AB23C4B1A803B4B1B881B02B1
S315080257309AB2394B1A80FB6893F829301A46364BC7
S315080257401B8813439AB2344B1A80344B01221A70BF
S31508025750FB682A333E21184604F084FBF869FFF7F2
S3150802576065FF55E02D4B1B781A46FB6893F82830DF
S3150802577003F00F039A4248D1FB68DB681846FEF726
S31508025780D1FF0346013B7B82FB6829337A8A11469D
S31508025790184604F067FB214B1B780133DAB21F4B1C
S315080257A01A701E4B1B780F2B2FD91C4B00221A700E
S315080257B02BE01B4BD3F84432FA699A420FD1FB68A5
S315080257C093F8283003F00F03DAB2154B83F86E22EA
S315080257D0FB6893F82920124B83F86F2217E0104BC7
S315080257E0D3F8843AFA699A4211D1FB6893F82830B9
S315080257F003F00F03DAB20A4B83F8AE2AFB6893F872
S315080258002920074B83F8AF2A01E000BF00E000BF5A
S3150802581000BF2037BD4680BD461A0120481A01201E
S315080258207407012080B500AF2CF086F900BF80BD51
S3150802583080B584B000AF78607B68FB60FFF79CFD9B
S315080258400346002B0AD0FB681B68B3F5806F10D19C
S31508025850FB6893F82830002B0BD10AE0FB681B681B
S31508025860B3F5806F05D1FB6893F82830002B00D179
S3150802587000BF00BF1037BD4680BD000080B500AF2F
S3150802588040220349034825F097FD0123184680BDA7
S315080258905C1A01204C1A012080B500AF054825F094
S315080258A015FE0346002B01D0012300E0002318460B
S315080258B080BD00BF4C1A012080B582B000AF786067
S315080258C00B46FB704FF47A710A4824F08DFF0346A3
S315080258D0002B0AD1FB781A467968074825F081FF1A
S315080258E0044824F0DBFF012300E0002318460837AA
S315080258F0BD4680BD48F600204C1A012080B584B00A
S3150802590000AF78600023FB734FF47A710A4824F0DB
S315080259106BFF0346002B0AD17968084825F072FF07
S315080259200346FB73044824F0B9FFFB7B00E000231F
S3150802593018461037BD4680BD48F600204C1A01208D
S31508025940F0B599B004AF0346FB71002387F84F30D0
S31508025950FFF7A2FF0346002B40F09784C44818F0CD
S3150802596035F807F10C034022002118462DF00AFDEE
S3150802597007F10C031846FFF7C1FF034687F84F30B5
S315080259803B7B012B40F07C8497F84F30002B00F0CC
S3150802599077847B7BFF2B00F36384F12B07DA052BD5
S315080259A000F05A84062B00F0A88300F059BCF13B9C
S315080259B00E2B00F2558401A252F823F0F959020877
S315080259C07F5B0208735D020873620208515F020870
S315080259D06162020861620208616202086162020883
S315080259E06162020861620208616202086162020873
S315080259F0616202084562020807F10C0302339D49F7
S31508025A00184629F056F815F0C9F80346184615F04F
S31508025A108DF90346002B40F0A980964828F0C9F86C
S31508025A2003461A46944B1A80924828F0DDF8034634
S31508025A301A46924B1A708F4828F0F1F803461A460E
S31508025A408F4B1A708F4B01221A708A4828F002F976
S31508025A5003461A468C4B1A80864828F016F90346DE
S31508025A601A468A4B1A70834828F02AF903461A46B8
S31508025A70874B1A707F4828F03EF903461A46854B2B
S31508025A801A707D4B1B881C467C4B1B781D467C4B2B
S31508025A901B781E467C4B1B881A467C4B1B7819467C
S31508025AA07B4B1B7818467B4B1B780393029001911C
S31508025AB0009233462A462146774812F0DFFE15F051
S31508025AC06DF802466C4B1B881946104615F055F9B7
S31508025AD015F064F80246694B1B781946104615F00C
S31508025AE05BF915F05BF80246654B1B7819461046BA
S31508025AF015F06DF915F052F80246624B1B781946F5
S31508025B00104615F07FF915F049F802465E4B1B88D8
S31508025B101946104615F091F915F040F802465B4B06
S31508025B201B781946104615F0A3F915F037F8024600
S31508025B30574B1B781946104615F0B5F915F02EF88D
S31508025B400246544B1B781946104615F0C7F915F04C
S31508025B5025F803460121184615F0DBF915F01EF85B
S31508025B6003460121184615F0EDF887E3414828F067
S31508025B7020F803461946494812F080FE7EE307F1EB
S31508025B800C0302334649184629F05FF8444828F0C0
S31508025B900FF903461946434812F070FE404828F0AA
S31508025BA007F90346002B24D12AF054FC034618466B
S31508025BB02AF08CFC03460021184628F0AAFB2AF094
S31508025BC049FC034618462AF081FC0346002118467A
S31508025BD028F0BAFB2AF03EFC034618462AF076FC61
S31508025BE003460021184628F07DFC2F4812F046FE8F
S31508025BF041E32B4828F0DCF80346012B0ED12AF0A4
S31508025C0029FC034618462AF061FC03460021184679
S31508025C1028F07FFB254812F031FE2CE3204828F0B5
S31508025C20C7F80346022B0ED12AF014FC034618467F
S31508025C302AF04CFC03460021184628F085FB1C482E
S31508025C4012F01CFE17E3164828F0B2F80346052B95
S31508025C5032D12AF0FFFB034618462AF037FC0346E0
S31508025C600021184628F03EFC124812F007FE02E30D
S31508025C70C47605089C1A0120C41A0120C61A0120F6
S31508025C80C71A0120C81A0120CA1A0120CC1A0120F3
S31508025C90CD1A0120CE1A0120F076050838770508B4
S31508025CA0B01A01206477050888770508AC770508D5
S31508025CB0D477050800780508964828F079F8034647
S31508025CC0062B0DD12AF0C6FB034618462AF0FEFB20
S31508025CD00346184628F01FFD8F4812F0CFFDCAE288
S31508025CE08C4828F065F80346FE2B1DD1894828F012
S31508025CF044F803461C4614F051FF0346184615F0AD
S31508025D0030F803469C4240F0B6822AF0A3FB0346CB
S31508025D1018462AF0DBFB03460421184628F014FB32
S31508025D207E4812F0ABFDA6E27A4828F041F803460F
S31508025D30FF2B40F0A082774828F01FF803461C463E
S31508025D4013F076F80346184613F06DF903469C429B
S31508025D5040F091822AF07EFB034618462AF0B6FBEB
S31508025D6003460921184628F0BDFB6D4812F086FD48
S31508025D7081E207F10C0302336A49184629F05DF8F5
S31508025D8013F056F80346184613F032F90346002B69
S31508025D9040F0A080634828F05CF803461A46624B36
S31508025DA01A80604828F070F803461A465F4B1A7044
S31508025DB05C4828F084F803461A465D4B1A7059481F
S31508025DC028F098F803461A465A4B1A80554828F07E
S31508025DD0ACF803461A46584B1A70524828F0C0F8CF
S31508025DE003461A46554B1A704E4828F0D4F803460D
S31508025DF01A46534B1A704C4B1B881C464B4B1B7846
S31508025E001D464B4B1B781E464A4B1B881A464A4B65
S31508025E101B781946494B1B781846494B1B7803933E
S31508025E2002900191009233462A462146454812F0CD
S31508025E3025FD12F0FDFF02463B4B1B88194610460C
S31508025E4013F0FDF812F0F4FF0246384B1B78194698
S31508025E50104613F003F912F0EBFF0246344B1B7897
S31508025E601946104613F015F912F0E2FF0246314BB5
S31508025E701B88194689000B441946880019460346A9
S31508025E800B449B009BB21946104613F01DF912F0FB
S31508025E90CFFF0246284B1B781946104613F023F902
S31508025EA012F0C6FF0246254B1B781946104613F018
S31508025EB035F912F0BDFF0246214B1B7819461046EA
S31508025EC013F047F912F0B4FF03460121184613F0FE
S31508025ED09BF8D3E105F09EFD0346184605F0B2FD90
S31508025EE00346184606F07AF90346002B08D00D48F1
S31508025EF027F0AFFF03461946134812F0BFFCBDE16F
S31508025F00084827F0A6FF03461946104812F0B6FCC1
S31508025F10B4E100BFB01A0120307805086478050894
S31508025F2090780508B41A0120D61A0120D81A012039
S31508025F30D91A0120DA1A0120DC1A0120DD1A0120F9
S31508025F40DE1A0120C07805080C7905083C7905088F
S31508025F5007F10C030233CF49184629F03BF812F031
S31508025F6067FF0346184613F043F80346002B40F032
S31508025F70868005F04FFD0346184605F063FD034685
S31508025F80184606F02BF90346002B78D105F042FD98
S31508025F900346184605F056FD0346184606F00DF860
S31508025FA00346002B6BD105F035FD0346184605F06E
S31508025FB049FD0346184606F01BF80346002B5ED138
S31508025FC0B44828F039F803461A46B34B1A70B14852
S31508025FD028F04DF803461A46B04B1A70AD4828F019
S31508025FE061F803461A46AE4B1A70AB4B1B78194634
S31508025FF0AA4B1B781A46AA4B1B78AA4812F03EFCF3
S3150802600012F016FF03460021184613F018F812F08C
S315080260100FFF0246A04B1B781946104613F01EF8CE
S3150802602012F006FF0346FF21184613F032F812F063
S31508026030FFFE03460021184613F046F812F0F8FE52
S3150802604003460021184613F04EF812F0F1FE0246F6
S31508026050924B1B781946104613F060F812F0E8FEC8
S3150802606002468F4B1B781946104613F072F812F047
S31508026070DFFE03460121184612F0C6FFFDE012F0C4
S31508026080D7FE0346184612F0B3FF0346002B02D08A
S31508026090854812F0F3FB05F0BDFC0346184605F0E9
S315080260A0D1FC0346184606F099F80346002B02D09F
S315080260B07E4812F0E3FB05F0ADFC0346184605F0F0
S315080260C0C1FC0346184605F078FF0346002B02D0AA
S315080260D0774812F0D3FB05F09DFC0346184605F0F7
S315080260E0B1FC0346184605F083FF0346002B00F071
S315080260F0C4806F4812F0C2FBBFE007F10C030233FB
S315080261006C49184628F0E0FF14F048FD0346184685
S3150802611014F00CFE0346002B40F08B80654828F0ED
S315080261202FF803461A46644B1A70624828F043F859
S3150802613003461A46614B1A705E4828F057F803461A
S315080261401A465F4B1A705B4828F06BF803461A46E4
S315080261505C4B1A70574828F07FF803461A465A4B82
S315080261601A80554B1B781946544B1B781846544BC4
S315080261701B781C46534B1B781A46534B1B880193B4
S31508026180009223460246514812F078FB14F006FDA7
S3150802619003460021184614F0F0FD14F0FFFC0246EF
S315080261A0454B1B781946104614F0F6FD14F0F6FC1A
S315080261B00246424B1B781946104614F008FE14F0A4
S315080261C0EDFC02463E4B1B781946104614F01AFEA1
S315080261D014F0E4FC02463C4B1B881946104614F0A0
S315080261E02CFE14F0DBFC0246364B1B78013BDBB275
S315080261F01946104614F03CFE14F0D0FC0346002162
S31508026200184614F050FE14F0C9FC0346012118463C
S3150802621014F064FE14F0C2FC03460021184614F07A
S3150802622078FE14F0BBFC03460121184614F08AFDD9
S3150802623024E0274827F0BDFC03461946254812F0F4
S315080262401DFB1BE0244812F019FB12F073FB0346F0
S31508026250184612F0CCFB11E0204812F00FFB0DE0B5
S315080262607B7B194697F84F301A461D4817F0AEFB46
S3150802627004E000BF02E000BF00E000BF00BF04E088
S315080262803B7B1946174817F0A1FB00BF5437BD469A
S31508026290F0BD00BFC01A0120DF1A0120E01A012052
S315080262A0E11A01206C7905089C790508C879050860
S315080262B0F4790508A81A0120CF1A0120D01A01205C
S315080262C0D11A0120D21A0120D41A0120207A0508EF
S315080262D09C1A012038770508607A0508807A05082D
S315080262E0987A0508C87A050880B500AF4FF4007297
S315080262F00349044825F060F80123184680BD00BF0B
S31508026300E41A0120E41C012080B582B000AF002304
S31508026310FB71074825F0DAF80346FB71FB79002B77
S3150802632001D0012300E0002318460837BD4680BD88
S31508026330E41C012080B584B000AF78600B46FB7080
S315080263400023FB604FF47A710F4824F04DFA034696
S31508026350002B0AD1FB781A4679680C4825F041FACF
S31508026360F860094824F09AFA02E0094817F02EFB69
S31508026370FB68002B02D1074817F028FB01231846B1
S315080263801037BD4680BD00BF18F70020E41C012067
S31508026390FC7A0508387B050880B584B000AF7860BA
S315080263A00023FB734FF47A710B4824F01DFA034657
S315080263B0002B09D17968094825F024FA0346FB73AC
S315080263C0054824F06BFA02E0054817F0FFFAFB7B52
S315080263D018461037BD4680BD18F70020E41C012078
S315080263E0647B050880B584B000AF78600B46FB7005
S315080263F00023FB600023FB6009E0FB78184617F0D0
S3150802640087FE012023F0A8FAFB680133FB60FA68CD
S315080264107B689A42F1D300BF00BF1037BD4680BDE4
S31508026420F0B587B004AF0346FB71FFF76DFF03466D
S31508026430002B40F00885A24B00221A708022002108
S31508026440A0482CF09FFF9F48FFF7A6FF03461A466F
S315080264509B4B1A709B4B1B78292B49DC212B2DDA77
S3150802646000F0E9BC603B112B00F2E58401A252F868
S3150802647023F000BF3D650208116702088F6802080B
S315080264808F6A0208376E0208376E0208376E0208EC
S31508026490376E0208376E0208376E0208376E020830
S315080264A0376E0208376E0208376E0208376E020820
S315080264B0376E0208516C0208F36C0208213B082B5E
S315080264C000F2B98401A252F823F000BFFF64020861
S315080264D01765020829650208376E0208376E020830
S315080264E0376E0208376E0208376E020833650208ED
S315080264F0712B00F3A084602BB4DA00F09CBC7248BE
S3150802650012F0BCF97149724824F06AFC6F4824F00B
S31508026510D4FB00F098BC6F4812F0B0F96E496C488B
S3150802652024F0B9FC00F08FBC6C4812F0A7F900F011
S315080265308ABC6B4812F0A2F900F085BC6949644826
S3150802654011F0A4F814F02AFB0346184614F0EEFBE1
S315080265500346002B40F0AC80634B00221A80614848
S3150802656010F08AFA03461A46604B1A705D4810F014
S315080265709EFA03461A465E4B1A705A4810F0CDFA2E
S3150802658003461A465B4B1A70564810F0ABFA034696
S315080265901A46594B1A80594B00221A70584B002238
S315080265A01A70504810F0D4FA03461A46554B1A7018
S315080265B04D4B1B881C464D4B1B781D464C4B1B7876
S315080265C01E464D4B1B881A464C4B1B781946494B9F
S315080265D01B7818464B4B1B78039302900191009245
S315080265E033462A462146484812F048F914F0D6FAA4
S315080265F002463D4B1B881946104614F0BEFB14F0A2
S31508026600CDFA0246394B1B781946104614F0C4FBDC
S3150802661014F0C4FA0246364B1B781946104614F093
S31508026620D6FB14F0BBFA0246324B1B7819461046C3
S3150802663014F0E8FB14F0B2FA02462F4B1B881946EF
S31508026640104614F0FAFB14F0A9FA02462B4B1B78F3
S315080266501946104614F00CFC14F0A0FA0246284B10
S315080266601B781946104614F01EFC14F097FA0246D7
S31508026670244B1B781946104614F030FC14F08EFA97
S3150802668003460021184614F044FC29F0E3FE0346AB
S31508026690184629F01BFF03460021184627F054FE28
S315080266A014F07CFA03460121184614F04BFBCAE3A0
S315080266B00D4B1B881946154812F0E0F8C3E300BFD4
S315080266C0741D0120F41C0120E07B05087C1E0120B4
S315080266D0F51C0120FC7B0508801E01201C7C050890
S315080266E0387C0508841E0120C01E0120C21E012016
S315080266F0C31E0120C41E0120C61E0120C81E012079
S31508026700C91E0120CA1E0120587C0508AC7C050852
S31508026710BB49BC4811F06BF814F040FA0346184618
S3150802672014F004FB0346002B40F0AA80B64B002265
S315080267301A80B34810F042FA03461A46B34B1A7047
S31508026740AF4810F056FA03461A46B14B1A70AC48CF
S3150802675010F06AFA03461A46AE4B1A80AE4B01226D
S315080267601A70A74810F07BFA03461A46AB4B1A7002
S31508026770A34810F08FFA03461A46A94B1A70A24B81
S315080267801B881C46A14B1B781D46A14B1B781E462F
S31508026790A04B1B881A46A04B1B7819469F4B1B78A1
S315080267A018469F4B1B780393029001910092334639
S315080267B02A4621469B4812F061F814F0EFF9024680
S315080267C0914B1B881946104614F0D7FA14F0E6F9CD
S315080267D002468E4B1B781946104614F0DDFA14F061
S315080267E0DDF902468A4B1B781946104614F0EFFA71
S315080267F014F0D4F903460121184614F003FB14F0E9
S31508026800CDF90246834B1B881946104614F015FB30
S3150802681014F0C4F90246804B1B781946104614F048
S3150802682027FB14F0BBF902467C4B1B781946104627
S3150802683014F039FB14F0B2F90246794B1B78194663
S31508026840104614F04BFB14F0A9F903460121184629
S3150802685014F05FFB29F0FEFD0346184629F036FEC2
S3150802686003460021184627F06FFD14F097F90346F0
S315080268700121184614F066FA6B4B01221A70E2E2FD
S31508026880614B1B881946694811F0F8FFDBE2684933
S315080268905C4811F083F812F0CBFA0346184612F058
S315080268A0A7FB0346002B40F0D780624B00221A80D2
S315080268B05F4810F040FA03461A465F4B1A705C4866
S315080268C010F054FA03461A465C4B1A70584810F0F0
S315080268D068FA03461A465A4B1A80554810F07CFA4B
S315080268E003461A46574B1A70514810F090FA034657
S315080268F01A46554B1A704E4810F0A4FA03461A4621
S31508026900524B1A704B4B1B881C464B4B1B781D4629
S315080269104A4B1B781E464A4B1B881A46494B1B781C
S315080269201946494B1B781846484B1B780393029025
S315080269300191009233462A462146454811F09EFFA8
S3150802694012F076FA02463B4B1B881946104612F09D
S3150802695076FB12F06DFA0246374B1B78194610463B
S3150802696012F07CFB12F064FA0246344B1B78194685
S31508026970104612F08EFB12F05BFA0246304B1B8869
S31508026980194689000B4419468800194603460B44E2
S315080269909B009BB21946104612F096FB12F048FA73
S315080269A00246284B1B781946104612F09CFB12F039
S315080269B03FFA0246244B1B781946104612F0AEFBE4
S315080269C012F036FA0246214B1B781946104612F087
S315080269D0C0FB29F03FFD0346184629F077FD03461A
S315080269E00021184627F07EFD12F022FA03460121FD
S315080269F0184612F009FB174B01221A7023E200BF50
S31508026A008C1E0120F51C0120C01E0120C21E012079
S31508026A10C31E0120C61E0120C81E0120C91E012050
S31508026A20CA1E0120E47C0508BC1E0120347D050827
S31508026A30981E0120CC1E0120CE1E0120CF1E012049
S31508026A40D01E0120D21E0120D31E0120D41E0120F1
S31508026A50687D0508BD1E012004F0DCFF03461846C2
S31508026A6004F0F0FF0346184605F0B8FB0346002B70
S31508026A7006D0BF4B1B881946BE4811F0FFFEE2E15D
S31508026A80BB4B1B881946BC4811F0F8FEDBE1BB4933
S31508026A90BB4811F04DF812F0CBF90346184612F02E
S31508026AA0A7FA0346002B40F0958004F0B3FF03468D
S31508026AB0184604F0C7FF0346184605F08FFB03463F
S31508026AC0002B40F0878004F0A5FF0346184604F021
S31508026AD0B9FF0346184605F070FA0346002B79D12A
S31508026AE004F098FF0346184604F0ACFF034618461E
S31508026AF005F07EFA0346002B6CD1A04810F0F3F994
S31508026B0003461A469F4B1A709C4810F007FA03462A
S31508026B101A469D4B1A70994810F01BFA03461A46F4
S31508026B209A4B1A70974B1B781946974B1B781A463D
S31508026B30964B1B78964811F0A1FE12F079F9034696
S31508026B400021184612F07BFA12F072F902468D4BB2
S31508026B501B781946104612F081FA12F069F90346B3
S31508026B60FF21184612F095FA12F062F9034600213F
S31508026B70184612F0A9FA12F05BF9034600211846E4
S31508026B8012F0B1FA12F054F902467F4B1B781946F5
S31508026B90104612F0C3FA12F04BF902467B4B1B78E9
S31508026BA01946104612F0D5FA29F054FC034618463F
S31508026BB029F08CFC03460021184627F093FC12F0B4
S31508026BC037F903460121184612F01EFA714B0122C3
S31508026BD01A7037E112F02CF90346184612F008FA31
S31508026BE00346002B02D06C4811F048FE04F012FF4F
S31508026BF00346184604F026FF0346184605F0EEFA41
S31508026C000346002B02D0654811F038FE04F002FF55
S31508026C100346184604F016FF0346184605F0CDF952
S31508026C200346002B02D05E4811F028FE04F0F2FE5D
S31508026C300346184604F006FF0346184605F0D8F937
S31508026C400346002B00F0FE80554811F017FEF9E0C6
S31508026C5054494B4811F011F8524810F0E8F9034626
S31508026C601A46514B1A704F4810F0FCF903461A4659
S31508026C704E4B1A704B4810F010FA03461A46920009
S31508026C8013441A4691001A460B4613449B009AB2BD
S31508026C90474B1A80454B1B78012B03D1454B0122E2
S31508026CA01A7002E0434B00221A703F4B1B783F4A88
S31508026CB012781146184605F0A5FD12F0B9F83A4BB6
S31508026CC01B78394A1278194612F062FA12F0B0F8AD
S31508026CD0354B1B78364A1288194612F07EFA12F09C
S31508026CE0A7F8314B1B78334A1278194612F09BFAE9
S31508026CF0A9E03149224811F05DF82F4810F005FA4B
S31508026D0003461A462D4B1A702B4810F019FA0346F9
S31508026D101A462B4B1A70284810F02DFA03461A46C3
S31508026D20284B1A70244810F041FA03461A46920074
S31508026D3013441A4691001A460B4613449B009AB20C
S31508026D40214B1A801E4B1B78012B03D11F4B0122A4
S31508026D501A7002E01D4B00221A70184B1B78012B81
S31508026D6036D1184B1B78184605F06EFA39E000BF83
S31508026D70CC1E0120BC7D0508F07D0508A41E012055
S31508026D80F51C0120D51E0120D61E0120D71E012082
S31508026D90247E0508BE1E01205C7E05088C7E050839
S31508026DA0BC7E0508AC1E0120D81E0120D91E012072
S31508026DB0DC1E0120DA1E0120B41E0120DE1E01207F
S31508026DC0DF1E0120E01E0120E21E0120E41E012032
S31508026DD01F4B1B78022B04D11E4B1B78184605F055
S31508026DE05DFAFB7919464FF4FA70FFF7FBFA184B6E
S31508026DF01B78194A12781146184605F003FD12F057
S31508026E0017F8134B1B78124A1278194612F030FA01
S31508026E1012F00EF80E4B1B78104A1288194612F019
S31508026E204CFA12F005F80A4B1B780D4A12781946E5
S31508026E3012F068FA07E00B4B1B7819460A4811F05C
S31508026E401DFD00E000BF00BF0C37BD46F0BD00BF08
S31508026E50DE1E0120E01E0120DF1E0120E21E0120A7
S31508026E60E41E0120F41C0120F07E050890B583B0CB
S31508026E7000AF0346FB71B44B1B78012B7AD129F07C
S31508026E80E9FA0346184629F021FB0346184627F075
S31508026E904FFA0346032B17D1AB4B00221A70012176
S31508026EA0AA480FF039FFAA49A84810F013FDA848C6
S31508026EB028F047FA0446A64828F04FFA0346194628
S31508026EC0204602F0BBFF55E029F0C4FA03461846ED
S31508026ED029F0FCFA0346184627F02AFA0346042B39
S31508026EE017D1994B00221A70002198480FF014FF07
S31508026EF09749964810F0EEFC954828F022FA04467F
S31508026F00934828F02AFA03461946204602F096FFC5
S31508026F1030E029F09FFA0346184629F0D7FA0346C5
S31508026F20184627F005FA0346002B23D029F092FAD1
S31508026F300346184629F0CAFA0346184627F0F8F90E
S31508026F400346022B16D0804B00221A7002217F4874
S31508026F500FF0E2FE7E497D4810F0BCFC7C4828F022
S31508026F60F0F904467A4828F0F8F903461946204605
S31508026F7002F064FF774B1B78012B40F0958029F0CD
S31508026F8069FA0346184629F0A1FA0346184627F075
S31508026F909DFA0346082B17D16E4B00221A7001215F
S31508026FA06D480FF091FF6A496B4810F075FD684805
S31508026FB028F0C7F90446664828F0CFF90346194669
S31508026FC0204602F03BFF6FE029F044FA03461846D2
S31508026FD029F07CFA0346184627F078FA0346092B65
S31508026FE017D15C4B00221A7000215B480FF06CFF28
S31508026FF05749594810F050FD554828F0A2F9044659
S31508027000534828F0AAF903461946204602F016FF05
S315080270104AE029F01FFA0346184629F057FA0346AA
S31508027020184627F053FA0346042B26D129F012FAFA
S315080270300346184629F04AFA0346184627F046FA3E
S315080270400346052B19D129F005FA0346184629F0F5
S315080270503DFA0346184627F039FA0346062B0CD1A1
S3150802706029F0F8F90346184629F030FA0346184675
S3150802707027F02CFA0346072B16D0364B00221A7035
S31508027080022135480FF020FF3149334810F004FD3C
S315080270902F4828F056F904462D4828F05EF903468B
S315080270A01946204602F0CAFE2C4B1B78012B40F0EB
S315080270B0978029F0CFF90346184629F007FA0346BE
S315080270C0184627F003FA0346082B17D1214B00224C
S315080270D01A70012122480FF07EFF1D49204810F040
S315080270E078FD1B4828F02DF90446194828F035F989
S315080270F003461946204602F0A1FE71E029F0AAF9D4
S315080271000346184629F0E2F90346184627F0DEF93F
S315080271100346092B26D10F4B00221A70002110486C
S315080271200FF059FF0A490E4810F053FD084828F097
S3150802713008F90446064828F010F903461946204677
S3150802714002F07CFE4CE000BFBC1E0120941E01200A
S31508027150781D0120BD1E0120A01E0120BE1E012091
S31508027160A81E012029F076F90346184629F0AEF939
S315080271700346184627F0AAF90346012B19D129F026
S3150802718069F90346184629F0A1F90346184627F075
S315080271909DF90346022B0CD129F05CF903461846E1
S315080271A029F094F90346184627F090F90346032B6B
S315080271B016D00D4B00221A7002210C480FF00BFF55
S315080271C00B490A4810F005FD094828F0BAF80446A2
S315080271D0074828F0C2F803461946204602F02EFE52
S315080271E000BF0C37BD4690BDBD1E0120A81E01205A
S315080271F0781D012080B582B000AF0346FB71FB798A
S31508027200332B02D101F00EFD4CE0FB79342B02D16F
S3150802721001F090FD46E0FB79352B02D101F00EFE16
S3150802722040E0FB79362B02D101F08CFE3AE0FB797D
S31508027230372B02D101F016FF34E0FB79382B02D145
S3150802724001F09CFF2EE0FB79392B02D102F022F8DD
S3150802725028E0FB793A2B02D102F0A8F822E0FB7962
S315080272603B2B02D102F02EF91CE0FB793C2B02D112
S3150802727002F0B4F916E0FB793D2B02D102F03EFA90
S3150802728010E0FB793E2B02D102F0C4FA0AE0FB7940
S315080272903F2B02D102F042FB04E0FB79402B01D1DD
S315080272A002F0C0FB00BF0837BD4680BD80B582B07C
S315080272B000AF0346FB71FB79332B02D101F0F6FCD2
S315080272C04CE0FB79342B02D101F076FD46E0FB79DE
S315080272D0352B02D101F0F4FD40E0FB79362B02D1C1
S315080272E001F078FE3AE0FB79372B02D101F000FF74
S315080272F034E0FB79382B02D101F086FF2EE0FB79C8
S31508027300392B02D102F00CF828E0FB793A2B02D18C
S3150802731002F092F822E0FB793B2B02D102F018F92F
S315080273201CE0FB793C2B02D102F0A0F916E0FB79AE
S315080273303D2B02D102F028FA10E0FB793E2B02D14E
S3150802734002F0AAFA0AE0FB793F2B02D102F028FBE7
S3150802735004E0FB79402B01D102F0A6FB00BF0837F7
S31508027360BD4680BD80B500AF01F07EFC01F0C0FCD1
S3150802737001F000FD01F040FD01F080FD01F0C0FDC5
S3150802738001F004FE01F04AFE01F08EFE01F0D2FE83
S3150802739001F016FF01F05AFF01F09EFF01F0E2FF2D
S315080273A002F026F802F06AF802F0AEF802F0F2F8F5
S315080273B002F038F902F07EF902F0C2F902F006FA92
S315080273C002F048FA02F088FA02F0C8FA02F008FB5C
S315080273D002F048FB02F088FB00BF80BD80B582B090
S315080273E000AF0346FB71FB79013B072B5AD801A272
S315080273F052F823F015740208277402083974020831
S315080274004B7402085D7402086F74020881740208DC
S315080274109374020811F08EFA0346184611F00EFB11
S31508027420F0EE407A40E011F085FA0346184611F06C
S3150802743023FBF0EE407A37E011F07CFA0346184651
S3150802744011F038FBF0EE407A2EE011F073FA03469B
S31508027450184611F04DFBF0EE407A25E011F06AFA73
S315080274600346184611F062FBF0EE407A1CE011F072
S3150802747061FA0346184611F077FBF0EE407A13E0FC
S3150802748011F058FA0346184611F08CFBF0EE407AD2
S315080274900AE011F04FFA0346184611F0A1FBF0EE86
S315080274A0407A01E0DFED037AB0EE670A0837BD4697
S315080274B080BD00BF0000000080B483B000AF034661
S315080274C00A46FB711346BB80FB79322B0BD9FB7933
S315080274D0402B08D8074AFB791370074ABB881380E2
S315080274E0064B01221A7000BF0C37BD465DF8047BB5
S315080274F0704700BFE81E0120E61E0120E51E012096
S3150802750080B500AF0F4B1B78002B19D00E4B1B888A
S31508027510002B08D10B4B00221A700C4B00221A7052
S3150802752000F0BAF80CE0084B1B88013B9AB2064BEE
S315080275301A80064B1B7864220221184600F08EF840
S3150802754000BF80BDE51E0120E61E0120E81E0120BF
S3150802755080B584B000AF03460A46FB711346BB7179
S315080275600023FB60FB7996211846FFF7A5FF002347
S31508027570FB6009E0642022F0EFF9BB79184616F0A1
S31508027580C7FDFB680133FB60FB68042BF2D900BF19
S3150802759000BF1037BD4680BD80B500AFFFF7B0FF0C
S315080275A02A4B1B78002B03D0294B1B78002B02D1C0
S315080275B0FFF7D8FE3BE0274B1B78002B02D1FFF7DB
S315080275C0D1FE34E0234B1B78642B13D1204B1B7856
S315080275D0012B05D11D4B1B781846FFF70BFE26E03B
S315080275E01B4B1B78022B22D1184B1B781846FFF728
S315080275F05DFE1CE0174B1B785B00174A1288934204
S3150802760013DB134B1B78012B05D1104B1B7818463D
S31508027610FFF7F0FD0BE00E4B1B78022B07D10B4B45
S315080276201B781846FFF742FE01E0FFF79BFE0A4B5E
S315080276301B8801339AB2084B1A80074B1B88C82B42
S3150802764002D9054B01221A8000BF80BDEA1E01201D
S31508027650EB1E0120E91E0120EC1E012080B483B036
S3150802766000AF0346FB710B46BB7113467B71074A93
S31508027670BB791370064AFB791370064A7B79137035
S3150802768000BF0C37BD465DF8047B7047EB1E012030
S31508027690EA1E0120E91E012080B400AF064B002233
S315080276A01A70064B00221A70054B00221A7000BF88
S315080276B0BD465DF8047B7047EB1E0120EA1E0120D9
S315080276C0E91E012090B585B000AF0446084611466A
S315080276D01A462346FB710346BB710B467B7113465A
S315080276E03B710023FB81FB79322B40F2F081FB7957
S315080276F0402B00F2EC81BB79022B00F2E881F97982
S315080277007A79BB79B64816F061F9FB79333B0D2BCA
S3150802771000F2A78101A252F823F000BF55770208AA
S315080277208D770208C5770208FD77020835780208C0
S315080277306D780208A5780208DD780208157902082C
S315080277404D79020885790208BB790208F779020899
S315080277502D7A0208BB79002B05D164220121332038
S31508027760FFF77CFF81E1BB79012B05D16422012158
S315080277703320FFF773FF78E1BB79022B40F075815E
S31508027780642202213320FFF769FF6EE1BB79002BE1
S3150802779005D1642201213420FFF760FF67E1BB7936
S315080277A0012B05D1642201213420FFF757FF5EE140
S315080277B0BB79022B40F05B81642202213420FFF759
S315080277C04DFF54E1BB79002B05D1642201213520F6
S315080277D0FFF744FF4DE1BB79012B05D16422012154
S315080277E03520FFF73BFF44E1BB79022B40F041818C
S315080277F0642202213520FFF731FF3AE1BB79002BDB
S3150802780005D1642201213620FFF728FF33E1BB792F
S31508027810012B05D1642201213620FFF71FFF2AE139
S31508027820BB79022B40F02781642202213620FFF71A
S3150802783015FF20E1BB79002B05D1642201213720EF
S31508027840FFF70CFF19E1BB79012B05D1642201214F
S315080278503720FFF703FF10E1BB79022B40F00D81B9
S31508027860642202213720FFF7F9FE06E1BB79002BD5
S3150802787005D1642201213820FFF7F0FEFFE0BB792B
S31508027880012B05D1642201213820FFF7E7FEF6E035
S31508027890BB79022B40F0F380642202213820FFF7DD
S315080278A0DDFEECE0BB79002B05D1642201213920EB
S315080278B0FFF7D4FEE5E0BB79012B05D1642201214D
S315080278C03920FFF7CBFEDCE0BB79022B40F0D980EA
S315080278D0642202213920FFF7C1FED2E0BB79002BD0
S315080278E005D1642201213A20FFF7B8FECBE0BB7925
S315080278F0012B05D1642201213A20FFF7AFFEC2E02F
S31508027900BB79022B40F0BF80642202213A20FFF79E
S31508027910A5FEB8E0BB79002B05D1642201213B20E4
S31508027920FFF79CFEB1E0BB79012B05D16422012148
S315080279303B20FFF793FEA8E0BB79022B40F0A58017
S31508027940642202213B20FFF789FE9EE0BB79002BC9
S3150802795005D1642201213C20FFF780FE97E0BB791E
S31508027960012B05D1642201213C20FFF777FE8EE028
S31508027970BB79022B40F08B80642202213C20FFF760
S315080279806DFE84E0BB79002B05D1642201213D20DE
S31508027990FFF764FE7DE0BB79012B05D16422012144
S315080279A03D20FFF75BFE74E0BB79022B71D164229E
S315080279B002213D20FFF752FE6BE0BB79002B05D171
S315080279C0642201213E20FFF749FE64E0BB79012BC0
S315080279D008D1642201213E20FFF740FE5BE000BF8A
S315080279E0107F0508BB79022B55D1642202213E205D
S315080279F0FFF734FE4FE0BB79002B05D16422012143
S31508027A003F20FFF72BFE48E0BB79012B05D1642204
S31508027A1001213F20FFF722FE3FE0BB79022B3CD132
S31508027A20642202213F20FFF719FE36E0BB79002BBC
S31508027A3005D1642201214020FFF710FE2FE0BB7911
S31508027A40012B05D1642201214020FFF707FE26E01B
S31508027A50BB79022B23D1642202214020FFF7FEFDC7
S31508027A601DE01D4815F0B2FF1AE000BF18E000BF7E
S31508027A7016E000BF14E000BF12E000BF10E000BF2E
S31508027A800EE000BF0CE000BF0AE000BF08E000BF3E
S31508027A9006E000BF04E000BF02E000BF00E000BF4E
S31508027AA00023FB810AE097F82030184616F030FBCF
S31508027AB0642021F051FFFB890133FB817B799BB25C
S31508027AC0FA899A42EFD3FFF7E7FD012300E0002384
S31508027AD018461437BD4690BD407F050880B582B06A
S31508027AE000AF034687ED000AFB710B46BB711346CE
S31508027AF07B71FB79012B02D0FB79032B2AD1BB7947
S31508027B001846FFF76BFCB0EE407AD7ED007A77EEAF
S31508027B10677AB7EE007A37EE877A7B7907EE903A7C
S31508027B20F8EEE77AB4EEE77AF1EE10FA0DDB214BBE
S31508027B301B6801331F4A13601E4B1B68B3F57A7F15
S31508027B4001D3022331E001232FE01A4B00221A60E7
S31508027B5000232AE0BB791846FFF740FCB0EE407ACC
S31508027B60D7ED007A77EE677AB7EE007A37EE877A3C
S31508027B707B7907EE903AF8EEE77AB4EEE77AF1EE19
S31508027B8010FA0EDB0B4B1B6801330A4A1360094BCA
S31508027B901B6840F2DB52934201D9022305E0012316
S31508027BA003E0044B00221A60002318460837BD4634
S31508027BB080BD00BFF01E0120B0B584B000AF0346F9
S31508027BC087ED020AC7ED010AFB730B46BB73134620
S31508027BD07B73FB7B012B02D0FB7B032B44D1BB7B44
S31508027BE01846FFF7FBFBB0EE407AD7ED027A77EE3E
S31508027BF0677A17EE900AF8F7D5FD04460D467868B7
S31508027C00F8F7D0FD4FF000023C4BF8F76DFC024640
S31508027C100B4620462946F9F7A3F80346002B21D13D
S31508027C20BB7B1846FFF7DAFBB0EE407AD7ED027A4D
S31508027C3077EE677A17EE900AF8F7B4FD04460D4612
S31508027C407868F8F7AFFD4FF000022C4BF8F74CFCBA
S31508027C5002460B4620462946F9F782F80346002BC8
S31508027C6000D145E0012344E0BB7B1846FFF7B6FB8B
S31508027C70B0EE407AD7ED027A77EE677A17EE900A77
S31508027C80F8F790FD04460D467868F8F78BFD4FF035
S31508027C9000021A4BF8F728FC02460B4620462946EC
S31508027CA0F9F75EF80346002B20D1BB7B1846FFF78F
S31508027CB095FBB0EE407AD7ED027A77EE677A17EE41
S31508027CC0900AF8F76FFD04460D467868F8F76AFDDC
S31508027CD04FF00002094BF8F707FC02460B4620460E
S31508027CE02946F9F73DF80346002B01D0012300E0A7
S31508027CF0002318461037BD46B0BD00BF0000044039
S31508027D0080B582B000AF034687ED000AFB710B46C9
S31508027D10BB7113467B71FB79012B02D0FB79032BCE
S31508027D2024D1BB791846FFF759FBB0EE407AD7ED56
S31508027D30007A77EE677AB7EE007AF4EEC77AF1EE52
S31508027D4010FA11DABB791846FFF748FBB0EE407A0B
S31508027D50D7ED007A77EE677AB7EE007AF4EEC77A4D
S31508027D60F1EE10FA00DA25E0012324E0BB79184681
S31508027D70FFF734FBB0EE407AD7ED007A77EE677AF2
S31508027D80B7EE007AF4EEC77AF1EE10FA10DABB799A
S31508027D901846FFF723FBB0EE407AD7ED007A77EE66
S31508027DA0677AB7EE007AF4EEC77AF1EE10FA01DBDB
S31508027DB0012300E0002318460837BD4680BD0000AF
S31508027DC0B0B584B000AF034687ED020AC7ED010AD3
S31508027DD0FB730B46BB7313467B73FB7B012B02D0EB
S31508027DE0FB7B032B44D1BB7B1846FFF7F7FAB0EEB1
S31508027DF0407AD7ED027A77EE677A17EE900AF8F7A5
S31508027E00D1FC04460D467868F8F7CCFC4FF0000220
S31508027E103C4BF8F769FB02460B4620462946F8F71B
S31508027E209FFF0346002B21D1BB7B1846FFF7D6FAE4
S31508027E30B0EE407AD7ED027A77EE677A17EE900AB5
S31508027E40F8F7B0FC04460D467868F8F7ABFC4FF035
S31508027E5000022C4BF8F748FB02460B4620462946F9
S31508027E60F8F77EFF0346002B00D145E0012344E0E4
S31508027E70BB7B1846FFF7B2FAB0EE407AD7ED027A24
S31508027E8077EE677A17EE900AF8F78CFC04460D46E9
S31508027E907868F8F787FC4FF000021A4BF8F724FBCC
S31508027EA002460B4620462946F8F75AFF0346002B98
S31508027EB020D1BB7B1846FFF791FAB0EE407AD7ED90
S31508027EC0027A77EE677A17EE900AF8F76BFC0446A1
S31508027ED00D467868F8F766FC4FF00002094BF8F78A
S31508027EE003FB02460B4620462946F8F739FF0346A6
S31508027EF0002B01D0012300E0002318461037BD46A7
S31508027F00B0BD00BF0000F03F80B582B000AF0346A7
S31508027F1087ED000AFB710B46BB7113467B71FB7931
S31508027F20012B02D0FB79032B32D1BB791846FFF716
S31508027F3055FAB0EE407AD7ED007A77EE677AB3EE65
S31508027F40027A37EE877A7B7907EE903AF8EEE77A85
S31508027F50B4EEE77AF1EE10FA18DABB791846FFF7AB
S31508027F603DFAB0EE407AD7ED007A77EE677AB3EE4D
S31508027F70027A37EE877A7B7907EE903AF8EEE77A55
S31508027F80B4EEE77AF1EE10FA00DA33E0012332E0D2
S31508027F90BB791846FFF722FAB0EE407AD7ED007A97
S31508027FA077EE677AB1EE047A37EE877A7B7907EE4F
S31508027FB0903AF8EEE77AB4EEE77AF1EE10FA17DAC3
S31508027FC0BB791846FFF70AFAB0EE407AD7ED007A7F
S31508027FD077EE677AB1EE047A37EE877A7B7907EE1F
S31508027FE0903AF8EEE77AB4EEE77AF1EE10FA01DBA8
S31508027FF0012300E0002318460837BD4680BD00006D
S3150802800080B582B000AF03463A60FB710B46BB717E
S31508028010BB79012B16D13B681B68B3F5FA6F5DD3A2
S315080280203B6800221A60FB79602B02D96423FB7134
S3150802803002E0FB790433FB71FB7919462A4815F0ED
S31508028040C5FC4BE0BB79022B17D13B681B6840F293
S31508028050DB52934242D93B6800221A60FB79582BBD
S3150802806002D96423FB7102E0FB790C33FB71FB79BD
S3150802807019461D4815F0AAFC30E0BB79032B16D128
S315080280803B681B68B3F5FA6F28D33B6800221A606F
S31508028090FB79602B02D96423FB7102E0FB79043376
S315080280A0FB71FB791946104815F090FC16E03B68FF
S315080280B01B6840F2DB52934210D93B6800221A60D1
S315080280C0FB79582B02D96423FB7102E0FB790C3346
S315080280D0FB71FB791946044815F078FCFB791846BA
S315080280E00837BD4680BD00BF4C7F050880B582B003
S315080280F000AF03463A60FB710B46BB71BB79012B95
S3150802810016D13B681B68B3F5FA6F5DD33B6800224C
S315080281101A60FB795E2B02D96423FB7102E0FB79B4
S315080281200633FB71FB7919462A4815F04FFC4BE0DA
S31508028130BB79022B17D13B681B6840F2DB5293428C
S3150802814042D93B6800221A60FB79582B02D964236C
S31508028150FB7102E0FB790C33FB71FB7919461D486A
S3150802816015F034FC30E0BB79032B16D13B681B684B
S31508028170B3F5FA6F28D33B6800221A60FB795E2BA7
S3150802818002D96423FB7102E0FB790633FB71FB79A2
S315080281901946104815F01AFC16E03B681B6840F2AF
S315080281A0DB52934210D93B6800221A60FB79582B9E
S315080281B002D96423FB7102E0FB790C33FB71FB796C
S315080281C01946044815F002FCFB7918460837BD46DD
S315080281D080BD00BF747F050890B58BB000AF04461A
S315080281E0084611461A462346FB710346BB710B46DF
S315080281F07B7113463B710023FB75002387F82730F2
S315080282004FF000033B614FF000033B620023FB770C
S315080282100023BB770023BB610023BB600023FB73EB
S315080282200023BB7300237B73FB79322B25D9FB7999
S31508028230402B22D8BB79002B1FD0BB79082B1CD820
S31508028240F979BA797B79A84815F0C0FB386AF8F744
S31508028250A9FA02460B46A54810F010FBBB79184648
S31508028260FFF7BCF887ED040A4FF000033B620023D0
S31508028270FB773B79012B06D002E0002300F015BC00
S315080282803B79032B13D17B790C2B01D80123FB777E
S315080282903B79012B02D10E23BB771BE03B79032BDB
S315080282A002D10E23BB7715E00E23BB7712E07B794A
S315080282B0062B01D80123FB773B79002B02D15023E9
S315080282C0BB7707E03B79022B02D15023BB7701E04B
S315080282D05023BB77FB7F002B40F016810023BB613E
S315080282E00023BB600023FB75002387F82730386A12
S315080282F0F8F758FA02460B467D4810F0BFFA7A7923
S31508028300B9793B7997ED040A1846FFF7E7FB034666
S31508028310FB75FB7D022B0ED1FFF7BEF997F83830B5
S31508028320002B06D097F83C20FB7911461846FFF732
S315080283300FF90123B9E37A79B9793B7997ED040AFA
S315080283401846FFF7DDFC0346FB73FB7B002B0AD0BE
S31508028350FFF7A2F9386AF8F725FA02460B46654886
S3150802836015F034FBD0E0FB7D012B02D1FFF794F91F
S315080283700FE03B79032B06D0BB6941F6583293428C
S3150802838001D96423BB77BA7FFB7901211846FFF727
S3150802839065F97A79B9793B79D7ED080A97ED040A2E
S315080283A01846FFF70DFD0346BB73BB7B83F001033B
S315080283B0DBB2002B35D097F82730012B11D1FB7D84
S315080283C0002B0ED10023BB60BB791846FFF706F8CF
S315080283D0B0EE407AD7ED047A77EE677AC7ED087A77
S315080283E002E0FB7D87F82730BB680133BB60BB68B8
S315080283F0B3F5FA6F25D30023BB60BB7F5A2B02D98C
S315080284006423BB7702E0BB7F0A33BB77BC7F386A3B
S31508028410F8F7C8F902460B462146374815F0D6FA48
S315080284200FE00023BB600023BB61BB791846FEF749
S31508028430D5FFB0EE407AD7ED047A77EE677AC7EDC4
S31508028440087ABB690133BB61BB6942F6DF629342B4
S3150802845011D9FFF721F9294810F010FA97F83830A0
S31508028460002B06D097F83C20FB7911461846FFF7F1
S315080284706FF8002319E310F05DFA0346184610F068
S31508028480C4FA0346002B06D0FFF706F91C4810F07B
S31508028490F5F9002309E327F0DDFF0346184628F01D
S315080284A015F80346184625F043FF0346022B06D065
S315080284B0FFF7F2F8134810F0E1F90023F5E201207C
S315080284C021F04AFA97F83C30184615F021FE27F0B3
S315080284D0C1FF0346184627F0F9FF034697ED080A37
S315080284E0184625F06AFF0AE79C7F0508C87F050833
S315080284F0E47F0508088005083480050868800508B1
S3150802850084800508A0800508BB791846FEF766FF31
S31508028510B0EE407AD7ED047A77EE677AB1EE007A52
S3150802852037EE877A7B7907EE903AF8EEE77AB4EE79
S31508028530E77AF1EE10FA47DABB791846FEF74EFFEC
S31508028540B0EE407AD7ED047A77EE677AB3EE027A1E
S3150802855037EE877A7B7907EE903AF8EEE77AB4EE49
S31508028560E77AF1EE10FA2FDABB791846FEF736FFEC
S31508028570B0EE407AD7ED047A77EE677AB1EE007AF2
S3150802858037EE877A7B7907EE903AF8EEE77AB4EE19
S31508028590E77AF1EE10FA17DABB791846FEF71EFFEC
S315080285A0B0EE407AD7ED047A77EE677AB3EE027ABE
S315080285B037EE877A7B7907EE903AF8EEE77AB4EEE9
S315080285C0E77AF1EE10FA01DB0123FB77386AF8F74E
S315080285D0E9F802460B46BC4810F050F9FB7F002B1F
S315080285E040F024813B79002B02D15A23BB7713E052
S315080285F03B79012B02D10E23BB770DE03B79022B87
S3150802860002D15A23BB7707E03B79032B02D10E230B
S31508028610BB7701E05A23BB770023BB610023BB600B
S315080286200023FB75002387F82730BB791846FEF727
S31508028630D5FEB0EE407AD7ED047A77EE677AC7EDC3
S31508028640087A386AF8F7AEF802460B469F4810F0E1
S3150802865015F97A79B9793B7997ED040A1846FFF73D
S315080286603DFA0346FB75FB7D022B0ED1FFF714F884
S3150802867097F83830002B06D097F83C20FB7911463C
S315080286801846FEF765FF01230FE27A79B9793B7935
S3150802869097ED040A1846FFF737FC03467B737B7B84
S315080286A0002B0AD0FEF7F8FF386AF8F77BF802467D
S315080286B00B46874815F08AF9B8E0FB7D012B02D1F3
S315080286C0FEF7EAFF0FE03B79032B06D0BB6944F2BB
S315080286D05062934201D96423BB77BA7FFB790121A1
S315080286E01846FEF7BBFF7A79B9793B79D7ED080ABE
S315080286F097ED040A1846FFF75FFA0346BB73BB7B7E
S3150802870083F00103DBB2002B25D097F82730012B23
S3150802871011D1FB7D002B0ED10023BB60BB79184615
S31508028720FEF75CFEB0EE407AD7ED047A77EE677A0A
S31508028730C7ED087A02E0FB7D87F82730BB6801336C
S31508028740BB6007F108023979BB7F1846FFF758FC68
S315080287500346BB7717E0386AF8F724F802460B4651
S315080287605C4815F033F90023BB600023BB61BB7973
S315080287701846FEF733FEB0EE407AD7ED047A77EE66
S31508028780677AC7ED087ABB690133BB61BB6945F6EF
S31508028790BF52934211D9FEF77FFF4F4810F06EF889
S315080287A097F83830002B06D097F83C20FB7911460B
S315080287B01846FEF7CDFE002377E110F0BBF8034614
S315080287C0184610F022F90346002B06D0FEF764FF7E
S315080287D0424810F053F8002367E127F03BFE0346B0
S315080287E0184627F073FE0346184625F0A1FD0346F0
S315080287F0022B06D0FEF750FF394810F03FF8002347
S3150802880053E1012021F0A8F897F83C30184615F0F4
S315080288107FFC27F01FFE0346184627F057FE03463D
S3150802882097ED080A184625F0C8FD12E73B79002B92
S3150802883002D12823BB7713E03B79012B02D10C2303
S31508028840BB770DE03B79022B02D12823BB7707E0E1
S315080288503B79032B02D10C23BB7701E02823BB7794
S315080288600023BB610023BB600023FB75002387F846
S315080288702730BB791846FEF7B1FDB0EE407AD7ED40
S31508028880047A77EE677AC7ED087A386AF7F78AFFC5
S3150802889002460B4613480FF0F1FF7A79B9793B790C
S315080288A097ED040A1846FFF719F90346FB75FB7D8F
S315080288B0022B19D1FEF7F0FE00BF97F83830002BCD
S315080288C000F0D280C9E000BFB4800508D880050848
S315080288D0FC80050828810508588105088480050852
S315080288E0A080050874810508FB7D012B02D1FEF7DD
S315080288F0D3FE0FE03B79032B06D0BB6944F25062E4
S31508028900934201D96423BB77BA7FFB7901211846C2
S31508028910FEF7A4FE7A79B9793B79D7ED080A97ED7D
S31508028920040A1846FFF748F90346BB73BB7B83F074
S315080289300103DBB2002B25D097F82730012B11D182
S31508028940FB7D002B0ED10023BB60BB791846FEF7D0
S3150802895045FDB0EE407AD7ED047A77EE677AC7ED31
S31508028960087A02E0FB7D87F82730BB680133BB60D3
S3150802897007F108023979BB7F1846FFF7B7FB0346AA
S31508028980BB7717E0386AF7F70DFF02460B464948E8
S3150802899015F01CF80023BB600023BB61BB7918469F
S315080289A0FEF71CFDB0EE407AD7ED047A77EE677AC9
S315080289B0C7ED087ABB690133BB61BB6945F6BF528D
S315080289C0934211D9FEF768FE3B480FF057FF97F816
S315080289D03830002B06D097F83C20FB79114618460A
S315080289E0FEF7B6FD002360E00FF0A4FF0346184623
S315080289F010F00BF80346002B06D0FEF74DFE2F4863
S31508028A000FF03CFF002350E027F024FD03461846EA
S31508028A1027F05CFD0346184625F08AFC0346022B1E
S31508028A2006D0FEF739FE26480FF028FF00233CE061
S31508028A30012020F091FF97F83C30184615F068FBA4
S31508028A4027F008FD0346184627F040FD034697ED32
S31508028A50080A184625F0B1FC1FE797F83C20FB796F
S31508028A6011461846FEF774FDBB791846FEF7B6FCA2
S31508028A70B0EE407AD7ED047A77EE677AC7ED087AD0
S31508028A80386AF7F78FFE02460B460E480FF0F6FED7
S31508028A9027F0E0FC0346184627F018FD034697ED33
S31508028AA0080A184625F089FC012318462C37BD46C4
S31508028AB090BD00BF98810508CC8105088480050809
S31508028AC0A0800508E881050880B400AF3B4B1B78F7
S31508028AD0002B6DD13A4B1B78002B69D1394B1B7889
S31508028AE0002B65D1384B1B78002B61D1374B1B788D
S31508028AF0002B5DD1364B1B78002B59D1354B1B7891
S31508028B00002B55D1344B1B78002B51D1334B1B7894
S31508028B10002B4DD1324B1B78002B49D1314B1B7898
S31508028B20002B45D1304B1B78002B41D12F4B1B789C
S31508028B30002B3DD12E4B1B78002B39D12D4B1B78A0
S31508028B40002B35D12C4B1B78002B31D12B4B1B78A4
S31508028B50002B2DD12A4B1B78002B29D1294B1B78A8
S31508028B60002B25D1284B1B78002B21D1274B1B78AC
S31508028B70002B1DD1254B1B78002B19D1244B1B78B2
S31508028B80002B15D1234B1B78002B11D1224B1B78B6
S31508028B90002B0DD1214B1B78002B09D1204B1B78BA
S31508028BA0002B05D11E4B1B78002B01D1012300E0B7
S31508028BB000231846BD465DF8047B7047F41E012063
S31508028BC0F51E0120F61E0120F71E0120F81E0120BF
S31508028BD0F91E0120FA1E0120FB1E0120FC1E01209F
S31508028BE0FD1E0120FE1E0120FF1E0120001F01207E
S31508028BF0011F0120021F0120031F0120041F01205B
S31508028C00051F0120071F0120061F0120091F012039
S31508028C100A1F01200B1F01200D1F01200C1F012016
S31508028C200F1F012080B500AF0C4B1B78002B12D109
S31508028C3011F00AFE00224FF48071094816F082FEEE
S31508028C4001228021064816F07DFE044B01221A7085
S31508028C50044B00221A7000BF80BD00BFF41E01201B
S31508028C6000180242F51E012080B500AF0C4B002207
S31508028C701A700C4B00221A7001224FF480710A48AE
S31508028C8016F060FE01228021074816F05BFEFFF708
S31508028C901BFF0346002B01D011F01AFE00BF80BD50
S31508028CA0F41E0120F51E01200018024280B500AF0D
S31508028CB00C4B1B78002B12D111F0C6FD01224FF482
S31508028CC08071094816F03EFE00228021064816F0F9
S31508028CD039FE064B00221A70024B01221A7000BF97
S31508028CE080BD00BFF51E012000180242F41E0120B5
S31508028CF080B500AF0C4B00221A700C4B00221A707A
S31508028D0001224FF480710A4816F01CFE01228021C6
S31508028D10074816F017FEFFF7D7FE0346002B01D0C9
S31508028D2011F0D6FD00BF80BDF41E0120F51E0120FC
S31508028D300018024280B500AF0B4B1B78002B11D1ED
S31508028D4011F082FD00224021084816F0FBFD01229F
S31508028D502021064816F0F6FD034B01221A70044B31
S31508028D6000221A7000BF80BDF61E012000180242BA
S31508028D70F71E012080B500AF0C4B00221A700C4B6F
S31508028D8000221A70012240210A4816F0DBFD012250
S31508028D902021084816F0D6FDFFF796FE0346002B5B
S31508028DA001D011F095FD00BF80BD00BFF61E01205F
S31508028DB0F71E01200018024280B500AF0B4B1B7844
S31508028DC0002B11D111F040FD01224021084816F06E
S31508028DD0B9FD00222021064816F0B4FD054B0022F3
S31508028DE01A70024B01221A7000BF80BDF71E0120BD
S31508028DF000180242F61E012080B500AF0C4B002275
S31508028E001A700C4B00221A70012240210A4816F0E9
S31508028E1099FD01222021084816F094FDFFF754FE19
S31508028E200346002B01D011F053FD00BF80BD00BFE1
S31508028E30F61E0120F71E01200018024280B500AF77
S31508028E400B4B1B78002B11D111F0FEFC00221021CE
S31508028E50084816F077FD01220821064816F072FD29
S31508028E60034B01221A70044B00221A7000BF80BD00
S31508028E70F81E012000180242F91E012080B500AF33
S31508028E800C4B00221A700C4B00221A700122102178
S31508028E900A4816F057FD01220821084816F052FD25
S31508028EA0FFF712FE0346002B01D011F011FD00BF99
S31508028EB080BD00BFF81E0120F91E012000180242DB
S31508028EC080B500AF0B4B1B78002B11D111F0BCFCFF
S31508028ED001221021084816F035FD0022082106480D
S31508028EE016F030FD054B00221A70024B01221A7049
S31508028EF000BF80BDF91E012000180242F81E01209B
S31508028F0080B500AF0C4B00221A700C4B00221A7067
S31508028F10012210210A4816F015FD012208210848E7
S31508028F2016F010FDFFF7D0FD0346002B01D011F015
S31508028F30CFFC00BF80BD00BFF81E0120F91E01202C
S31508028F400018024280B500AF0C4B1B78002B12D1D9
S31508028F5011F07AFC00220421094816F0F3FC0122DA
S31508028F604FF40041074816F0EDFC044B01221A7033
S31508028F70054B00221A7000BF80BD00BFFA1E0120F1
S31508028F8000180242000C0242FB1E012080B500AF07
S31508028F900C4B00221A700C4B00221A700122042173
S31508028FA00A4816F0CFFC01224FF40041084816F091
S31508028FB0C9FCFFF789FD0346002B01D011F088FC96
S31508028FC000BF80BDFA1E0120FB1E012000180242C6
S31508028FD0000C024280B500AF0C4B1B78002B12D155
S31508028FE011F032FC01220421094816F0ABFC0022DA
S31508028FF04FF40041074816F0A5FC074B00221A70E9
S31508029000024B01221A7000BF80BD00BFFB1E012061
S3150802901000180242000C0242FA1E012080B500AF77
S315080290200C4B00221A700C4B00221A7001220421E2
S315080290300A4816F087FC01224FF40041084816F048
S3150802904081FCFFF741FD0346002B01D011F040FCDD
S3150802905000BF80BDFA1E0120FB1E01200018024235
S31508029060000C024280B500AF0C4B1B78002B13D1C3
S3150802907011F0EAFB00224FF40061094816F062FC7F
S3150802908001224FF48061064816F05CFC034B01226C
S315080290901A70044B00221A7000BF80BDFC1E012004
S315080290A0000C0242FD1E012080B500AF0D4B0022C6
S315080290B01A700D4B00221A7001224FF400610B48F8
S315080290C016F040FC01224FF48061084816F03AFC7B
S315080290D0FFF7FAFC0346002B01D011F0F9FB00BF9B
S315080290E080BD00BFFC1E0120FD1E0120000C0242AD
S315080290F080B500AF0C4B1B78002B13D111F0A4FBE3
S3150802910001224FF40061094816F01CFC00224FF4B4
S315080291108061064816F016FC054B00221A70024BAF
S3150802912001221A7000BF80BDFD1E0120000C0242FA
S31508029130FC1E012080B500AF0D4B00221A700D4BA4
S3150802914000221A7001224FF400610B4816F0FAFB4E
S3150802915001224FF48061084816F0F4FBFFF7B4FCCD
S315080291600346002B01D011F0B3FB00BF80BD00BF40
S31508029170FC1E0120FD1E0120000C024280B500AF34
S315080291800C4B1B78002B13D111F05EFB00224FF417
S315080291900071094816F0D6FB01224FF48071064881
S315080291A016F0D0FB034B01221A70044B00221A70E8
S315080291B000BF80BDFE1E0120000C0242FF1E0120D8
S315080291C080B500AF0D4B00221A700D4B00221A70A3
S315080291D001224FF400710B4816F0B4FB01224FF43A
S315080291E08071084816F0AEFBFFF76EFC0346002BAB
S315080291F001D011F06DFB00BF80BD00BFFE1E01202D
S31508029200FF1E0120000C024280B500AF0C4B1B78F2
S31508029210002B13D111F018FB01224FF400710948F3
S3150802922016F090FB00224FF48071064816F08AFB6E
S31508029230054B00221A70024B01221A7000BF80BD2C
S31508029240FF1E0120000C0242FE1E012080B500AF5F
S315080292500D4B00221A700D4B00221A7001224FF490
S3150802926000710B4816F06EFB01224FF48071084814
S3150802927016F068FBFFF728FC0346002B01D011F015
S3150802928027FB00BF80BD00BFFE1E0120FF1E012076
S31508029290000C024280B500AF0C4B1B78002B13D191
S315080292A011F0D2FA00224FF40051094816F04AFB8F
S315080292B001224FF48051064816F044FB034B012263
S315080292C01A70044B00221A7000BF80BD001F0120CD
S315080292D000040242011F012080B500AF0D4B002297
S315080292E01A700D4B00221A7001224FF400510B48D6
S315080292F016F028FB01224FF48051084816F022FB8B
S31508029300FFF7E2FB0346002B01D011F0E1FA00BF9A
S3150802931080BD00BF001F0120011F01200004024278
S3150802932080B500AF0C4B1B78002B13D111F08CFAC9
S3150802933001224FF40051094816F004FB00224FF4AB
S315080293408051064816F0FEFA054B00221A70024BA7
S3150802935001221A7000BF80BD011F012000040242CB
S31508029360001F012080B500AF0D4B00221A700D4B6D
S3150802937000221A7001224FF400510B4816F0E2FA45
S3150802938001224FF48051084816F0DCFAFFF79CFBDD
S315080293900346002B01D011F09BFA00BF80BD00BF27
S315080293A0001F0120011F01200004024280B500AF00
S315080293B00C4B1B78002B13D111F046FA00224FF4FE
S315080293C00071094816F0BEFA01224FF48071064868
S315080293D016F0B8FA034B01221A70044B00221A70CF
S315080293E000BF80BD021F012000100242031F012098
S315080293F080B500AF0D4B00221A700D4B00221A7071
S3150802940001224FF400710B4816F09CFA01224FF420
S315080294108071084816F096FAFFF756FB0346002BAA
S3150802942001D011F055FA00BF80BD00BF021F01200E
S31508029430031F01200010024280B500AF0C4B1B78B7
S31508029440002B13D111F000FA01224FF400710948DA
S3150802945016F078FA00224FF48071064816F072FA6E
S31508029460054B00221A70024B01221A7000BF80BDFA
S31508029470031F012000100242021F012080B500AF1F
S315080294800D4B00221A700D4B00221A7001224FF45E
S3150802949000710B4816F056FA01224FF480710848FB
S315080294A016F050FAFFF710FB0346002B01D011F015
S315080294B00FFA00BF80BD00BF021F0120031F012053
S315080294C00010024280B500AF0B4B1B78002B11D15E
S315080294D011F0BAF900228021084816F033FA01225F
S315080294E00221074816F02EFA034B01221A70054B81
S315080294F000221A7000BF80BD041F0120001002421C
S3150802950000180242051F012080B500AF0C4B00224D
S315080295101A700C4B00221A70012280210A4816F092
S3150802952011FA01220221094816F00CFAFFF7CCFAC1
S315080295300346002B01D011F0CBF900BF80BD00BF56
S31508029540041F0120051F01200010024200180242D2
S3150802955080B500AF0B4B1B78002B11D111F074F9B3
S3150802956001228021084816F0EDF900220221074857
S3150802957016F0E8F9064B00221A70024B01221A70FD
S3150802958000BF80BD051F01200010024200180242DA
S31508029590041F012080B500AF0C4B00221A700C4B39
S315080295A000221A70012280210A4816F0CBF90122FC
S315080295B00221094816F0C6F9FFF786FA0346002B78
S315080295C001D011F085F900BF80BD00BF041F01203C
S315080295D0051F0120001002420018024280B500AFA2
S315080295E00C4B1B78002B12D111F02EF90022012107
S315080295F0094816F0A7F901224FF40041074816F068
S31508029600A1F9044B01221A70054B00221A7000BFF9
S3150802961080BD00BF061F0120001802420014024244
S31508029620071F012080B500AF0C4B00221A700C4BA5
S3150802963000221A70012201210A4816F083F9012232
S315080296404FF40041084816F07DF9FFF73DFA034644
S31508029650002B01D011F03CF900BF80BD061F012086
S31508029660071F0120001802420014024280B500AF0B
S315080296700C4B1B78002B12D111F0E6F801220121BE
S31508029680094816F05FF900224FF40041074816F020
S3150802969059F9074B00221A70024B01221A7000BFB1
S315080296A080BD00BF071F01200018024200140242B3
S315080296B0061F012080B500AF0C4B00221A700C4B16
S315080296C000221A70012201210A4816F03BF90122EA
S315080296D04FF40041084816F035F9FFF7F5F9034645
S315080296E0002B01D011F0F4F800BF80BD061F01203F
S315080296F0071F0120001802420014024280B500AF7B
S315080297000C4B1B78002B13D111F09EF800224FF454
S315080297108041094816F016F901224FF4005106480D
S3150802972016F010F9034B01221A70044B00221A7024
S3150802973000BF80BD081F012000140242091F012034
S3150802974080B500AF0D4B00221A700D4B00221A701D
S3150802975001224FF480410B4816F0F4F801224FF427
S315080297600051084816F0EEF8FFF7AEF90346002B4B
S3150802977001D011F0ADF800BF80BD00BF081F01205F
S31508029780091F01200014024280B500AF0C4B1B785A
S31508029790002B13D111F058F801224FF480410948E1
S315080297A016F0D0F800224FF40051064816F0CAF80F
S315080297B0054B00221A70024B01221A7000BF80BDA7
S315080297C0091F012000140242081F012080B500AFBC
S315080297D00D4B00221A700D4B00221A7001224FF40B
S315080297E080410B4816F0AEF801224FF400510848A2
S315080297F016F0A8F8FFF768F90346002B01D011F016
S3150802980067F800BF80BD00BF081F0120091F01209D
S315080298100014024280B500AF0B4B1B78002B11D106
S3150802982011F012F800222021084816F08BF80122BE
S315080298301021064816F086F8034B01221A70044BCB
S3150802984000221A7000BF80BD0A1F012000080242CA
S315080298500B1F012080B500AF0C4B00221A700C4B6F
S3150802986000221A70012220210A4816F06BF80122FA
S315080298701021084816F066F8FFF726F90346002B6A
S3150802988001D011F025F800BF80BD00BF0A1F0120D4
S315080298900B1F01200008024280B500AF0B4B1B7854
S315080298A0002B11D110F0D0FF01222021084816F012
S315080298B049F800221021064816F044F8054B002202
S315080298C01A70024B01221A7000BF80BD0B1F0120BD
S315080298D0000802420A1F012080B500AF0C4B002285
S315080298E01A700C4B00221A70012220210A4816F01F
S315080298F029F801221021084816F024F8FFF7E4F89F
S315080299000346002B01D010F0E3FF00BF80BD00BF65
S315080299100A1F01200B1F01200008024280B500AF72
S315080299200B4B1B78002B11D110F08EFF00228021E1
S31508029930084816F007F801224021064816F002F8F0
S31508029940034B01221A70044B00221A7000BF80BD15
S315080299500C1F0120000002420D1F012080B500AF36
S315080299600C4B00221A700C4B00221A70012280211D
S315080299700A4815F0E7FF01224021084815F0E2FFE0
S31508029980FFF7A2F80346002B01D010F0A1FF00BF93
S3150802999080BD00BF0C1F01200D1F012000000242DE
S315080299A080B500AF0B4B1B78002B11D110F04CFF82
S315080299B001228021084815F0C5FF002240210648E9
S315080299C015F0C0FF054B00221A70024B01221A70CD
S315080299D000BF80BD0D1F0120000002420C1F01209E
S315080299E080B500AF0C4B00221A700C4B00221A707D
S315080299F0012280210A4815F0A5FF012240210848C4
S31508029A0015F0A0FFFFF760F80346002B01D010F00F
S31508029A105FFF00BF80BD00BF0C1F01200D1F012084
S31508029A200000024280B500AF0B4B1B78002B11D108
S31508029A3010F00AFF00222021084815F083FF0122B0
S31508029A401021064815F07EFF034B01221A70044BBB
S31508029A5000221A7000BF80BD0E1F012000000242BC
S31508029A600F1F012080B500AF0C4B00221A700C4B59
S31508029A7000221A70012220210A4815F063FF0122EA
S31508029A801021084815F05EFFFFF71EF80346002B63
S31508029A9001D010F01DFF00BF80BD00BF0E1F0120C0
S31508029AA00F1F01200000024280B500AF0B4B1B7846
S31508029AB0002B11D110F0C8FE01222021084815F00A
S31508029AC041FF00221021064815F03CFF054B0022F3
S31508029AD01A70024B01221A7000BF80BD0F1F0120A7
S31508029AE0000002420E1F012080B500AF0C4B002277
S31508029AF01A700C4B00221A70012220210A4815F00E
S31508029B0021FF01221021084815F01CFFFEF7DCFF91
S31508029B100346002B01D010F0DBFE00BF80BD00BF5C
S31508029B200E1F01200F1F01200000024280B500AF60
S31508029B3000220121044815F005FF002202210248ED
S31508029B4015F000FF00BF80BD000C024280B500AFD1
S31508029B5001220121044815F0F5FE012202210248DC
S31508029B6015F0F0FE00BF80BD000C024280B500AFC2
S31508029B7000220421024815F0E5FE00BF80BD00BFA1
S31508029B800010024280B500AF01220421024815F0F6
S31508029B90D9FE00BF80BD00BF0010024280B582B068
S31508029BA000AF78600B467B80104821F031FC0246F4
S31508029BB07B889A4214D34FF47A710D4820F014FE2A
S31508029BC00346002B0AD17B881A467968074821F092
S31508029BD008FE074820F062FE012302E0002300E0A7
S31508029BE0002318460837BD4680BD00BF101F012056
S31508029BF0B0F6002080B5C4B000AF024607F58873F8
S31508029C00A3F209131A70002387F80F312E4821F0A0
S31508029C105DFC034683F00103DBB2002B50D02B4BCD
S31508029C201B78002B4CD107F10C034FF480720021EC
S31508029C30184629F0A7FB4FF47A71254820F0D4FD7F
S31508029C400346002B39D107F10C0319461E4821F0A9
S31508029C503FFE034687F80F311D4820F01FFE4FF4DA
S31508029C607A711B4820F0C0FD0346002B27D107F165
S31508029C700C031946144821F0C5FD034687F80F312F
S31508029C80134820F00BFE4FF47A71124820F0ACFD0F
S31508029C900346002B0DD1FBF796FB97F80F319AB2C4
S31508029CA007F10C031946FBF7CFFC0A4820F0F6FD2C
S31508029CB006E0094813F08AFE02E000BF00E000BF92
S31508029CC007F58877BD4680BD101F01202020012098
S31508029CD0B0F60020E4F600200482050880B483B0BA
S31508029CE000AF78600B467B8000BF00BF0C37BD46CD
S31508029CF05DF8047B7047000080B582B000AF002390
S31508029D00FB712E4B1B78002B51D02D4B1B78013340
S31508029D10DAB22B4B1A702A4B1B78092B4AD9284BD5
S31508029D2000221A70254B5B78012B1FD8234B5B78D0
S31508029D300133DAB2214B5A704FF47A71214820F076
S31508029D4053FD0346002B0DD1FBF73DFB03461B4A89
S31508029D5092F883201C491846FBF776FC194820F02E
S31508029D609DFD27E0194813F031FE23E00023FB711D
S31508029D7002E0FB790133FB71104B93F88330FA79D1
S31508029D809A42F6D34FF47A71114820F02DFD034614
S31508029D90002B0FD10C490F4821F034FD0C4820F056
S31508029DA07DFD84220021054829F0ECFA02E0044BE5
S31508029DB000221A7000BF0837BD4680BD2020012048
S31508029DC0A4200120E4F600202320012004820508AD
S31508029DD0B0F60020101F012080B500AF4FF4807244
S31508029DE00249034821F0E8FA00BF80BD201F01207E
S31508029DF0101F012080B500AFFFF7EEFF00BF80BD40
S31508029E0080B582B000AF786039603B68DBB219462C
S31508029E10786800F04BF800BF0837BD4680BD80B5AC
S31508029E2082B000AF786039603B689BB219467868A1
S31508029E30FFF7B4FE00BF0837BD4680BD80B582B0C5
S31508029E4000AF78603960064B1B683A6892B2796847
S31508029E50184621F0ABF800BF0837BD4680BD00BFE3
S31508029E60A810002080B582B000AF78603960054B33
S31508029E701B683A687968184621F032F900BF083734
S31508029E80BD4680BDA810002080B500AF044B1868F7
S31508029E90044B054A002121F04EF800BF80BD00BFE1
S31508029EA0A81000201F9E0208019E02082DE9F04311
S31508029EB089B004AF78600B46FB700EF03BFDF86084
S31508029EC001F0A8FDB860FB789BB219467868FFF7DF
S31508029ED005FF7B681B78013BA12B01F2C28001A218
S31508029EE052F823F06DA1020863B0020863B00208B3
S31508029EF063B00208D3A1020863B0020863B002087D
S31508029F0063B0020863B0020863B0020863B00208CD
S31508029F1063B0020863B0020863B00208A9A1020886
S31508029F2063B0020863B0020863B0020863B00208AD
S31508029F3063B0020863B0020863B0020863B002089D
S31508029F4063B0020863B0020863B0020863B002088D
S31508029F5063B0020863B0020863B0020863B002087D
S31508029F600BA202083DA2020817A30208E5A30208EB
S31508029F7063B0020863B0020863B0020863B002085D
S31508029F80EFA3020839A4020863B0020863B0020804
S31508029F9063B0020863B0020863B0020863B002083D
S31508029FA063B0020863B0020863B0020863B002082D
S31508029FB063B0020863B0020863B0020863B002081D
S31508029FC063B0020863B0020863B0020863B002080D
S31508029FD063B0020863B0020863B0020863B00208FD
S31508029FE063B0020863B0020863B0020863B00208ED
S31508029FF063B0020863B0020863B0020863B00208DD
S3150802A00063B0020863B0020863B0020863B00208CC
S3150802A01063B0020863B0020863B0020863B00208BC
S3150802A02063B0020863B0020863B0020863B00208AC
S3150802A03063B0020863B0020863B0020863B002089C
S3150802A04063B0020863B0020863B0020863B002088C
S3150802A05063B0020863B0020863B0020863B002087C
S3150802A06043A40208DBA50208F5AA020837AC0208CF
S3150802A07039B0020863B0020863B0020863B0020886
S3150802A08063B0020863B0020863B0020863B002084C
S3150802A09063B0020863B0020863B0020863B002083C
S3150802A0A029AE02082BAF020863B0020863B00208A1
S3150802A0B063B0020863B0020863B0020863B002081C
S3150802A0C063B0020863B0020863B0020863B002080C
S3150802A0D063B0020801A2020863B0020863B002086C
S3150802A0E063B0020863B0020863B0020863B00208EC
S3150802A0F063B0020863B0020863B0020863B00208DC
S3150802A10063B0020863B0020863B0020863B00208CB
S3150802A11063B0020863B0020863B0020863B00208BB
S3150802A12063B0020863B0020863B0020863B00208AB
S3150802A13063B0020863B0020863B0020863B002089B
S3150802A14063B0020863B0020863B0020863B002088B
S3150802A15063B0020863B0020863B0020863B002087B
S3150802A16063B0020849A7020815A90208CB4B9B78D7
S3150802A1701946CB4825F009F9C84BDB781946C84871
S3150802A18025F01FF9C749C64825F08DF8C54825F0B8
S3150802A190D8F80446C34825F0E0F80346194620468F
S3150802A1A0FFF74CFE00F05EBFBF4B01221A70BD4995
S3150802A1B0BD4825F09BF8BB4825F0C3F80446B948C4
S3150802A1C025F0CBF8034619462046FFF737FE00F07E
S3150802A1D049BFB64813F0FAFBF8680EF008FCB14816
S3150802A1E025F09DF8AF4825F0ACF80446AD4825F0B1
S3150802A1F0B4F8034619462046FFF720FE00F032BFA0
S3150802A200AB4813F0E3FB00F02DBF26F023F9034613
S3150802A210184626F05BF90346A24918460DF058F887
S3150802A220A04825F08EF804469E4825F096F803467F
S3150802A23019462046FFF702FE00F014BF9D4813F0A8
S3150802A240C5FB7B6801339C49184620F0C9FD20F0FE
S3150802A250B3FC0346184620F0DCFC03461C46964827
S3150802A26020F010FD03469C4211D1934820F00AFDC6
S3150802A27003461C4620F0A0FC0346184620F0C9FCFB
S3150802A28003461A4621468D4813F0A0FB31E08A4858
S3150802A29020F0F8FC884820F0F5FC03460F2B1ED860
S3150802A2A0854820F0EFFC03461C46834820F005FD4E
S3150802A2B003461A462146824813F088FB20F07CFCA6
S3150802A2C004467D4820F0DEFC03461946204620F067
S3150802A2D0ACFCFB7819467868FCF72CF809E0764856
S3150802A2E020F0D0FC034619460F230022754813F0C6
S3150802A2F06DFB6C49704820F09AFD6A4825F021F8F2
S3150802A3000446684825F029F8034619462046FFF709
S3150802A31095FD00F0A7BE6C4813F058FB7B68013325
S3150802A3206A49184620F0B7FD20F046FC034618464F
S3150802A33020F06FFC03461C46644820F0D9FC03460D
S3150802A3409C4211D1614820F0D3FC03461C4620F0FA
S3150802A35033FC0346184620F05CFC03461A4621469F
S3150802A3605B4813F033FB2BE0584820F0C1FC5748F2
S3150802A37020F0BEFC03460F2B18D8544820F0B8FC30
S3150802A38003461946534813F021FB20F015FC0446F0
S3150802A3904E4820F0ADFC03461946204620F045FCFF
S3150802A3A0FB7819467868FBF7C5FF09E0474820F0AD
S3150802A3B09FFC034619460F230022474813F006FB63
S3150802A3C03849424820F083FD364824F0BAFF04464D
S3150802A3D0344824F0C2FF034619462046FFF72EFDED
S3150802A3E000F040BE3D4813F0F1FA00F03BBE3C488F
S3150802A3F013F0ECFA012200213A4828F0C3FF20F0B4
S3150802A400DBFB0346184620F004FC0346194635488A
S3150802A41020F095FC2349334820F06FFD214824F0AB
S3150802A42090FF04461F4824F098FF03461946204623
S3150802A430FFF704FD00F016BE2B4813F0C7FA00F02A
S3150802A44011BE2A4813F0C2FA7B6801332849184616
S3150802A4500DF01CF920F0B0FB0346184620F0D9FB94
S3150802A46003461C4622480CF007FB03469C4245D18C
S3150802A470022120480CF093FB1D480CF0FDFA034616
S3150802A4801C4620F099FB0346184620F0C2FB0346F9
S3150802A4901A462146184813F099FA8CE0E0BF1F08BD
S3150802A4A0DC310120D4300120D8310120248205086C
S3150802A4B04082050858820508E031012074820508A1
S3150802A4C0A0820508D082050800830508E431012028
S3150802A4D0208305085083050878830508AC83050898
S3150802A4E0C8830508E8310120E483050804840508C1
S3150802A4F010320120183201202484050885480CF000
S3150802A500BBFA84480CF0B8FA03460F2B45D810F06C
S3150802A51045FB0346184610F009FC0346002B34D1C6
S3150802A52001217D480CF03BFB7A480CF0A5FA03465C
S3150802A5301D4678480CF0BBFA03461E4675480CF0D1
S3150802A540D1FA0346984673480CF0E7FA03461C46C6
S3150802A55070480CF0FDFA03460193009443463246CE
S3150802A56029466E4813F032FA20F026FB044669485B
S3150802A5700CF082FA03461946204620F056FBFB7871
S3150802A58019467868FBF7D6FE15E0032162480CF0F7
S3150802A59006FB634813F01AFA0DE002215E480CF036
S3150802A5A0FEFA5C480CF068FA034619460F230022A5
S3150802A5B05C4813F00BFA5C4957480DF0BCF85A4848
S3150802A5C024F0BFFE0446584824F0C7FE034619463F
S3150802A5D02046FFF733FC00F045BD544813F0F6F960
S3150802A5E07B680133524918460DF001F920F0E4FA66
S3150802A5F00346184620F00DFB03461C464C480CF051
S3150802A600DDFA03469C4215D102214A480CF069FB41
S3150802A61047480CF0D3FA03461C4620F0CDFA034607
S3150802A620184620F0F6FA03461A462146424813F01F
S3150802A630CDF95CE03E480CF0C1FA3D480CF0BEFA92
S3150802A64003460F2B45D810F0A9FA0346184610F010
S3150802A6506DFB0346002B34D1012136480CF041FB31
S3150802A66033480CF0ABFA03461D4631480CF0C1FAE2
S3150802A67003461E462E480CF0D7FA034698462C483F
S3150802A6800CF0EDFA03461C4629480CF003FB034678
S3150802A69001930094434632462946284813F096F910
S3150802A6A020F08AFA044622480CF088FA034619462C
S3150802A6B0204620F0BAFAFB7819467868FBF73AFE84
S3150802A6C015E003211B480CF00CFB1D4813F07EF91C
S3150802A6D00DE0022117480CF004FB15480CF06EFA3F
S3150802A6E0034619460F230022164813F06FF90E493E
S3150802A6F010480DF0D1F80C4824F023FE04460A4807
S3150802A70024F02BFE034619462046FFF797FB00F076
S3150802A710A9BC00BF10320120183201205484050852
S3150802A720A0840508C8840508D430012000850508D8
S3150802A7301C3201202432012020850508508505088F
S3150802A74098850508C0850508E54813F03FF901F024
S3150802A75061F90346184601F082F90346184601F0E4
S3150802A760F3F903461946DF480BF09DFE01F052F94C
S3150802A7700346184601F073F90346184601F000FA33
S3150802A78003461946D7480BF0A9FE01F043F90346DA
S3150802A790184601F064F90346184601F00CFA034616
S3150802A7A01946D0480BF0B5FE01F034F903461846AF
S3150802A7B001F055F90346184601F018FA03461946F8
S3150802A7C0C8480BF0C1FE01F025F90346184601F008
S3150802A7D046F90346184601F090FA03461946C14857
S3150802A7E00BF0CDFE01F016F90346184601F037F9CB
S3150802A7F00346184601F09CFA03461946B9480BF077
S3150802A800D9FE01F007F90346184601F028F903466E
S3150802A810184601F0A8FA03461946B2480BF0E5FEB7
S3150802A82001F0F8F80346184601F019F903461846E6
S3150802A83001F0B4FA03461946AA480BF0F2FE01F0F3
S3150802A840E9F80346184601F00AF90346184601F0E4
S3150802A85012FB03461946A3480BF0FEFE01F0DAF88E
S3150802A8600346184601F0FBF80346184601F01EFB9C
S3150802A870034619469B480BF00AFF01F0CBF803463C
S3150802A880184601F0ECF80346184601F0A3FA034607
S3150802A890194694480BF016FF01F0BCF80346184611
S3150802A8A001F0DDF80346184601F0AFFA03461946E9
S3150802A8B08C480BF022FF01F0ADF80346184601F06A
S3150802A8C0CEF80346184601F0BBFA034619468548F0
S3150802A8D00BF02EFF01F09EF80346184601F0BFF86A
S3150802A8E00346184601F0FDFA034619467D480BF061
S3150802A8F03AFF7D497B480CF07DFD7B4824F021FD1B
S3150802A9000446794824F029FD034619462046FFF7EE
S3150802A91095FAA7E3754813F059F801F07BF8034650
S3150802A920184601F08FF80346184601F0F5FA034671
S3150802A93019466F480BF032FF01F06CF803461846C9
S3150802A94001F080F80346184601F001FB0346194652
S3150802A95067480BF03EFF01F05DF80346184601F022
S3150802A96071F80346184601F00DFB0346194660487E
S3150802A9700BF04AFF01F04EF80346184601F062F85A
S3150802A9800346184601F019FB0346194658480BF0C8
S3150802A99056FF01F03FF80346184601F053F80346FE
S3150802A9A0184601F025FB0346194651480BF062FF8B
S3150802A9B001F030F80346184601F044F803461846F3
S3150802A9C001F031FB0346194649480BF06EFF01F0C8
S3150802A9D021F80346184601F035F80346184601F0F1
S3150802A9E0E2FB0346194642480BF07AFF01F012F8D9
S3150802A9F00346184601F026F80346184601F09DFB61
S3150802AA00034619463A480BF086FF01F003F8034657
S3150802AA10184601F017F80346184601F0A9FB034643
S3150802AA20194633480BF092FF00F0F4FF0346184626
S3150802AA3001F008F80346184601F064FB0346194676
S3150802AA402B480BF09EFF00F0E5FF0346184600F080
S3150802AA50F9FF0346184601F02BFB0346194624481C
S3150802AA600BF0AAFF00F0D6FF0346184600F0EAFFED
S3150802AA700346184601F001FB034619461C480BF02B
S3150802AA80B6FF00F0C7FF0346184600F0DBFF034691
S3150802AA90184601F0BEFB0346194615480BF0C2FFDD
S3150802AAA000F0B8FF0346184600F0CCFF03461846E6
S3150802AAB001F094FB034619460D480BF0CEFF0A49EE
S3150802AAC00B480CF01FFD084824F03BFC04460648D8
S3150802AAD024F043FC034619462046FFF7AFF9C1E2C4
S3150802AAE0F4850508EC310120D430012018860508C2
S3150802AAF000320120BC4812F069FF7B680133BB496A
S3150802AB0018460CF04BFF20F057F80346184620F07B
S3150802AB1080F803461C46B5480CF00DF903469C42DC
S3150802AB2015D10221B2480CF0B4F9B0480CF003F979
S3150802AB3003461C4620F040F80346184620F069F8FA
S3150802AB4003461A462146AB4812F040FF62E0A74880
S3150802AB500CF0F1F8A5480CF0EEF803460F2B4BD88B
S3150802AB600EF066F9034618460EF042FA0346002B23
S3150802AB703AD101219E480CF08CF99C480CF0DBF87E
S3150802AB8003461E4699480CF0F1F80346984697483C
S3150802AB900CF007F90346994694480CF01DF903464A
S3150802ABA01C4692480CF033F903461D468F480CF0B2
S3150802ABB049F903460293019500944B4642463146AB
S3150802ABC08D4812F003FF1FF0F7FF044687480CF082
S3150802ABD0B2F803461946204620F027F8FB781946AC
S3150802ABE07868FBF7A7FB15E0032181480CF051F9B9
S3150802ABF0824812F0EBFE0DE002217D480CF049F97D
S3150802AC007A480CF098F8034619460F2300227C4826
S3150802AC1012F0DCFE7B4976480CF020FF794824F0D6
S3150802AC2090FB0446774824F098FB034619462046CB
S3150802AC30FFF704F916E2744812F0C8FE7B6801337E
S3150802AC40724918460CF074FF1FF0B6FF0346184601
S3150802AC501FF0DFFF03461C466C480CF044F9034616
S3150802AC609C4215D102216A480CF09AF967480CF001
S3150802AC703AF903461C461FF09FFF034618461FF083
S3150802AC80C8FF03461A462146624812F09FFE9AE01A
S3150802AC905E480CF028F95D480CF025F903460F2B9F
S3150802ACA000F283800EF0C4F8034618460EF0A0F9A7
S3150802ACB00346002B4ED100F0ADFE0346184600F0BF
S3150802ACC0C1FE0346184601F089FA0346002B41D114
S3150802ACD000F0A0FE0346184600F0B4FE03461846E6
S3150802ACE001F06BF90346002B34D100F093FE0346BC
S3150802ACF0184600F0A7FE0346184601F079F90346FE
S3150802AD00002B27D1012142480CF04AF93F480CF0A2
S3150802AD10EAF803461C463D480CF000F903461D4670
S3150802AD203A480CF016F903462A4621463A4812F0E2
S3150802AD304DFE1FF041FF044634480CF0D4F8034692
S3150802AD40194620461FF071FFFB7819467868FBF70B
S3150802AD50F1FA29E000F05EFE0346184600F072FE9C
S3150802AD600346184601F029F90346012B0CD000F0D8
S3150802AD7051FE0346184600F065FE0346184601F0E2
S3150802AD8037F90346012B07D1042121480CF008F9AB
S3150802AD90224812F01BFE07E003211D480CF000F9B9
S3150802ADA01F4812F013FE0EE00DE0022118480CF0BF
S3150802ADB0F7F816480CF097F8034619460F230022AF
S3150802ADC0184812F003FE0F4911480CF0E4FE0D482C
S3150802ADD024F0B7FA04460B4824F0BFFA034619468C
S3150802ADE02046FFF72BF83DE13C860508283201206C
S3150802ADF0303201205C8605088C860508E48605083B
S3150802AE000C870508D4300120408705083432012012
S3150802AE10383201206087050890870508CC8705081F
S3150802AE20FC87050824880508914812F0CFFD7B683F
S3150802AE300133904918460CF020FF1FF0BDFE034669
S3150802AE4018461FF0E6FE03461C468A480CF0D2F85E
S3150802AE5003469C4211D187480CF0CCF803461C469F
S3150802AE601FF0AAFE034618461FF0D3FE03461A46EB
S3150802AE702146814812F0AAFD47E07E480CF0BAF84E
S3150802AE807C480CF0B7F803460F2B34D879480CF0F7
S3150802AE90B1F803461C4677480CF0C9F803461D4626
S3150802AEA074480CF0DFF803461E4672480CF0F5F8B3
S3150802AEB00346009333462A462146704812F086FD19
S3150802AEC01FF07AFE04466B480CF094F803461946BE
S3150802AED020461FF0AAFEB86800F0B4FD03461846DD
S3150802AEE001F07CF90346002B0FD1FB7819467868E6
S3150802AEF0FBF720FA09E05F480CF07CF8034619468E
S3150802AF000F2300225E4812F061FD5E480CF0FFFE38
S3150802AF105C4824F016FA04465A4824F01EFA0346F8
S3150802AF2019462046FEF78AFF9CE0574812F04EFD66
S3150802AF307B680133554918460CF03CFF1FF03CFE6E
S3150802AF40034618461FF065FE03461C464F480CF09A
S3150802AF50BFF803469C4211D14C480CF0B9F8034697
S3150802AF601C461FF029FE034618461FF052FE0346EA
S3150802AF701A462146464812F029FD4DE043480CF090
S3150802AF80A7F842480CF0A4F803460F2B3AD83F48D4
S3150802AF900CF09EF803461D463C480CF0B6F80346EC
S3150802AFA01E463A480CF0CCF80346984637480CF049
S3150802AFB0E2F803461C4635480CF0F8F803460193B6
S3150802AFC00094434632462946324812F0FFFC1FF0E7
S3150802AFD0F3FD04462D480CF07BF803461946204635
S3150802AFE01FF023FEB86800F02DFD0346184601F04F
S3150802AFF0F5F80346002B0FD1FB7819467868FBF75C
S3150802B00099F909E021480CF063F8034619460F231B
S3150802B0100022214812F0DAFC1A480CF020FF1948DF
S3150802B02024F08FF90446174824F097F9034619467F
S3150802B0302046FEF703FF15E0184812F0C7FC01F098
S3150802B040B7F910480CF020FF0E4824F07AF90446A6
S3150802B0500C4824F082F9034619462046FEF7EEFE0E
S3150802B06000E000BF00BF1437BD46BDE8F08300BF4D
S3150802B0705C8805083C32012080880508B4880508E2
S3150802B08000890508D43001203C890508443201208C
S3150802B0906089050894890508E4890508208A05084F
S3150802B0A080B500AF03481BF019FA02481BF0D6F820
S3150802B0B000BF80BDC432012080B500AF00F02CF974
S3150802B0C012F074FC00BF80BD80B500AF03481BF0C8
S3150802B0D005FA02481BF0C2F800BF80BD58330120AA
S3150802B0E080B500AF00F064F912F0F4FE00BF80BD2F
S3150802B0F080B500AF174B184A9A6062B600BF13F0C4
S3150802B100C7F800F02DF800F09FF900F093F800F068
S3150802B110D9F800F0F9F800F0FFF800F049F90DF057
S3150802B12009FCFEF767FE0D48FAF770F8FEF7ACFE63
S3150802B13012F03CFC12F0CEFE00F0F2FB26F08CFC7C
S3150802B140FAF79CFBFBF7D0F80AF05AFEF9F7A2FACF
S3150802B15000BFFDE700ED00E0000002084C320120C6
S3150802B16080B59CB000AF07F1200350220021184693
S3150802B17028F008F907F1080300221A605A609A6053
S3150802B180DA601A615A612A4B1B69294A43F030036D
S3150802B1901361274B1B6903F030037B607B6800BF92
S3150802B1A0234B5B6903F00803082BF9D109233B6299
S3150802B1B04FF480337B624FF08063BB630223BB6428
S3150802B1C00323FB6403233B657D237B650223BB655F
S3150802B1D00223FB6502233B6608237B660023BB66C4
S3150802B1E00023FB6607F12003184614F075FC034694
S3150802B1F0002B01D000F082FA1F23BB600323FB60F9
S3150802B20000233B6100237B610023BB610023FB61B2
S3150802B21007F108030521184615F096F80346002B90
S3150802B22001D000F06BFA00BF7037BD4680BD00BF83
S3150802B2300008024480B500AF204B214A1A601F4B12
S3150802B24000225A601D4B4FF440729A601B4B002233
S3150802B250DA601A4B00221A74184B00225A74174BDA
S3150802B26000229A74154B05225A61144B0A229A61D6
S3150802B270124B2722DA61114B0A221A620F4B052258
S3150802B2805A620E4B02229A620C4B0722DA620B4B67
S3150802B29002221A63094B01225A63084B01229A6356
S3150802B2A0064B0022DA63054813F0F0F90346002B31
S3150802B2B001D000F023FA00BF80BD00BF4C32012046
S3150802B2C000A4004080B500AF0D4B0E4A1A600C4B25
S3150802B2D005225A600A4B40F2EE22DA60084B40F227
S3150802B2E0EE229A60064B00221A61054814F05CFBAE
S3150802B2F00346002B01D000F001FA00BF80BD00BF53
S3150802B300B03201200030004080B400AF00BFBD4615
S3150802B3105DF8047B7047000080B500AF224B234AD4
S3150802B3201A60214B4FF4E1325A601F4B00229A6091
S3150802B3301D4B0022DA601C4B00221A611A4B0C22A2
S3150802B3405A61194B00229A61174B0022DA61164B91
S3150802B35000221A62144B00225A62134B00229A6286
S3150802B36011481AF02BFF0346002B01D000F0C6F94C
S3150802B37000210D481CF09BFF0346002B01D000F06C
S3150802B380BDF9002108481CF0D0FF0346002B01D066
S3150802B39000F0B4F904481CF051FF0346002B01D013
S3150802B3A000F0ACF900BF80BDC4320120003801406C
S3150802B3B080B500AF224B234A1A60214B4FF4E13283
S3150802B3C05A601F4B00229A601D4B0022DA601C4B02
S3150802B3D000221A611A4B0C225A61194B00229A61F1
S3150802B3E0174B0022DA61164B00221A62144B00220E
S3150802B3F05A62134B00229A6211481AF0DFFE03467C
S3150802B400002B01D000F07AF900210D481CF04FFFFD
S3150802B4100346002B01D000F071F9002108481CF000
S3150802B42084FF0346002B01D000F068F904481CF09B
S3150802B43005FF0346002B01D000F060F900BF80BD6E
S3150802B440583301200048004080B58EB000AF07F19E
S3150802B450240300221A605A609A60DA601A61934BD2
S3150802B460D3F88C30914A43F01003C2F88C308F4BD4
S3150802B470D3F88C3003F010033B623B6A8B4BD3F84C
S3150802B4808C308A4A43F02003C2F88C30874BD3F8B3
S3150802B4908C3003F02003FB61FB69844BD3F88C30B4
S3150802B4A0824A43F08003C2F88C30804BD3F88C3042
S3150802B4B003F08003BB61BB697C4BD3F88C307B4AB3
S3150802B4C043F00403C2F88C30784BD3F88C3003F07F
S3150802B4D004037B617B69754BD3F88C30734A43F05E
S3150802B4E00103C2F88C30714BD3F88C3003F0010398
S3150802B4F03B613B696D4BD3F88C306C4A43F00203CF
S3150802B500C2F88C30694BD3F88C3003F00203FB6027
S3150802B510FB68664BD3F88C30644A43F04003C2F8A2
S3150802B5208C30624BD3F88C3003F04003BB60BB68A7
S3150802B5305E4BD3F88C305D4A43F00803C2F88C3070
S3150802B5405A4BD3F88C3003F008037B607B680122E0
S3150802B55048F28431564814F0F5F900224FF4026194
S3150802B560534814F0EFF901224EF2D831514814F03B
S3150802B570E9F901223321504814F0E4F900220421A2
S3150802B5804D4814F0DFF9012206214C4814F0DAF985
S3150802B5900022F021494814F0D5F900220121484831
S3150802B5A014F0D0F9012240F2FF11464814F0CAF904
S3150802B5B001224FF45051424814F0C4F901224FF4C3
S3150802B5C00F41414814F0BEF9002245F203013E48F4
S3150802B5D014F0B8F948F6A4337B620123BB62002350
S3150802B5E0FB6200233B6307F124031946304813F034
S3150802B5F09BFF4EF2D8337B620123BB620023FB62B8
S3150802B60000233B6307F1240319462A4813F08CFFEB
S3150802B61037237B620123BB620023FB6200233B6361
S3150802B62007F124031946244813F07EFFF6237B62AA
S3150802B6300123BB620023FB6200233B6307F1240359
S3150802B64019461E4813F070FF43F201437B62012339
S3150802B650BB620023FB6200233B6307F124031946FE
S3150802B660174813F061FF40F2FF137B620123BB62A6
S3150802B6700023FB6200233B6307F1240319461148A2
S3150802B68013F052FF4DF603737B620123BB6200235C
S3150802B690FB6200233B6307F1240319460A4813F0A9
S3150802B6A043FF00BF3837BD4680BD00BF000C0244C9
S3150802B6B0001002420014024200080242000002423E
S3150802B6C00004024200180242000C024280B582B00F
S3150802B6D000AF78607B681B68074A934201D112F073
S3150802B6E0FDFD7B681B68044A934201D1FBF754FFB0
S3150802B6F000BF0837BD4680BD0010004080B400AFC9
S3150802B70072B600BF00BFFDE780B58EB000AF7860A5
S3150802B710396000237B6365E04D4B4E4A40217868C9
S3150802B72013F030FA0346002B03D04B4812F086F981
S3150802B73058E0F9F721FE0346002B03D0454B1B6858
S3150802B7407B6302E0434B1B687B63F9F72FFE0246D5
S3150802B7507B6B934204D168213E48F9F71DFD41E00F
S3150802B76020F0FAFC02467B6B93422FD020F002FDB2
S3150802B77002467B6B934229D020F0E0FC02467B6BA3
S3150802B780934223D020F03AFD02467B6B93421DD0AA
S3150802B79020F048FD02467B6B934217D020F050FDFD
S3150802B7A002467B6B934211D020F00CFD02467B6B5E
S3150802B7B093420BD020F014FD02467B6B934205D0D0
S3150802B7C020F026FD02467B6B93420BD1214BDB68A8
S3150802B7D01846F8F7A7FF0346DBB21A461C49786BE8
S3150802B7E026F098F94021786813F03AFB0346002BB5
S3150802B7F092D17868F9F764FD03461A46174B9A60A0
S3150802B8007868F9F727FD0346144A13607868F9F74A
S3150802B81039FD0346114A5360104B9B68002B12D020
S3150802B8200E4B1A680D4B5B6807F10C000C4927F0A2
S3150802B83015FD07F10C03184612F000F9074B9B6831
S3150802B8401846F9F785FD00BF3837BD4680BD00BFEB
S3150802B85014340120EC330120408A0508281A0120F5
S3150802B860608A050880B58AB002AF78600B467B808D
S3150802B87013463B800023BB600023FB607B683B6169
S3150802B88001237B617B88BB613B88FB6107F1080367
S3150802B8901946074813F054F801230093012302229C
S3150802B8A00221034813F0A6F800BF2037BD4680BD23
S3150802B8B04C32012080B58CB002AFF860B9607A606C
S3150802B8C04FF080433B6100237B61FB68BB61012328
S3150802B8D0FB61BB683B627B687B6207F11003194612
S3150802B8E0074813F02DF801230093012302220221AF
S3150802B8F0034813F07FF800BF2837BD4680BD00BF56
S3150802B9004C32012080B500AF044813F0A4F8002297
S3150802B9100121024813F0C2FA00BF80BD4C32012051
S3150802B92080B500AFF9F728FD0346002B09D0F9F7D1
S3150802B9303DFD03461A466FF060410220FFF7BAFF43
S3150802B94009E0F9F733FD03469BB21A464FF6FF7133
S3150802B9500220FFF787FFFFF7D5FF00BF80BD000073
S3150802B96080B58EB000AFF860B9601346FB71FB79FB
S3150802B970002B02D0FB79402B01D900233FE007F1C7
S3150802B980140324220021184627F0FCFCFB687B617D
S3150802B990F9F7F2FC0346002B03D04FF08043BB6154
S3150802B9A001E00023BB610023FB61FB799BB21846C9
S3150802B9B0F8F70EFF03463B6200237B624FF48013BF
S3150802B9C0BB624FF40013FB6200233B6300237B63D5
S3150802B9D04FF47A710C481EF007FF0346002B0AD172
S3150802B9E007F11403BA6819460848F9F753F80648DE
S3150802B9F01EF054FF02E0064812F020F8012318460A
S3150802BA003837BD4680BD00BF7CF600204C32012087
S3150802BA10848A050880B500AF084B1B78DBB2002B79
S3150802BA2008D1064B01221A704FF4B072002104485D
S3150802BA3027F0A8FC024B184680BD00BFB43501208A
S3150802BA405434012080B483B000AF78607B6803F574
S3150802BA509B7318460C37BD465DF8047B704780B465
S3150802BA6083B000AF78607B6803F5A37318460C377A
S3150802BA70BD465DF8047B704780B487B000AF786036
S3150802BA800B46FB704FF6FF73FB8200233B6123E0F4
S3150802BA903B697A6813441B781A46FB8A5340FB8231
S3150802BAA00023FB6012E0FB8A03F00103002B03D19B
S3150802BAB0FB8A5B089BB205E0FB8A5B089AB20D4BD0
S3150802BAC053409BB2FB82FB680133FB60FB68072B82
S3150802BAD0E9DD3B6901333B61FB783A699A42D7DB78
S3150802BAE0FB8ADB439BB218461C37BD465DF8047BCE
S3150802BAF0704700BF0884FFFF80B584B000AF0346D5
S3150802BB000A46FB711346BB710023FB81FB79012BA5
S3150802BB1014D1FEF72BF80023FB8109E0BB791846FE
S3150802BB2012F0F6FA64201DF017FFFB890133FB8138
S3150802BB30FB89042BF2D9FEF725F801E0FEF722F875
S3150802BB4000BF1037BD4680BD80B483B000AF7860B1
S3150802BB507B6893F9003018460C37BD465DF8047BBE
S3150802BB60704780B483B000AF78600B46FB707B6881
S3150802BB70FA781A7000BF0C37BD465DF8047B704729
S3150802BB8080B483B000AF78607B685B8818460C3750
S3150802BB90BD465DF8047B704780B483B000AF786019
S3150802BBA00B467B807B687A885A8000BF0C37BD4675
S3150802BBB05DF8047B704780B483B000AF78607B6819
S3150802BBC01B7918460C37BD465DF8047B704780B46E
S3150802BBD083B000AF78600B46FB707B68FA781A71FF
S3150802BBE000BF0C37BD465DF8047B704780B483B04E
S3150802BBF000AF78607B685B7918460C37BD465DF8FE
S3150802BC00047B704780B483B000AF78600B46FB7044
S3150802BC107B68FA785A7100BF0C37BD465DF8047B1B
S3150802BC20704780B483B000AF78607B689B7918460A
S3150802BC300C37BD465DF8047B704780B483B000AF0D
S3150802BC4078600B46FB707B68FA789A7100BF0C37EE
S3150802BC50BD465DF8047B704780B483B000AF786058
S3150802BC607B68DB7918460C37BD465DF8047B70475E
S3150802BC7080B483B000AF78600B46FB707B68FA78B5
S3150802BC80DA7100BF0C37BD465DF8047B704780B495
S3150802BC9083B000AF78607B681B7A18460C37BD46BE
S3150802BCA05DF8047B704780B483B000AF78600B46BA
S3150802BCB0FB707B68FA781A7200BF0C37BD465DF8CE
S3150802BCC0047B704780B483B000AF78607B685B7A88
S3150802BCD018460C37BD465DF8047B704780B483B0BE
S3150802BCE000AF78600B46FB707B68FA785A7200BF21
S3150802BCF00C37BD465DF8047B704780B483B000AF4D
S3150802BD0078607B685B8918460C37BD465DF8047B0C
S3150802BD10704780B483B000AF78600B467B807B683F
S3150802BD207A885A8100BF0C37BD465DF8047B704796
S3150802BD3080B483B000AF78607B689B8918460C375D
S3150802BD40BD465DF8047B704780B483B000AF786067
S3150802BD500B467B807B687A889A8100BF0C37BD4682
S3150802BD605DF8047B704780B483B000AF78607B6867
S3150802BD70DB8918460C37BD465DF8047B704780B4EC
S3150802BD8083B000AF78600B467B807B687A88DA815D
S3150802BD9000BF0C37BD465DF8047B704780B483B09C
S3150802BDA000AF78607B6893F9103018460C37BD46A9
S3150802BDB05DF8047B704780B483B000AF78600B46A9
S3150802BDC0FB707B68FA781A7400BF0C37BD465DF8BB
S3150802BDD0047B704780B483B000AF78607B685B7C75
S3150802BDE018460C37BD465DF8047B704780B483B0AD
S3150802BDF000AF78600B46FB707B68FA785A7400BF0E
S3150802BE000C37BD465DF8047B704780B483B000AF3B
S3150802BE1078607B689B7C18460C37BD465DF8047BC8
S3150802BE20704780B483B000AF78600B46FB707B68BE
S3150802BE30FA789A7400BF0C37BD465DF8047B7047E2
S3150802BE4080B483B000AF78607B68DB7C18460C3719
S3150802BE50BD465DF8047B704780B483B000AF786056
S3150802BE600B46FB707B68FA78DA7400BF0C37BD465E
S3150802BE705DF8047B704780B483B000AF78607B6856
S3150802BE801B7D18460C37BD465DF8047B704780B4A7
S3150802BE9083B000AF78600B46FB707B68FA781A7538
S3150802BEA000BF0C37BD465DF8047B704780B483B08B
S3150802BEB000AF78607B68DB8A18460C37BD465DF8AA
S3150802BEC0047B704780B483B000AF78600B467B80F2
S3150802BED07B687A88DA8200BF0C37BD465DF8047B38
S3150802BEE0704780B483B000AF78607B681B7E1846C3
S3150802BEF00C37BD465DF8047B704780B483B000AF4B
S3150802BF0078600B46FB707B68FA781A7600BF0C37A6
S3150802BF10BD465DF8047B704780B483B000AF786095
S3150802BF207B681B7818460C37BD465DF8047B70475C
S3150802BF3080B483B000AF78600B46FB707B68FA78F2
S3150802BF401A7000BF0C37BD465DF8047B704780B493
S3150802BF5083B000AF78607B685B7818460C37BD46BD
S3150802BF605DF8047B704780B483B000AF78600B46F7
S3150802BF70FB707B68FA785A7000BF0C37BD465DF8CD
S3150802BF80047B704780B483B000AF78607B689B7887
S3150802BF9018460C37BD465DF8047B704780B483B0FB
S3150802BFA000AF78600B46FB707B68FA789A7000BF20
S3150802BFB00C37BD465DF8047B704780B483B000AF8A
S3150802BFC078607B68DB7818460C37BD465DF8047BDB
S3150802BFD0704780B483B000AF78600B46FB707B680D
S3150802BFE0FA78DA7000BF0C37BD465DF8047B7047F5
S3150802BFF080B483B000AF78607B681B7918460C372B
S3150802C000BD465DF8047B704780B483B000AF7860A4
S3150802C0100B46FB707B68FA781A7100BF0C37BD466F
S3150802C0205DF8047B704780B483B000AF78607B68A4
S3150802C0305B7918460C37BD465DF8047B704780B4B9
S3150802C04083B000AF78600B46FB707B68FA785A714A
S3150802C05000BF0C37BD465DF8047B704780B483B0D9
S3150802C06000AF78600B46FB707B68FA789A7100BF5E
S3150802C0700C37BD465DF8047B704780B483B000AFC9
S3150802C08078607B68DB7918460C37BD465DF8047B19
S3150802C090704780B483B000AF78600B46FB707B684C
S3150802C0A0FA78DA7100BF0C37BD465DF8047B704733
S3150802C0B080B483B000AF78607B681B7A18460C3769
S3150802C0C0BD465DF8047B704780B483B000AF7860E4
S3150802C0D00B46FB707B68FA781A7200BF0C37BD46AE
S3150802C0E05DF8047B704780B483B000AF78600B4676
S3150802C0F0FB707B68FA785A7200BF0C37BD465DF84A
S3150802C100047B704780B483B000AF78607B689B7A03
S3150802C11018460C37BD465DF8047B704780B483B079
S3150802C12000AF78600B46FB707B68FA789A7200BF9C
S3150802C1300C37BD465DF8047B704780B483B000AF08
S3150802C14078607B68DB7A18460C37BD465DF8047B57
S3150802C150704780B483B000AF78600B46FB707B688B
S3150802C160FA78DA7200BF0C37BD465DF8047B704771
S3150802C17080B483B000AF78607B681B7B18460C37A7
S3150802C180BD465DF8047B704780B483B000AF786023
S3150802C1900B46FB707B68FA781A7300BF0C37BD46EC
S3150802C1A05DF8047B704780B483B000AF78607B6823
S3150802C1B05B7B18460C37BD465DF8047B704780B436
S3150802C1C083B000AF78600B46FB707B68FA785A73C7
S3150802C1D000BF0C37BD465DF8047B704780B483B058
S3150802C1E000AF78607B689B7B18460C37BD465DF8C6
S3150802C1F0047B704780B483B000AF78600B46FB704F
S3150802C2007B68FA789A7300BF0C37BD465DF8047BE3
S3150802C210704780B483B000AF78607B68DB7B1846D2
S3150802C2200C37BD465DF8047B704780B483B000AF17
S3150802C23078600B46FB707B68FA78DA7300BF0C37B6
S3150802C240BD465DF8047B704780B582B000AF0346F1
S3150802C250FB71104B02221A700E4B01225A700D4BBB
S3150802C26008229A700B4AFB79D3700A4BFF221A717D
S3150802C270084BFF225A71084B06221A70064B1B7886
S3150802C2801946044809F00AFC024B1B781846083777
S3150802C290BD4680BDB8350120CC35012080B582B0B7
S3150802C2A000AF0346FB71104B02221A700E4B012295
S3150802C2B05A700D4B09229A700B4AFB79D3700A4BB6
S3150802C2C0FF221A71084BFF225A71084B06221A706E
S3150802C2D0064B1B781946044809F0E0FB024B1B780B
S3150802C2E018460837BD4680BDD0350120E435012001
S3150802C2F080B500AF14220021104827F043F8104BEE
S3150802C30000221A700D4B02221A700C4B00225A7028
S3150802C3100A4B00229A70094BFF22DA70074BFF225A
S3150802C3201A71074B05221A70054B1B7819460348E2
S3150802C33009F0B4FB014B1B78184680BDE83501208D
S3150802C340FC35012080B582B000AF78601422002146
S3150802C350154827F017F8786800F000FC124B0222FD
S3150802C3601A70114B02225A700F4B01229A707B687F
S3150802C3701A780D4BDA707B685A780B4B1A710A4B8E
S3150802C380FF225A71084BFF229A71084B07221A702C
S3150802C390064B1B781946044809F080FB024B1B78AA
S3150802C3A018460837BD4680BD0036012014360120DE
S3150802C3B080B500AF14220021104826F0E3FF104B87
S3150802C3C000221A700D4B02221A700C4B00225A7068
S3150802C3D00A4B02229A70094BFF22DA70074BFF2298
S3150802C3E01A71074B05221A70054B1B781946034822
S3150802C3F009F054FB014B1B78184680BD18360120FC
S3150802C4002C36012080B582B000AF78600846114606
S3150802C4101A460346FB700B46BB7013467B70FB78C5
S3150802C420702B00F3EB80002BC0F2E681702B00F232
S3150802C430E38101A252F823F003C6020811C60208D4
S3150802C44029C6020841C6020859C6020873C6020866
S3150802C4508DC60208A7C60208C1C60208DBC60208BC
S3150802C460F5C602080FC7020829C7020843C7020809
S3150802C4705DC7020877C70208F9C70208F9C70208A2
S3150802C480F9C70208F9C70208F9C70208F9C7020874
S3150802C490F9C70208F9C70208F9C70208F9C7020864
S3150802C4A0F9C70208F9C70208F9C70208F9C7020854
S3150802C4B0F9C70208F9C70208F9C70208F9C7020844
S3150802C4C0F9C70208F9C70208F9C70208F9C7020834
S3150802C4D0F9C70208F9C70208F9C70208F9C7020824
S3150802C4E0F9C70208F9C70208F9C70208F9C7020814
S3150802C4F0F9C70208F9C70208F9C70208F9C7020804
S3150802C500F9C70208F9C70208F9C70208F9C70208F3
S3150802C510F9C70208F9C70208F9C70208F9C70208E3
S3150802C520F9C70208F9C70208F9C70208F9C70208D3
S3150802C530F9C70208F9C70208F9C70208F9C70208C3
S3150802C540F9C70208F9C70208F9C70208F9C70208B3
S3150802C550F9C70208F9C70208F9C70208F9C70208A3
S3150802C560F9C70208F9C70208F9C70208F9C7020893
S3150802C570F9C70208F9C70208F9C70208F9C7020883
S3150802C580F9C70208F9C70208F9C70208F9C7020873
S3150802C590F9C70208F9C70208F9C70208F9C7020863
S3150802C5A0F9C70208F9C70208F9C70208F9C7020853
S3150802C5B0F9C70208F9C70208F9C70208F9C7020843
S3150802C5C0F9C70208F9C70208F9C7020891C702089B
S3150802C5D0ABC70208F9C70208F9C70208F9C7020871
S3150802C5E0F9C70208F9C70208F9C70208F9C7020813
S3150802C5F0F9C70208C5C70208DFC70208FF2B03D01E
S3150802C600FAE0FFF7D5FEF8E07868FFF79BFEF4E05C
S3150802C6107B781946786800F0F1FD7B6800221A706B
S3150802C6207B6800225A70E8E07B781946786801F040
S3150802C630F3F87B6800221A707B6801225A70DCE0E4
S3150802C6407B781946786801F0F1FB7B6800221A703C
S3150802C6507B6802225A70D0E07A78BB7819467868E5
S3150802C66002F00AFD7B6803221A707B6800225A7060
S3150802C670C3E07A78BB781946786803F021F87B68B4
S3150802C68003221A707B6801225A70B6E07A78BB7860
S3150802C6901946786803F052FB7B6803221A707B6896
S3150802C6A002225A70A9E07A78BB781946786803F0AC
S3150802C6B083FE7B6806221A707B6800225A709CE009
S3150802C6C07A78BB781946786804F0B4F97B6806224A
S3150802C6D01A707B6801225A708FE07A78BB781946FD
S3150802C6E0786804F0E5FC7B6806221A707B680222E9
S3150802C6F05A7082E07A78BB781946786805F016F897
S3150802C7007B6809221A707B6800225A7075E07A786B
S3150802C710BB781946786805F019FB7B6809221A70F6
S3150802C7207B6801225A7068E07A78BB78194678687D
S3150802C73005F01CFE7B6809221A707B6802225A7071
S3150802C7405BE07A78BB781946786806F01FF97B6849
S3150802C7500C221A707B6800225A704EE07A78BB78EF
S3150802C7601946786806F03CFC7B680C221A707B68CE
S3150802C77001225A7041E07A78BB781946786806F041
S3150802C78059FF7B680C221A707B6802225A7034E0C1
S3150802C7907B783A8AB978786807F076FA7B68032252
S3150802C7A01A707B6800225A7027E07B783A8AB97831
S3150802C7B0786807F0B9FD7B6806221A707B68002242
S3150802C7C05A701AE07B783A8AB978786808F0FCF8E1
S3150802C7D07B6809221A707B6800225A700DE07B7802
S3150802C7E03A8AB978786808F009FC7B680C221A70CC
S3150802C7F07B6800225A7000E000BF012318460837FA
S3150802C800BD4680BD80B582B000AF03460A46FB71BD
S3150802C8101346BB7114220021AA4826F0B3FDAA4B7F
S3150802C82000221A70FB79013B0B2B00F2448101A20C
S3150802C83052F823F065C80208A7C80208E9C8020820
S3150802C8402BC902086DC90208AFC90208F1C9020854
S3150802C850B7CA0208B7CA0208B7CA020833CA020820
S3150802C86075CA0208974B02221A70964B01225A7011
S3150802C870BB79002B01D0062200E00722914B9A7061
S3150802C880904B0122DA708F4BFF221A718D4BFF22D1
S3150802C8905A718D4B06221A708B4B1B78194689489A
S3150802C8A009F0FCF808E1874B02221A70854B01222F
S3150802C8B05A70BB79002B01D0062200E00722814B71
S3150802C8C09A70804B0222DA707E4BFF221A717D4BD8
S3150802C8D0FF225A717C4B06221A707B4B1B7819462B
S3150802C8E0784809F0DBF8E7E0764B02221A70754BB6
S3150802C8F001225A70BB79002B01D0062200E00722DA
S3150802C900704B9A706F4B0322DA706E4BFF221A71C4
S3150802C9106C4BFF225A716C4B06221A706A4B1B78B3
S3150802C9201946684809F0BAF8C6E0664B02221A7038
S3150802C930644B01225A70BB79002B01D0062200E013
S3150802C9400722604B9A705F4B0422DA705D4BFF2216
S3150802C9501A715C4BFF225A715B4B06221A705A4BAC
S3150802C9601B781946574809F099F8A5E0554B022253
S3150802C9701A70544B01225A70BB79002B01D0062239
S3150802C98000E007224F4B9A704E4B0622DA704D4B47
S3150802C990FF221A714B4BFF225A714B4B06221A7011
S3150802C9A0494B1B781946474809F078F884E0454B05
S3150802C9B002221A70434B01225A70BB79002B01D00E
S3150802C9C0062200E007223F4B9A703E4B0722DA7096
S3150802C9D03C4BFF221A713B4BFF225A713A4B0622F5
S3150802C9E01A70394B1B781946364809F057F863E02E
S3150802C9F0344B02221A70334B01225A70BB79002B30
S3150802CA0001D0062200E007222E4B9A702D4B0822EF
S3150802CA10DA702C4BFF221A712A4BFF225A712A4BC3
S3150802CA2006221A70284B1B781946264809F036F84A
S3150802CA3042E0244B02221A70224B01225A70BB7919
S3150802CA40002B01D0062200E007221E4B9A701D4BCE
S3150802CA500922DA701B4BFF221A711A4BFF225A71EE
S3150802CA60194B06221A70184B1B781946154809F0F5
S3150802CA7015F821E0134B02221A70124B01225A7042
S3150802CA80BB79002B01D0062200E007220D4B9A70D3
S3150802CA900C4B0A22DA700B4BFF221A71094BFF2242
S3150802CAA05A71094B06221A70074B1B781946054814
S3150802CAB008F0F4FF00E000BF024B1B78184608375F
S3150802CAC0BD4680BD303601204436012080B582B08D
S3150802CAD000AF78600B46FB702DE01C4B00221A80D3
S3150802CAE00CE0FB78184611F013FB01201CF034FF0A
S3150802CAF0164B1B8801339AB2144B1A80134B1A88A9
S3150802CB00134B1B889A42ECD3124B1B885A1C91B2C0
S3150802CB10104A1180104A1288934202D2FFF7E8FBA4
S3150802CB2009E00C4B00221A80FB7819460120FEF711
S3150802CB30E3FF002306E07868FFF782F90346002B35
S3150802CB40CBD0012318460837BD4680BD463601209C
S3150802CB50AC10002048360120AE10002080B582B005
S3150802CB6000AF7860142200218B4826F00BFC8B4B11
S3150802CB7000221A7006E1894B1B781A467B68134411
S3150802CB8093F89C30002B14BF01230023DBB21BB29F
S3150802CB90824A127811467A680A4492F8AD20002A27
S3150802CBA001D0022200E0002213431BB27B4A12780C
S3150802CBB011467A680A4492F8BE20002A01D0042255
S3150802CBC000E0002213431BB2744A127811467A68AF
S3150802CBD00A4492F8CF20002A01D0082200E0002257
S3150802CBE013431BB26D4A127811467A680A4492F8C0
S3150802CBF0E020002A01D0102200E0002213431BB2D3
S3150802CC00664A127811467A680A4492F8F120002A8E
S3150802CC1001D0202200E0002213431BB25F4A127899
S3150802CC2011467A680A4492F80221002A01D0402263
S3150802CC3000E0002213431BB2584A127811467A685A
S3150802CC400A4492F81321002A01D0802200E0002229
S3150802CC5013431BB2514A127811467A680A4492F86B
S3150802CC602421002A02D04FF4807200E000221343E6
S3150802CC701BB29AB24A4B1A80474B02221A70464B8B
S3150802CC800D225A70444B04229A707B681A78424BDA
S3150802CC90DA707B685A78404B1A71404B1A783E4BC9
S3150802CCA05A713E4B1B787A6808335B0013449B889B
S3150802CCB0DAB2394B9A71394B1B787A6808335B00BA
S3150802CCC013449B881B0A9BB2DAB2334BDA71334B95
S3150802CCD01B787A6818335B001344DB88DAB22E4B6A
S3150802CCE01A722E4B1B787A6818335B001344DB885A
S3150802CCF01B0A9BB2DAB2284B5A72284B1B781A4681
S3150802CD007B68134493F85820234B9A72234B1B785B
S3150802CD101A467B68134493F869201F4BDA721F4B35
S3150802CD201B781A467B68134493F87A201A4B1A73AF
S3150802CD301A4B1B781A467B68134493F88B20164BBA
S3150802CD405A73174B1B88DAB2134B9A73144B1B8808
S3150802CD501B0A9BB2DAB2104BDA730F4BFF221A7414
S3150802CD600D4BFF225A740F4B12221A700D4B1B7869
S3150802CD701946094808F092FE084B1B780133DAB2C5
S3150802CD80064B1A70054B1B78102B7FF6F4AE00BFC4
S3150802CD9000BF0837BD4680BD4C36012060360120EB
S3150802CDA062360120643601202DE9F04788B006AFC5
S3150802CDB078607868FEF7C8FE03461A465A4B93F916
S3150802CDC000309A423FD17868FEF7E8FF03461A46D2
S3150802CDD0564B93F900309A4235D17868FEF78DFFA3
S3150802CDE003461A46524B1B889A422CD1514B1B7842
S3150802CDF01C467868FEF79CFF03469C4223D1786856
S3150802CE00FEF7D9FE03461A464B4B1B789A421AD1AD
S3150802CE107868FEF7EBFE03461A46484B1B789A4299
S3150802CE2011D17868FFF70CF803461A46444B1B786B
S3150802CE309A4208D17868FFF754F803461A46414BD6
S3150802CE401B789A426AD07868FEF77EFE03469846B1
S3150802CE507868FEF7A3FF034699467868FEF74DFF02
S3150802CE6003469A467868FEF763FF03461C467868C7
S3150802CE70FEF7A1FE03461D467868FEF7B7FE03468F
S3150802CE801E467868FEF7DCFF03463B607868FFF7C4
S3150802CE9028F8034604933B68039302960195009487
S3150802CEA053464A464146284810F090FD7868FEF7F0
S3150802CEB04BFE03461A461C4B1A707868FEF76EFF3D
S3150802CEC003461A46194B1A707868FEF716FF034688
S3150802CED01A46174B1A807868FEF72AFF0346DAB213
S3150802CEE0144B1A707868FEF766FE03461A46124B0A
S3150802CEF01A707868FEF77AFE03461A460F4B1A70BE
S3150802CF007868FEF79DFF03461A460D4B1A70786835
S3150802CF10FEF7E7FF03461A460A4B1A7000BF0837A0
S3150802CF20BD46BDE8F08700BF65360120663601209A
S3150802CF30683601206A3601206B3601206C360120DC
S3150802CF406D3601206E360120A48A05082DE9F047C0
S3150802CF508AB006AFF860F868FEF7DEFF03461A469F
S3150802CF60644B1B789A4247D1F868FEF7F0FF0346EE
S3150802CF701A46614B1B789A423ED1F868FFF71DF8AC
S3150802CF8003461A465D4B1B789A4235D1F868FFF775
S3150802CF902FF803461A465A4B1B789A422CD1F86840
S3150802CFA0FFF737F903461A46564B1B789A4223D19E
S3150802CFB0F868FFF77DF803461A46534B1B789A42E0
S3150802CFC01AD1F868FFF79EF803461A464F4B1B78A4
S3150802CFD09A4211D1F868FFF7B0F803461A464C4B45
S3150802CFE01B789A4208D1F868FFF7C2F803461A4630
S3150802CFF0484B1B789A4278D0F868FEF78DFF0346AD
S3150802D0009846F868FEF7A3FF03469946F868FEF7BE
S3150802D010D4FF03469A46F868FEF7EAFF03461C461B
S3150802D020F868FFF7F6F803461D46F868FFF740F872
S3150802D03003461E46F868FFF765F80346BB60F868BC
S3150802D040FFF77BF803467B60F868FFF791F803461B
S3150802D05005937A680492BB68039302960195009435
S3150802D06053464A4641462C4810F0B0FCF868FEF78B
S3150802D07053FF03461A461F4B1A70F868FEF767FFF6
S3150802D08003461A461C4B1A70F868FEF796FF0346C3
S3150802D0901A461A4B1A70F868FEF7AAFF03461A468A
S3150802D0A0174B1A70F868FFF7B4F803461A46154B79
S3150802D0B01A70F868FEF7FCFF03461A46124B1A70F6
S3150802D0C0F868FFF71FF803461A46104B1A70F868F5
S3150802D0D0FFF733F803461A460D4B1A70F868FFF73E
S3150802D0E047F803461A460B4B1A7000BF1037BD465F
S3150802D0F0BDE8F0876F3601207036012071360120AF
S3150802D10072360120733601207436012075360120E5
S3150802D1107636012077360120088B050880B582B05D
S3150802D12000AF03463960FB71FB79013B072B43D8F5
S3150802D13001A252F823F000BF59D1020865D10208AC
S3150802D14071D102087DD1020889D1020895D1020857
S3150802D150A1D10208ADD10208386820F048F8F0EEED
S3150802D160407A2BE0386820F060F8F0EE407A25E045
S3150802D170386820F078F8F0EE407A1FE0386820F038
S3150802D18090F8F0EE407A19E0386820F0A8F8F0EE48
S3150802D190407A13E0386820F0C0F8F0EE407A0DE0E5
S3150802D1A0386820F0D8F8F0EE407A07E0386820F0C0
S3150802D1B0F0F8F0EE407A01E0DFED037AB0EE670AA6
S3150802D1C00837BD4680BD00BF0000000080B483B0AA
S3150802D1D000AF0346FB71FB79022B01D1012306E05E
S3150802D1E0FB79032B01D1002301E04FF0FF331846E8
S3150802D1F00C37BD465DF8047B7047000080B5ADF577
S3150802D2000C7D00AF07F50C73A3F50B7318600A467D
S3150802D21007F50C73A3F22D231A7007F50C73A3F501
S3150802D2200B734FF49B720021186826F0ABF807F5CA
S3150802D2300C73A3F22D231B781846FFF7C7FF034684
S3150802D240002BC0F2E38207F50C73A3F22D231B7899
S3150802D2501846FFF7BBFF0346DAB2B54B1A7007F555
S3150802D2600C73A3F5097318464FF408731A4600217E
S3150802D27026F088F807F50C73A3F5097340F6B83259
S3150802D2805A8007F50C73A3F5097332221A81A84B43
S3150802D2901B781A4607F50C73A3F50973DA8207F5A4
S3150802D2A00C73A3F5097301221A8407F50C73A3F507
S3150802D2B009734FF4FA625A8407F50C73A3F50973D6
S3150802D2C032221A859A4B1B781A4607F50C73A3F570
S3150802D2D00973DA8607F50C73A3F5097301225A87CF
S3150802D2E007F50C73A3F509730222A3F8402007F584
S3150802D2F00C73A3F509734FF47A72A3F842208C4B88
S3150802D3001B781A4607F50C73A3F50973A3F856207A
S3150802D31007F50C73A3F509730122A3F85E2007F536
S3150802D3200C73A3F509730322A3F8602007F50C739F
S3150802D330A3F5097341F28832A3F8622007F50C7344
S3150802D340A3F509736422A3F86A20794B1B781A4657
S3150802D35007F50C73A3F50973A3F8762007F50C7382
S3150802D360A3F509730122A3F87E2007F50C73A3F52A
S3150802D37009730422A3F8802007F50C73A3F5097331
S3150802D3804FF47A62A3F8822007F50C73A3F50973A2
S3150802D3904B22A3F88A20664B1B781A4607F50C73AC
S3150802D3A0A3F50973A3F8962007F50C73A3F5097379
S3150802D3B00122A3F89A2007F50C73A3F50973012233
S3150802D3C0A3F89E2007F50C73A3F509730522A3F8A3
S3150802D3D0A02007F50C73A3F5097340F2DC52A3F8F3
S3150802D3E0A22007F50C73A3F509733222A3F8A82025
S3150802D3F007F50C73A3F509734B22A3F8AA204C4B25
S3150802D4001B781A4607F50C73A3F50973A3F8B62019
S3150802D41007F50C73A3F509730122A3F8BE2007F5D5
S3150802D4200C73A3F509730622A3F8C02007F50C733B
S3150802D430A3F509734FF47A62A3F8C22007F50C73B1
S3150802D440A3F509733222A3F8C820394B1B781A466A
S3150802D45007F50C73A3F50973A3F8D62007F50C7321
S3150802D460A3F509730722A3F8E02007F50C73A3F5C1
S3150802D470097340F6B832A3F8E22007F50C73A3F550
S3150802D48009733222A3F8E820294B1B781A4607F5B6
S3150802D4900C73A3F50973A3F8F62007F50C73A3F525
S3150802D4A009730122A3F8FA2007F50C73A3F5097389
S3150802D4B00822A3F8002107F50C73A3F509730922BC
S3150802D4C0A3F8202107F50C73A3F509730A22A3F81A
S3150802D4D0402107F50C73A3F509730B22A3F8602103
S3150802D4E007F50C73A3F509730C22A3F8802107F537
S3150802D4F00C73A3F509730D22A3F8A02107F50C7383
S3150802D500A3F509730E22A3F8C02107F50C73A3F538
S3150802D51009730F22A3F8E02107F50C73A3F5097323
S3150802D5206322A3F800220023C7F82C3269E100BF60
S3150802D5307836012007F50C73A3F50972D7F82C3251
S3150802D5405B0113441B88D9B207F50C73A3F50B7359
S3150802D5501A68D7F82C32134402330A461A7007F5AA
S3150802D5600C73A3F50972D7F82C325B011344023304
S3150802D570198807F50C73A3F50B731A68D7F82C32BA
S3150802D58008335B0013440A469A8007F50C73A3F521
S3150802D5900972D7F82C325B0113440433198807F54C
S3150802D5A00C73A3F50B731A68D7F82C3218335B0081
S3150802D5B013440A46DA8007F50C73A3F50972D7F8FD
S3150802D5C02C325B01134406331B88D9B207F50C7358
S3150802D5D0A3F50B731A68D7F82C32134458330A4644
S3150802D5E01A7007F50C73A3F50972D7F82C325B018A
S3150802D5F0134408331B88D9B207F50C73A3F50B73CA
S3150802D6001A68D7F82C32134469330A461A7007F592
S3150802D6100C73A3F50972D7F82C325B0113440A334B
S3150802D6201B88D9B207F50C73A3F50B731A68D7F8DA
S3150802D6302C3213447A330A461A7007F50C73A3F58B
S3150802D6400972D7F82C325B0113440C331B88D9B202
S3150802D65007F50C73A3F50B731A68D7F82C32134423
S3150802D6608B330A461A7007F50C73A3F50972D7F8B5
S3150802D6702C325B0113440E331B88D9B207F50C739F
S3150802D680A3F50B731A68D7F82C3213449C330A464F
S3150802D6901A7007F50C73A3F50972D7F82C325B01D9
S3150802D6A0134410331B88D9B207F50C73A3F50B7311
S3150802D6B01A68D7F82C321344AD330A461A7007F59E
S3150802D6C00C73A3F50972D7F82C325B011344123393
S3150802D6D01B88D9B207F50C73A3F50B731A68D7F82A
S3150802D6E02C321344BE330A461A7007F50C73A3F597
S3150802D6F00972D7F82C325B01134414331B88D9B24A
S3150802D70007F50C73A3F50B731A68D7F82C32134472
S3150802D710CF330A461A7007F50C73A3F50972D7F8C0
S3150802D7202C325B01134416331B88D9B207F50C73E6
S3150802D730A3F50B731A68D7F82C321344E0330A465A
S3150802D7401A7007F50C73A3F50972D7F82C325B0128
S3150802D750134418331B88D9B207F50C73A3F50B7358
S3150802D7601A68D7F82C321344F1330A461A7007F5A9
S3150802D7700C73A3F50972D7F82C325B0113441A33DA
S3150802D7801B88D9B207F50C73A3F50B731A68D7F879
S3150802D7902C32134403F581730A461A7007F50C7383
S3150802D7A0A3F50972D7F82C325B0113441C331B8884
S3150802D7B0D9B207F50C73A3F50B731A68D7F82C328E
S3150802D7C0134403F213130A461A7007F50C73A3F5EA
S3150802D7D00972D7F82C325B0113441E331B88D9B25F
S3150802D7E007F50C73A3F50B731A68D7F82C32134492
S3150802D7F003F592730A461A70D7F82C320133C7F822
S3150802D8002C32D7F82C32102B7FF794AE00BF07F5CF
S3150802D8100C77BD4680BD00BF80B5ADF50C7D00AF67
S3150802D82007F50C73A3F50B7318600A4607F50C7314
S3150802D830A3F22D231A7007F50C73A3F50B734FF495
S3150802D8409B720021186825F09DFD07F50C73A3F25B
S3150802D8502D231B781846FFF7B9FC0346002BC0F2A6
S3150802D860DF8207F50C73A3F22D231B781846FFF700
S3150802D870ADFC0346DAB2B34B1A7007F50C73A3F57F
S3150802D880097318464FF408731A46002125F07AFDE3
S3150802D89007F50C73A3F509734FF47A625A8007F5F4
S3150802D8A00C73A3F5097350225A81A64B1B781A46A4
S3150802D8B007F50C73A3F50973DA8207F50C73A3F55A
S3150802D8C009730122DA8307F50C73A3F5097301229A
S3150802D8D01A8407F50C73A3F5097340F6B8325A840D
S3150802D8E007F50C73A3F5097364225A85954B1B78C1
S3150802D8F01A4607F50C73A3F50973DA8607F50C734E
S3150802D900A3F5097301225A8707F50C73A3F5097360
S3150802D9100122DA8707F50C73A3F509730222A3F825
S3150802D920402007F50C73A3F5097340F6B832A3F83D
S3150802D930422007F50C73A3F509733222A3F848208F
S3150802D940804B1B781A4607F50C73A3F50973A3F8DF
S3150802D950562007F50C73A3F509730322A3F8602072
S3150802D96007F50C73A3F509734FF4FA62A3F862205C
S3150802D97007F50C73A3F509733222A3F86820714BD5
S3150802D9801B781A4607F50C73A3F50973A3F87620D4
S3150802D99007F50C73A3F509730122A3F87A2007F594
S3150802D9A00C73A3F509730422A3F8802007F50C73F8
S3150802D9B0A3F509733222A3F8842007F50C73A3F59D
S3150802D9C009733C22A3F88A205E4B1B781A4607F590
S3150802D9D00C73A3F50973A3F8962007F50C73A3F540
S3150802D9E009730122A3F89E2007F50C73A3F50973A0
S3150802D9F00522A3F8A02007F50C73A3F5097340F6D0
S3150802DA00B832A3F8A22007F50C73A3F509736422AA
S3150802DA10A3F8AA2007F50C73A3F509730122A3F844
S3150802DA20B420484B1B781A4607F50C73A3F50973FD
S3150802DA30A3F8B62007F50C73A3F509730622A3F813
S3150802DA40C02007F50C73A3F5097340F6B832A3F89C
S3150802DA50C22007F50C73A3F509736422A3F8CA203A
S3150802DA6007F50C73A3F509730122A3F8D220354BE7
S3150802DA701B781A4607F50C73A3F50973A3F8D62083
S3150802DA8007F50C73A3F509730722A3F8E02007F537
S3150802DA900C73A3F509734FF47A62A3F8E22007F52B
S3150802DAA00C73A3F509733222A3F8E820254B1B78D9
S3150802DAB01A4607F50C73A3F50973A3F8F62007F5BA
S3150802DAC00C73A3F509730822A3F8002107F50C7352
S3150802DAD0A3F509730922A3F8202107F50C73A3F508
S3150802DAE009730A22A3F8402107F50C73A3F50973F3
S3150802DAF00B22A3F8602107F50C73A3F509730C2210
S3150802DB00A3F8802107F50C73A3F509730D22A3F870
S3150802DB10A02107F50C73A3F509730E22A3F8C021F9
S3150802DB2007F50C73A3F509730F22A3F8E02107F58D
S3150802DB300C73A3F509736322A3F800220023C7F81E
S3150802DB402C3268E17936012007F50C73A3F50972C0
S3150802DB50D7F82C325B0113441B88D9B207F50C732C
S3150802DB60A3F50B731A68D7F82C32134402330A4604
S3150802DB701A7007F50C73A3F50972D7F82C325B01F4
S3150802DB8013440233198807F50C73A3F50B731A6845
S3150802DB90D7F82C3208335B0013440A469A8007F5F5
S3150802DBA00C73A3F50972D7F82C325B0113440433BC
S3150802DBB0198807F50C73A3F50B731A68D7F82C3274
S3150802DBC018335B0013440A46DA8007F50C73A3F58B
S3150802DBD00972D7F82C325B01134406331B88D9B273
S3150802DBE007F50C73A3F50B731A68D7F82C3213448E
S3150802DBF058330A461A7007F50C73A3F50972D7F853
S3150802DC002C325B01134408331B88D9B207F50C730F
S3150802DC10A3F50B731A68D7F82C32134469330A46EC
S3150802DC201A7007F50C73A3F50972D7F82C325B0143
S3150802DC3013440A331B88D9B207F50C73A3F50B7381
S3150802DC401A68D7F82C3213447A330A461A7007F53B
S3150802DC500C73A3F50972D7F82C325B0113440C3303
S3150802DC601B88D9B207F50C73A3F50B731A68D7F894
S3150802DC702C3213448B330A461A7007F50C73A3F534
S3150802DC800972D7F82C325B0113440E331B88D9B2BA
S3150802DC9007F50C73A3F50B731A68D7F82C321344DD
S3150802DCA09C330A461A7007F50C73A3F50972D7F85E
S3150802DCB02C325B01134410331B88D9B207F50C7357
S3150802DCC0A3F50B731A68D7F82C321344AD330A46F8
S3150802DCD01A7007F50C73A3F50972D7F82C325B0193
S3150802DCE0134412331B88D9B207F50C73A3F50B73C9
S3150802DCF01A68D7F82C321344BE330A461A7007F547
S3150802DD000C73A3F50972D7F82C325B01134414334A
S3150802DD101B88D9B207F50C73A3F50B731A68D7F8E3
S3150802DD202C321344CF330A461A7007F50C73A3F53F
S3150802DD300972D7F82C325B01134416331B88D9B201
S3150802DD4007F50C73A3F50B731A68D7F82C3213442C
S3150802DD50E0330A461A7007F50C73A3F50972D7F869
S3150802DD602C325B01134418331B88D9B207F50C739E
S3150802DD70A3F50B731A68D7F82C321344F1330A4603
S3150802DD801A7007F50C73A3F50972D7F82C325B01E2
S3150802DD9013441A331B88D9B207F50C73A3F50B7310
S3150802DDA01A68D7F82C32134403F581730A461A7097
S3150802DDB007F50C73A3F50972D7F82C325B011344E5
S3150802DDC01C331B88D9B207F50C73A3F50B731A68B3
S3150802DDD0D7F82C32134403F213130A461A7007F5BE
S3150802DDE00C73A3F50972D7F82C325B0113441E3360
S3150802DDF01B88D9B207F50C73A3F50B731A68D7F803
S3150802DE002C32134403F592730A461A70D7F82C3249
S3150802DE100133C7F82C32D7F82C32102B7FF794AE81
S3150802DE2000BF07F50C77BD4680BD00BF80B5ADF5CE
S3150802DE300C7D00AF07F50C73A3F50B7318600A4641
S3150802DE4007F50C73A3F22D231A7007F50C73A3F5C5
S3150802DE500B734FF49B720021186825F093FA07F5A5
S3150802DE600C73A3F22D231B781846FFF7AFF9034666
S3150802DE70002BC1F2FC8007F50C73A3F22D231B7845
S3150802DE801846FFF7A3F90346DAB2EA4B1A7007F502
S3150802DE900C73A3F5097300221A8007F50C73A3F510
S3150802DEA0097341F288325A8007F50C73A3F5097390
S3150802DEB000229A8007F50C73A3F509730022DA800B
S3150802DEC007F50C73A3F5097300221A8107F50C737B
S3150802DED0A3F5097364225A8107F50C73A3F509732E
S3150802DEE000229A8107F50C73A3F509730022DA81D9
S3150802DEF007F50C73A3F5097300221A8207F50C734A
S3150802DF00A3F5097300225A8207F50C73A3F5097360
S3150802DF1000229A82C74B1B781A4607F50C73A3F59B
S3150802DF200973DA8207F50C73A3F5097300221A83BB
S3150802DF3007F50C73A3F5097300225A8307F50C73C8
S3150802DF40A3F5097300229A8307F50C73A3F50973DF
S3150802DF500122DA8307F50C73A3F5097301221A84E1
S3150802DF6007F50C73A3F5097300225A8407F50C7397
S3150802DF70A3F50973FA229A8407F50C73A3F50973B4
S3150802DF804B22DA8407F50C73A3F5097300221A8566
S3150802DF9007F50C73A3F5097364225A8507F50C7302
S3150802DFA0A3F5097300229A8507F50C73A3F509737D
S3150802DFB00022DA8507F50C73A3F5097300221A867F
S3150802DFC007F50C73A3F5097300225A8607F50C7335
S3150802DFD0A3F5097300229A86964B1B781A4607F50B
S3150802DFE00C73A3F50973DA8607F50C73A3F509739F
S3150802DFF000221A8707F50C73A3F5097300225A87BC
S3150802E00007F50C73A3F5097301229A8707F50C73B2
S3150802E010A3F509730122DA8707F50C73A3F50973C9
S3150802E0200222A3F8402007F50C73A3F5097347F2F9
S3150802E0303052A3F8422007F50C73A3F509730022A0
S3150802E040A3F8442007F50C73A3F509734B22A3F82A
S3150802E050462007F50C73A3F509730022A3F8482096
S3150802E06007F50C73A3F509736422A3F84A2007F58A
S3150802E0700C73A3F509730022A3F84C2007F50C7359
S3150802E080A3F509730022A3F84E2007F50C73A3F52E
S3150802E09009730022A3F8502007F50C73A3F5097338
S3150802E0A00022A3F8522007F50C73A3F5097301227F
S3150802E0B0A3F854205F4B1B781A4607F50C73A3F591
S3150802E0C00973A3F8562007F50C73A3F50973002202
S3150802E0D0A3F8582007F50C73A3F509730022A3F8D1
S3150802E0E05A2007F50C73A3F509730122A3F85C20DD
S3150802E0F007F50C73A3F509730022A3F85E2007F54A
S3150802E1000C73A3F509730322A3F8602007F50C73B1
S3150802E110A3F5097347F23052A3F8622007F50C7388
S3150802E120A3F509730022A3F8642007F50C73A3F577
S3150802E13009734B22A3F8662007F50C73A3F5097336
S3150802E1403222A3F8682007F50C73A3F50973642233
S3150802E150A3F86A2007F50C73A3F509730022A3F83E
S3150802E1606C2007F50C73A3F509730022A3F86E2039
S3150802E17007F50C73A3F509730022A3F8702007F5B7
S3150802E1800C73A3F509730022A3F8722007F50C7322
S3150802E190A3F509730122A3F87420264B1B781A46A5
S3150802E1A007F50C73A3F50973A3F8762007F50C7324
S3150802E1B0A3F509730022A3F8782007F50C73A3F5D3
S3150802E1C009730022A3F87A2007F50C73A3F50973DD
S3150802E1D00122A3F87C2007F50C73A3F50973002224
S3150802E1E0A3F87E2007F50C73A3F509730422A3F896
S3150802E1F0802007F50C73A3F5097347F23052A3F88A
S3150802E200822007F50C73A3F509730022A3F884206C
S3150802E21007F50C73A3F509734B22A3F8862007F5B5
S3150802E2200C73A3F509730022A3F8882007F50C736B
S3150802E23002E000BF7A360120A3F509736422A3F827
S3150802E2408A2007F50C73A3F509730022A3F88C201C
S3150802E25007F50C73A3F509730022A3F88E2007F5B8
S3150802E2600C73A3F509730022A3F8902007F50C7323
S3150802E270A3F509730122A3F8922007F50C73A3F5F7
S3150802E28009730022A3F89420F84B1B781A4607F55F
S3150802E2900C73A3F50973A3F8962007F50C73A3F577
S3150802E2A009730022A3F8982007F50C73A3F50973DE
S3150802E2B00022A3F89A2007F50C73A3F50973012225
S3150802E2C0A3F89C2007F50C73A3F509730022A3F89B
S3150802E2D09E2007F50C73A3F509730522A3F8A0205F
S3150802E2E007F50C73A3F5097347F23052A3F8A22077
S3150802E2F007F50C73A3F509730022A3F8A42007F502
S3150802E3000C73A3F509734B22A3F8A62007F50C7321
S3150802E310A3F509733222A3F8A82007F50C73A3F50F
S3150802E32009736422A3F8AA2007F50C73A3F50973E7
S3150802E3300022A3F8AC2007F50C73A3F50973002293
S3150802E340A3F8AE2007F50C73A3F509730022A3F808
S3150802E350B02007F50C73A3F509730122A3F8B220BE
S3150802E36007F50C73A3F509730022A3F8B420BF4B73
S3150802E3701B781A4607F50C73A3F50973A3F8B6209A
S3150802E38007F50C73A3F509730022A3F8B82007F55D
S3150802E3900C73A3F509730022A3F8BA2007F50C73C8
S3150802E3A0A3F509730122A3F8BC2007F50C73A3F59C
S3150802E3B009730022A3F8BE2007F50C73A3F50973A7
S3150802E3C00622A3F8C02007F50C73A3F5097347F2D2
S3150802E3D03052A3F8C22007F50C73A3F5097300227D
S3150802E3E0A3F8C42007F50C73A3F509734B22A3F807
S3150802E3F0C62007F50C73A3F509730022A3F8C820F3
S3150802E40007F50C73A3F509736422A3F8CA2007F566
S3150802E4100C73A3F509730022A3F8CC2007F50C7335
S3150802E420A3F509730022A3F8CE2007F50C73A3F50A
S3150802E43009730022A3F8D02007F50C73A3F5097314
S3150802E4400022A3F8D22007F50C73A3F5097301225B
S3150802E450A3F8D420854B1B781A4607F50C73A3F547
S3150802E4600973A3F8D62007F50C73A3F509730022DE
S3150802E470A3F8D82007F50C73A3F509730022A3F8AD
S3150802E480DA2007F50C73A3F509730122A3F8DC2039
S3150802E49007F50C73A3F509730022A3F8DE2007F526
S3150802E4A00C73A3F509730722A3F8E02007F50C738A
S3150802E4B0A3F5097347F23052A3F8E22007F50C7365
S3150802E4C0A3F509730022A3F8E42007F50C73A3F554
S3150802E4D009734B22A3F8E62007F50C73A3F5097313
S3150802E4E00022A3F8E82007F50C73A3F50973642242
S3150802E4F0A3F8EA2007F50C73A3F509730022A3F81B
S3150802E500EC2007F50C73A3F509730022A3F8EE2095
S3150802E51007F50C73A3F509730022A3F8F02007F593
S3150802E5200C73A3F509730122A3F8F22007F50C73FD
S3150802E530A3F509730022A3F8F4204C4B1B781A465C
S3150802E54007F50C73A3F50973A3F8F62007F50C7300
S3150802E550A3F509730022A3F8F82007F50C73A3F5AF
S3150802E56009730022A3F8FA2007F50C73A3F50973B9
S3150802E5700122A3F8FC2007F50C73A3F50973002200
S3150802E580A3F8FE2007F50C73A3F509730822A3F86E
S3150802E590002107F50C73A3F5097342F21072A3F86A
S3150802E5A0022107F50C73A3F509730022A3F80421C7
S3150802E5B007F50C73A3F509730022A3F8062107F5DC
S3150802E5C00C73A3F509730022A3F8082107F50C7347
S3150802E5D0A3F509736422A3F80A2107F50C73A3F5B8
S3150802E5E009730022A3F80C2107F50C73A3F5097326
S3150802E5F00022A3F80E2107F50C73A3F5097300226E
S3150802E600A3F8102107F50C73A3F509730022A3F8E2
S3150802E610122107F50C73A3F509730122A3F8142135
S3150802E620124B1B781A4607F50C73A3F50973A3F860
S3150802E630162107F50C73A3F509730022A3F818210E
S3150802E64007F50C73A3F509730022A3F81A2107F537
S3150802E6500C73A3F509730022A3F81C2107F50C73A2
S3150802E660A3F509730022A3F81E2101E07A360120D8
S3150802E67007F50C73A3F509730922A3F8202107F5F8
S3150802E6800C73A3F5097342F21072A3F8222107F557
S3150802E6900C73A3F509730022A3F8242107F50C735A
S3150802E6A0A3F509730022A3F8262107F50C73A3F52F
S3150802E6B009730022A3F8282107F50C73A3F5097339
S3150802E6C06422A3F82A2107F50C73A3F5097300221D
S3150802E6D0A3F82C2107F50C73A3F509730022A3F8F6
S3150802E6E02E2107F50C73A3F509730022A3F830212E
S3150802E6F007F50C73A3F509730122A3F8322107F56E
S3150802E7000C73A3F509730022A3F83421F94B1B787D
S3150802E7101A4607F50C73A3F50973A3F8362107F50C
S3150802E7200C73A3F509730022A3F8382107F50C73B5
S3150802E730A3F509730022A3F83A2107F50C73A3F58A
S3150802E74009730022A3F83C2107F50C73A3F5097394
S3150802E7500022A3F83E2107F50C73A3F509730A22D2
S3150802E760A3F8402107F50C73A3F509730022A3F851
S3150802E770422107F50C73A3F509734FF4C872A3F87F
S3150802E780442107F50C73A3F509730022A3F8462161
S3150802E79007F50C73A3F509730022A3F8482107F5B8
S3150802E7A00C73A3F509736422A3F84A2107F50C73BF
S3150802E7B0A3F509730022A3F84C2107F50C73A3F5F8
S3150802E7C009730022A3F84E2107F50C73A3F5097302
S3150802E7D00022A3F8502107F50C73A3F5097300224A
S3150802E7E0A3F8522107F50C73A3F509730022A3F8BF
S3150802E7F05421C04B1B781A4607F50C73A3F5097307
S3150802E800A3F8562107F50C73A3F509730022A3F89A
S3150802E810582107F50C73A3F509730022A3F85A21A8
S3150802E82007F50C73A3F509730122A3F85C2107F512
S3150802E8300C73A3F509730122A3F85E2107F50C737D
S3150802E840A3F509730B22A3F8602107F50C73A3F548
S3150802E850097342F21072A3F8622107F50C73A3F545
S3150802E86009730022A3F8642107F50C73A3F509734B
S3150802E8700022A3F8662107F50C73A3F50973002293
S3150802E880A3F8682107F50C73A3F509736422A3F8A4
S3150802E8906A2107F50C73A3F509730022A3F86C2104
S3150802E8A007F50C73A3F509730022A3F86E2107F581
S3150802E8B00C73A3F509730022A3F8702107F50C73EC
S3150802E8C0A3F509730022A3F8722107F50C73A3F5C1
S3150802E8D009730122A3F87421864B1B781A4607F599
S3150802E8E00C73A3F50973A3F8762107F50C73A3F540
S3150802E8F009730022A3F8782107F50C73A3F50973A7
S3150802E9000022A3F87A2107F50C73A3F509730122ED
S3150802E910A3F87C2107F50C73A3F509730022A3F863
S3150802E9207E2107F50C73A3F509730C22A3F880213F
S3150802E93007F50C73A3F5097342F21072A3F8822144
S3150802E94007F50C73A3F509730022A3F8842107F5CA
S3150802E9500C73A3F509730022A3F8862107F50C7335
S3150802E960A3F509730022A3F8882107F50C73A3F50A
S3150802E97009736422A3F88A2107F50C73A3F50973B0
S3150802E9800022A3F88C2107F50C73A3F5097300225C
S3150802E990A3F88E2107F50C73A3F509730022A3F8D1
S3150802E9A0902107F50C73A3F509730122A3F89221A6
S3150802E9B007F50C73A3F509730022A3F894214D4BAE
S3150802E9C01B781A4607F50C73A3F50973A3F8962163
S3150802E9D007F50C73A3F509730022A3F8982107F526
S3150802E9E00C73A3F509730022A3F89A2107F50C7391
S3150802E9F0A3F509730022A3F89C2107F50C73A3F566
S3150802EA0009730022A3F89E2107F50C73A3F509736F
S3150802EA100D22A3F8A02107F50C73A3F509730022AA
S3150802EA20A3F8A22107F50C73A3F509733222A3F8FA
S3150802EA30A42107F50C73A3F509730022A3F8A621EE
S3150802EA4007F50C73A3F509730022A3F8A82107F5A5
S3150802EA500C73A3F509733222A3F8AA2107F50C73DE
S3150802EA60A3F509730022A3F8AC2107F50C73A3F5E5
S3150802EA7009730022A3F8AE2107F50C73A3F50973EF
S3150802EA800022A3F8B02107F50C73A3F50973002237
S3150802EA90A3F8B22107F50C73A3F509730022A3F8AC
S3150802EAA0B42107F50C73A3F509730022A3F8B6215E
S3150802EAB007F50C73A3F509730022A3F8B82107F525
S3150802EAC00C73A3F509730022A3F8BA2107F50C7390
S3150802EAD0A3F509730022A3F8BC2107F50C73A3F565
S3150802EAE009730122A3F8BE2107F50C73A3F509736E
S3150802EAF00E2201E07A360120A3F8C02107F50C732D
S3150802EB00A3F509730022A3F8C22107F50C73A3F52E
S3150802EB1009730022A3F8C42107F50C73A3F5097338
S3150802EB200022A3F8C62107F50C73A3F50973002280
S3150802EB30A3F8C82107F50C73A3F509730022A3F8F5
S3150802EB40CA2107F50C73A3F509730022A3F8CC2191
S3150802EB5007F50C73A3F509730022A3F8CE2107F56E
S3150802EB600C73A3F509730022A3F8D02107F50C73D9
S3150802EB70A3F509730022A3F8D22107F50C73A3F5AE
S3150802EB8009730022A3F8D42107F50C73A3F50973B8
S3150802EB900022A3F8D62107F50C73A3F50973002200
S3150802EBA0A3F8D82107F50C73A3F509730022A3F875
S3150802EBB0DA2107F50C73A3F509730022A3F8DC2101
S3150802EBC007F50C73A3F509730022A3F8DE2107F5EE
S3150802EBD00C73A3F509730F22A3F8E02107F50C734A
S3150802EBE0A3F509730022A3F8E22107F50C73A3F52E
S3150802EBF009730022A3F8E42107F50C73A3F5097338
S3150802EC000022A3F8E62107F50C73A3F5097300227F
S3150802EC10A3F8E82107F50C73A3F509730022A3F8F4
S3150802EC20EA2107F50C73A3F509730022A3F8EC2170
S3150802EC3007F50C73A3F509730022A3F8EE2107F56D
S3150802EC400C73A3F509730022A3F8F02107F50C73D8
S3150802EC50A3F509730022A3F8F22107F50C73A3F5AD
S3150802EC6009730022A3F8F42107F50C73A3F50973B7
S3150802EC700022A3F8F62107F50C73A3F509730022FF
S3150802EC80A3F8F82107F50C73A3F509730022A3F874
S3150802EC90FA2107F50C73A3F509730022A3F8FC21E0
S3150802ECA007F50C73A3F509730022A3F8FE2107F5ED
S3150802ECB00C73A3F509736322A3F8002207F50C73F4
S3150802ECC0A3F509730022A3F8022207F50C73A3F52C
S3150802ECD009730022A3F8042207F50C73A3F5097336
S3150802ECE00022A3F8062207F50C73A3F5097300227E
S3150802ECF0A3F8082207F50C73A3F509730022A3F8F3
S3150802ED000A2207F50C73A3F509730022A3F80C224D
S3150802ED1007F50C73A3F509730022A3F80E2207F56B
S3150802ED200C73A3F509730022A3F8102207F50C73D6
S3150802ED30A3F509730022A3F8122207F50C73A3F5AB
S3150802ED4009730022A3F8142207F50C73A3F50973B5
S3150802ED500022A3F8162207F50C73A3F509730022FD
S3150802ED60A3F8182207F50C73A3F509730022A3F872
S3150802ED701A2207F50C73A3F509730022A3F81C22BD
S3150802ED8007F50C73A3F509730022A3F81E220023C4
S3150802ED90C7F82C3266E107F50C73A3F50972D7F8A2
S3150802EDA02C325B0113441B88D9B207F50C73A3F501
S3150802EDB00B731A68D7F82C32134402330A461A70B0
S3150802EDC007F50C73A3F50972D7F82C325B011344C5
S3150802EDD00233198807F50C73A3F50B731A68D7F86B
S3150802EDE02C3208335B0013440A469A8007F50C73E3
S3150802EDF0A3F50972D7F82C325B0113440433198838
S3150802EE0007F50C73A3F50B731A68D7F82C32183367
S3150802EE105B0013440A46DA8007F50C73A3F50972F8
S3150802EE20D7F82C325B01134406331B88D9B207F58F
S3150802EE300C73A3F50B731A68D7F82C32134458339C
S3150802EE400A461A7007F50C73A3F50972D7F82C321D
S3150802EE505B01134408331B88D9B207F50C73A3F573
S3150802EE600B731A68D7F82C32134469330A461A7098
S3150802EE7007F50C73A3F50972D7F82C325B01134414
S3150802EE800A331B88D9B207F50C73A3F50B731A68F4
S3150802EE90D7F82C3213447A330A461A7007F50C73DC
S3150802EEA0A3F50972D7F82C325B0113440C331B887D
S3150802EEB0D9B207F50C73A3F50B731A68D7F82C3277
S3150802EEC013448B330A461A7007F50C73A3F50972B5
S3150802EED0D7F82C325B0113440E331B88D9B207F5D7
S3150802EEE00C73A3F50B731A68D7F82C3213449C33A8
S3150802EEF00A461A7007F50C73A3F50972D7F82C326D
S3150802EF005B01134410331B88D9B207F50C73A3F5BA
S3150802EF100B731A68D7F82C321344AD330A461A70A3
S3150802EF2007F50C73A3F50972D7F82C325B01134463
S3150802EF3012331B88D9B207F50C73A3F50B731A683B
S3150802EF40D7F82C321344BE330A461A7007F50C73E7
S3150802EF50A3F50972D7F82C325B01134414331B88C4
S3150802EF60D9B207F50C73A3F50B731A68D7F82C32C6
S3150802EF701344CF330A461A7007F50C73A3F50972C0
S3150802EF80D7F82C325B01134416331B88D9B207F51E
S3150802EF900C73A3F50B731A68D7F82C321344E033B3
S3150802EFA00A461A7007F50C73A3F50972D7F82C32BC
S3150802EFB05B01134418331B88D9B207F50C73A3F502
S3150802EFC00B731A68D7F82C321344F1330A461A70AF
S3150802EFD007F50C73A3F50972D7F82C325B011344B3
S3150802EFE01A331B88D9B207F50C73A3F50B731A6883
S3150802EFF0D7F82C32134403F581730A461A7007F5BB
S3150802F0000C73A3F50972D7F82C325B0113441C332F
S3150802F0101B88D9B207F50C73A3F50B731A68D7F8D0
S3150802F0202C32134403F213130A461A7007F50C73AB
S3150802F030A3F50972D7F82C325B0113441E331B88D9
S3150802F040D9B207F50C73A3F50B731A68D7F82C32E5
S3150802F050134403F592730A461A70D7F82C32013311
S3150802F060C7F82C32D7F82C32102B7FF794AE00BF94
S3150802F07007F50C77BD4680BD80B5ADF50C7D00AFB2
S3150802F08007F50C73A3F50B7318600846114607F5C6
S3150802F0900C73A3F22D2302461A7007F50C73A3F21A
S3150802F0A02E230A461A7007F50C73A3F50B734FF451
S3150802F0B09B720021186824F065F907F50C73A3F210
S3150802F0C02E231B781846FEF781F80346002BC0F25A
S3150802F0D0F18207F50C73A3F22E231B781846FEF766
S3150802F0E075F80346DAB2BC4B1A7007F50C73A3F52A
S3150802F0F0097318464FF408731A46002124F042F998
S3150802F10007F50C73A3F5097340F6B8325A8007F56A
S3150802F1100C73A3F5097350225A81AF4B1B781A4612
S3150802F12007F50C73A3F50973DA8207F50C73A3F5D1
S3150802F13009730122DA8307F50C73A3F50973012211
S3150802F1401A8407F50C73A3F509734FF47A625A8485
S3150802F15007F50C73A3F5097323221A8507F50C73B1
S3150802F160A3F5097364225A8507F50C73A3F22D23B6
S3150802F1701B789AB207F50C73A3F509735A8607F535
S3150802F1800C73A3F22D231B789BB2DB439AB207F5C5
S3150802F1900C73A3F509739A868F4B1B781A4607F5E3
S3150802F1A00C73A3F50973DA8607F50C73A3F50973CD
S3150802F1B00222A3F8402007F50C73A3F5097340F65B
S3150802F1C0C412A3F8422007F50C73A3F50973322279
S3150802F1D0A3F8482007F50C73A3F509736422A3F86C
S3150802F1E04A2007F50C73A3F22D231B789AB207F56A
S3150802F1F00C73A3F50973A3F8522007F50C73A3F24F
S3150802F2002D231B789BB2DB439AB207F50C73A3F541
S3150802F2100973A3F85420704B1B781A4607F50C732A
S3150802F220A3F50973A3F8562007F50C73A3F509731A
S3150802F2300122A3F85A2007F50C73A3F509730322D2
S3150802F240A3F8602007F50C73A3F5097340F6C412F8
S3150802F250A3F8622007F50C73A3F509733C22A3F8F9
S3150802F260682007F50C73A3F509733C22A3F86A20F4
S3150802F270594B1B781A4607F50C73A3F50973A3F8BD
S3150802F280762007F50C73A3F509730122A3F87A20F1
S3150802F29007F50C73A3F509730422A3F8802007F572
S3150802F2A00C73A3F5097340F6C412A3F8822007F576
S3150802F2B00C73A3F509733222A3F88A20464B1B78EE
S3150802F2C01A4607F50C73A3F50973A3F8962007F5F2
S3150802F2D00C73A3F509730122A3F89A2007F50C7398
S3150802F2E0A3F509730122A3F89E2007F50C73A3F56B
S3150802F2F009730522A3F8A02007F50C73A3F5097371
S3150802F30041F28832A3F8A22007F50C73A3F5097314
S3150802F3102322A3F8AA20304B1B781A4607F50C734A
S3150802F320A3F50973A3F8B62007F50C73A3F50973B9
S3150802F3300122A3F8BE2007F50C73A3F5097306226A
S3150802F340A3F8C02007F50C73A3F509730722A3F8DF
S3150802F350E02007F50C73A3F509730822A3F8002128
S3150802F36007F50C73A3F509730922A3F8202107F5FB
S3150802F3700C73A3F509730A22A3F8402107F50C7347
S3150802F380A3F509730B22A3F8602107F50C73A3F5FD
S3150802F39009730C22A3F8802107F50C73A3F50973E8
S3150802F3A00D22A3F8A02107F50C73A3F509730E2203
S3150802F3B0A3F8C02107F50C73A3F509730F22A3F866
S3150802F3C0E02107F50C73A3F509736322A3F800225B
S3150802F3D00023C7F82C3268E17B36012007F50C7347
S3150802F3E0A3F50972D7F82C325B0113441B88D9B2EC
S3150802F3F007F50C73A3F50B731A68D7F82C32134466
S3150802F40002330A461A7007F50C73A3F50972D7F880
S3150802F4102C325B0113440233198807F50C73A3F5E2
S3150802F4200B731A68D7F82C3208335B0013440A4662
S3150802F4309A8007F50C73A3F50972D7F82C325B018B
S3150802F44013440433198807F50C73A3F50B731A686A
S3150802F450D7F82C3218335B0013440A46DA8007F5CC
S3150802F4600C73A3F50972D7F82C325B0113440633E1
S3150802F4701B88D9B207F50C73A3F50B731A68D7F86C
S3150802F4802C32134458330A461A7007F50C73A3F53F
S3150802F4900972D7F82C325B01134408331B88D9B298
S3150802F4A007F50C73A3F50B731A68D7F82C321344B5
S3150802F4B069330A461A7007F50C73A3F50972D7F869
S3150802F4C02C325B0113440A331B88D9B207F50C7335
S3150802F4D0A3F50B731A68D7F82C3213447A330A4603
S3150802F4E01A7007F50C73A3F50972D7F82C325B016B
S3150802F4F013440C331B88D9B207F50C73A3F50B73A7
S3150802F5001A68D7F82C3213448B330A461A7007F551
S3150802F5100C73A3F50972D7F82C325B0113440E3328
S3150802F5201B88D9B207F50C73A3F50B731A68D7F8BB
S3150802F5302C3213449C330A461A7007F50C73A3F54A
S3150802F5400972D7F82C325B01134410331B88D9B2DF
S3150802F55007F50C73A3F50B731A68D7F82C32134404
S3150802F560AD330A461A7007F50C73A3F50972D7F874
S3150802F5702C325B01134412331B88D9B207F50C737C
S3150802F580A3F50B731A68D7F82C321344BE330A460E
S3150802F5901A7007F50C73A3F50972D7F82C325B01BA
S3150802F5A0134414331B88D9B207F50C73A3F50B73EE
S3150802F5B01A68D7F82C321344CF330A461A7007F55D
S3150802F5C00C73A3F50972D7F82C325B011344163370
S3150802F5D01B88D9B207F50C73A3F50B731A68D7F80B
S3150802F5E02C321344E0330A461A7007F50C73A3F556
S3150802F5F00972D7F82C325B01134418331B88D9B227
S3150802F60007F50C73A3F50B731A68D7F82C32134453
S3150802F610F1330A461A7007F50C73A3F50972D7F87F
S3150802F6202C325B0113441A331B88D9B207F50C73C3
S3150802F630A3F50B731A68D7F82C32134403F58173B2
S3150802F6400A461A7007F50C73A3F50972D7F82C3215
S3150802F6505B0113441C331B88D9B207F50C73A3F557
S3150802F6600B731A68D7F82C32134403F213130A469B
S3150802F6701A7007F50C73A3F50972D7F82C325B01D9
S3150802F68013441E331B88D9B207F50C73A3F50B7303
S3150802F6901A68D7F82C32134403F592730A461A707D
S3150802F6A0D7F82C320133C7F82C32D7F82C32102B64
S3150802F6B07FF794AE00BF07F50C77BD4680BD00BF45
S3150802F6C080B5ADF50C7D00AF07F50C73A3F50B738A
S3150802F6D018600846114607F50C73A3F22D23024655
S3150802F6E01A7007F50C73A3F22E230A461A7007F549
S3150802F6F00C73A3F50B734FF49B720021186823F061
S3150802F70041FE07F50C73A3F22E231B781846FDF764
S3150802F7105DFD0346002BC0F20B8307F50C73A3F2BB
S3150802F7202E231B781846FDF751FD0346DAB2C94B5C
S3150802F7301A7007F50C73A3F5097318464FF4087384
S3150802F7401A46002123F01EFE07F50C73A3F509736A
S3150802F75040F6B8325A8007F50C73A3F509732322CB
S3150802F760DA8007F50C73A3F5097350225A81B94B4F
S3150802F7701B781A4607F50C73A3F50973DA8207F59F
S3150802F7800C73A3F509730122DA8307F50C73A3F543
S3150802F790097301221A8407F50C73A3F509734FF44A
S3150802F7A07A625A8407F50C73A3F509732322DA845D
S3150802F7B007F50C73A3F5097328221A8507F50C7346
S3150802F7C0A3F5097364225A8507F50C73A3F22D2350
S3150802F7D01B789AB207F50C73A3F509735A8607F5CF
S3150802F7E00C73A3F22D231B789BB2DB439AB207F55F
S3150802F7F00C73A3F509739A86964B1B781A4607F576
S3150802F8000C73A3F50973DA8607F50C73A3F5097366
S3150802F8100222A3F8402007F50C73A3F5097340F6F4
S3150802F820AC52A3F8422007F50C73A3F509732322F9
S3150802F830A3F8462007F50C73A3F509733722A3F834
S3150802F840482007F50C73A3F509736422A3F84A2026
S3150802F85007F50C73A3F22D231B789AB207F50C73DE
S3150802F860A3F50973A3F8522007F50C73A3F22D2307
S3150802F8701B789BB2DB439AB207F50C73A3F509739F
S3150802F880A3F85420734B1B781A4607F50C73A3F595
S3150802F8900973A3F8562007F50C73A3F50973012219
S3150802F8A0A3F85A2007F50C73A3F509730322A3F8E4
S3150802F8B0602007F50C73A3F5097340F6C412A3F882
S3150802F8C0622007F50C73A3F509732322A3F86620B1
S3150802F8D007F50C73A3F509733C22A3F8682007F50C
S3150802F8E00C73A3F509733C22A3F86A20594B1B78BB
S3150802F8F01A4607F50C73A3F50973A3F8762007F5DC
S3150802F9000C73A3F509730122A3F87A2007F50C7381
S3150802F910A3F509730422A3F8802007F50C73A3F54F
S3150802F920097340F6C412A3F8822007F50C73A3F5EF
S3150802F93009733222A3F88A20464B1B781A4607F522
S3150802F9400C73A3F50973A3F8962007F50C73A3F5B0
S3150802F95009730122A3F89A2007F50C73A3F5097314
S3150802F9600122A3F89E2007F50C73A3F50973052255
S3150802F970A3F8A02007F50C73A3F5097341F28832A0
S3150802F980A3F8A22007F50C73A3F509732322A3F89B
S3150802F990AA20304B1B781A4607F50C73A3F5097390
S3150802F9A0A3F8B62007F50C73A3F509730122A3F889
S3150802F9B0BE2007F50C73A3F509730622A3F8C02027
S3150802F9C007F50C73A3F509730722A3F8E02007F5D8
S3150802F9D00C73A3F509730822A3F8002107F50C7323
S3150802F9E0A3F509730922A3F8202107F50C73A3F5D9
S3150802F9F009730A22A3F8402107F50C73A3F50973C4
S3150802FA000B22A3F8602107F50C73A3F509730C22E0
S3150802FA10A3F8802107F50C73A3F509730D22A3F841
S3150802FA20A02107F50C73A3F509730E22A3F8C021CA
S3150802FA3007F50C73A3F509730F22A3F8E02107F55E
S3150802FA400C73A3F509736322A3F800220023C7F8EF
S3150802FA502C3268E17C36012007F50C73A3F509728E
S3150802FA60D7F82C325B0113441B88D9B207F50C73FD
S3150802FA70A3F50B731A68D7F82C32134402330A46D5
S3150802FA801A7007F50C73A3F50972D7F82C325B01C5
S3150802FA9013440233198807F50C73A3F50B731A6816
S3150802FAA0D7F82C3208335B0013440A469A8007F5C6
S3150802FAB00C73A3F50972D7F82C325B01134404338D
S3150802FAC0198807F50C73A3F50B731A68D7F82C3245
S3150802FAD018335B0013440A46DA8007F50C73A3F55C
S3150802FAE00972D7F82C325B01134406331B88D9B244
S3150802FAF007F50C73A3F50B731A68D7F82C3213445F
S3150802FB0058330A461A7007F50C73A3F50972D7F823
S3150802FB102C325B01134408331B88D9B207F50C73E0
S3150802FB20A3F50B731A68D7F82C32134469330A46BD
S3150802FB301A7007F50C73A3F50972D7F82C325B0114
S3150802FB4013440A331B88D9B207F50C73A3F50B7352
S3150802FB501A68D7F82C3213447A330A461A7007F50C
S3150802FB600C73A3F50972D7F82C325B0113440C33D4
S3150802FB701B88D9B207F50C73A3F50B731A68D7F865
S3150802FB802C3213448B330A461A7007F50C73A3F505
S3150802FB900972D7F82C325B0113440E331B88D9B28B
S3150802FBA007F50C73A3F50B731A68D7F82C321344AE
S3150802FBB09C330A461A7007F50C73A3F50972D7F82F
S3150802FBC02C325B01134410331B88D9B207F50C7328
S3150802FBD0A3F50B731A68D7F82C321344AD330A46C9
S3150802FBE01A7007F50C73A3F50972D7F82C325B0164
S3150802FBF0134412331B88D9B207F50C73A3F50B739A
S3150802FC001A68D7F82C321344BE330A461A7007F517
S3150802FC100C73A3F50972D7F82C325B01134414331B
S3150802FC201B88D9B207F50C73A3F50B731A68D7F8B4
S3150802FC302C321344CF330A461A7007F50C73A3F510
S3150802FC400972D7F82C325B01134416331B88D9B2D2
S3150802FC5007F50C73A3F50B731A68D7F82C321344FD
S3150802FC60E0330A461A7007F50C73A3F50972D7F83A
S3150802FC702C325B01134418331B88D9B207F50C736F
S3150802FC80A3F50B731A68D7F82C321344F1330A46D4
S3150802FC901A7007F50C73A3F50972D7F82C325B01B3
S3150802FCA013441A331B88D9B207F50C73A3F50B73E1
S3150802FCB01A68D7F82C32134403F581730A461A7068
S3150802FCC007F50C73A3F50972D7F82C325B011344B6
S3150802FCD01C331B88D9B207F50C73A3F50B731A6884
S3150802FCE0D7F82C32134403F213130A461A7007F58F
S3150802FCF00C73A3F50972D7F82C325B0113441E3331
S3150802FD001B88D9B207F50C73A3F50B731A68D7F8D3
S3150802FD102C32134403F592730A461A70D7F82C321A
S3150802FD200133C7F82C32D7F82C32102B7FF794AE52
S3150802FD3000BF07F50C77BD4680BD00BF80B5ADF59F
S3150802FD400C7D00AF07F50C73A3F50B731860084614
S3150802FD50114607F50C73A3F22D2302461A7007F50E
S3150802FD600C73A3F22E230A461A7007F50C73A3F531
S3150802FD700B734FF49B720021186823F003FB07F5F7
S3150802FD800C73A3F22E231B781846FDF71FFA0346B7
S3150802FD90002BC0F20B8307F50C73A3F22E231B78F4
S3150802FDA01846FDF713FA0346DAB2C94B1A7007F575
S3150802FDB00C73A3F5097318464FF408731A46002103
S3150802FDC023F0E0FA07F50C73A3F5097340F6B83287
S3150802FDD05A8007F50C73A3F509732322DA8007F50F
S3150802FDE00C73A3F5097350225A81B94B1B781A462C
S3150802FDF007F50C73A3F50973DA8207F50C73A3F5F5
S3150802FE0009730122DA8307F50C73A3F50973012234
S3150802FE101A8407F50C73A3F509734FF47A625A84A8
S3150802FE2007F50C73A3F509732322DA8407F50C7315
S3150802FE30A3F5097323221A8507F50C73A3F509732B
S3150802FE4064225A8507F50C73A3F22D231B789AB2FE
S3150802FE5007F50C73A3F509735A8607F50C73A3F213
S3150802FE602D231B789BB2DB439AB207F50C73A3F5D5
S3150802FE7009739A86964B1B781A4607F50C73A3F5EF
S3150802FE800973DA8607F50C73A3F509730222A3F838
S3150802FE90402007F50C73A3F5097341F29412A3F8EF
S3150802FEA0422007F50C73A3F509732322A3F846200B
S3150802FEB007F50C73A3F509732D22A3F8482007F555
S3150802FEC00C73A3F509736422A3F84A2007F50C7389
S3150802FED0A3F22D231B789AB207F50C73A3F50973BF
S3150802FEE0A3F8522007F50C73A3F22D231B789BB2B5
S3150802FEF0DB439AB207F50C73A3F50973A3F85420EA
S3150802FF00734B1B781A4607F50C73A3F50973A3F806
S3150802FF10562007F50C73A3F509730122A3F85A2094
S3150802FF2007F50C73A3F509730322A3F8602007F5F6
S3150802FF300C73A3F5097340F6C412A3F8622007F5F9
S3150802FF400C73A3F509732322A3F8662007F50C732D
S3150802FF50A3F509733222A3F8682007F50C73A3F5F3
S3150802FF6009733222A3F86A20594B1B781A4607F5F9
S3150802FF700C73A3F50973A3F8762007F50C73A3F59A
S3150802FF8009730122A3F87A2007F50C73A3F50973FE
S3150802FF900422A3F8802007F50C73A3F5097340F62B
S3150802FFA0C412A3F8822007F50C73A3F5097332224B
S3150802FFB0A3F88A20464B1B781A4607F50C73A3F555
S3150802FFC00973A3F8962007F50C73A3F509730122A2
S3150802FFD0A3F89A2007F50C73A3F509730122A3F86F
S3150802FFE09E2007F50C73A3F509730522A3F8A02032
S3150802FFF007F50C73A3F5097341F28832A3F8A22018
S3150803000007F50C73A3F509732322A3F8AA20304B2B
S315080300101B781A4607F50C73A3F50973A3F8B620DC
S3150803002007F50C73A3F509730122A3F8BE2007F598
S315080300300C73A3F509730622A3F8C02007F50C73FE
S31508030040A3F509730722A3F8E02007F50C73A3F5B4
S3150803005009730822A3F8002107F50C73A3F509739E
S315080300600922A3F8202107F50C73A3F509730A22BD
S31508030070A3F8402107F50C73A3F509730B22A3F81C
S31508030080602107F50C73A3F509730C22A3F88021E5
S3150803009007F50C73A3F509730D22A3F8A02107F539
S315080300A00C73A3F509730E22A3F8C02107F50C7385
S315080300B0A3F509730F22A3F8E02107F50C73A3F53B
S315080300C009736322A3F800220023C7F82C3268E1D8
S315080300D07D36012007F50C73A3F50972D7F82C3280
S315080300E05B0113441B88D9B207F50C73A3F50B738D
S315080300F01A68D7F82C32134402330A461A7007F5DE
S315080301000C73A3F50972D7F82C325B011344023337
S31508030110198807F50C73A3F50B731A68D7F82C32ED
S3150803012008335B0013440A469A8007F50C73A3F554
S315080301300972D7F82C325B0113440433198807F57F
S315080301400C73A3F50B731A68D7F82C3218335B00B4
S3150803015013440A46DA8007F50C73A3F50972D7F830
S315080301602C325B01134406331B88D9B207F50C738B
S31508030170A3F50B731A68D7F82C32134458330A4677
S315080301801A7007F50C73A3F50972D7F82C325B01BD
S31508030190134408331B88D9B207F50C73A3F50B73FD
S315080301A01A68D7F82C32134469330A461A7007F5C6
S315080301B00C73A3F50972D7F82C325B0113440A337F
S315080301C01B88D9B207F50C73A3F50B731A68D7F80E
S315080301D02C3213447A330A461A7007F50C73A3F5BF
S315080301E00972D7F82C325B0113440C331B88D9B236
S315080301F007F50C73A3F50B731A68D7F82C32134457
S315080302008B330A461A7007F50C73A3F50972D7F8E8
S315080302102C325B0113440E331B88D9B207F50C73D2
S31508030220A3F50B731A68D7F82C3213449C330A4682
S315080302301A7007F50C73A3F50972D7F82C325B010C
S31508030240134410331B88D9B207F50C73A3F50B7344
S315080302501A68D7F82C321344AD330A461A7007F5D1
S315080302600C73A3F50972D7F82C325B0113441233C6
S315080302701B88D9B207F50C73A3F50B731A68D7F85D
S315080302802C321344BE330A461A7007F50C73A3F5CA
S315080302900972D7F82C325B01134414331B88D9B27D
S315080302A007F50C73A3F50B731A68D7F82C321344A6
S315080302B0CF330A461A7007F50C73A3F50972D7F8F4
S315080302C02C325B01134416331B88D9B207F50C731A
S315080302D0A3F50B731A68D7F82C321344E0330A468E
S315080302E01A7007F50C73A3F50972D7F82C325B015C
S315080302F0134418331B88D9B207F50C73A3F50B738C
S315080303001A68D7F82C321344F1330A461A7007F5DC
S315080303100C73A3F50972D7F82C325B0113441A330D
S315080303201B88D9B207F50C73A3F50B731A68D7F8AC
S315080303302C32134403F581730A461A7007F50C73B6
S31508030340A3F50972D7F82C325B0113441C331B88B7
S31508030350D9B207F50C73A3F50B731A68D7F82C32C1
S31508030360134403F213130A461A7007F50C73A3F51D
S315080303700972D7F82C325B0113441E331B88D9B292
S3150803038007F50C73A3F50B731A68D7F82C321344C5
S3150803039003F592730A461A70D7F82C320133C7F855
S315080303A02C32D7F82C32102B7FF794AE00BF07F503
S315080303B00C77BD4680BD00BF80B5ADF50C7D00AF9B
S315080303C007F50C73A3F50B7318600846114607F572
S315080303D00C73A3F22D2302461A7007F50C73A3F2C6
S315080303E02E230A461A7007F50C73A3F50B734FF4FD
S315080303F09B720021186822F0C5FF07F50C73A3F258
S315080304002E231B781846FCF7E1FE0346002BC0F2A1
S315080304100B8307F50C73A3F22E231B781846FCF7F8
S31508030420D5FE0346DAB2C94B1A7007F50C73A3F562
S31508030430097318464FF408731A46002122F0A2FFDF
S3150803044007F50C73A3F5097340F6B8325A8007F516
S315080304500C73A3F509734122DA8007F50C73A3F528
S31508030460097350225A81B94B1B781A4607F50C7340
S31508030470A3F50973DA8207F50C73A3F50973012249
S31508030480DA8307F50C73A3F5097301221A8407F5B2
S315080304900C73A3F509734FF47A625A8407F50C7340
S315080304A0A3F509734122DA8407F50C73A3F50973D7
S315080304B028221A8507F50C73A3F5097364225A854E
S315080304C007F50C73A3F22D231B789AB207F50C7361
S315080304D0A3F509735A8607F50C73A3F22D231B7824
S315080304E09BB2DB439AB207F50C73A3F509739A8695
S315080304F0964B1B781A4607F50C73A3F50973DA8628
S3150803050007F50C73A3F509730222A3F8402007F530
S315080305100C73A3F5097340F6C412A3F8422007F532
S315080305200C73A3F509734122A3F8462007F50C7348
S31508030530A3F509733722A3F8482007F50C73A3F527
S3150803054009736422A3F84A2007F50C73A3F22D2333
S315080305501B789AB207F50C73A3F50973A3F852200F
S3150803056007F50C73A3F22D231B789BB2DB439AB2D0
S3150803057007F50C73A3F50973A3F85420734B1B787B
S315080305801A4607F50C73A3F50973A3F8562007F55E
S315080305900C73A3F509730122A3F85A2007F50C7304
S315080305A0A3F509730322A3F8602007F50C73A3F5D3
S315080305B009734FF4FA62A3F8622007F50C73A3F5DF
S315080305C009733722A3F8662007F50C73A3F5097395
S315080305D04122A3F8682007F50C73A3F509733C2297
S315080305E0A3F86A20594B1B781A4607F50C73A3F52B
S315080305F00973A3F8762007F50C73A3F5097301228B
S31508030600A3F87A2007F50C73A3F509730422A3F854
S31508030610802007F50C73A3F5097340F2DC52A3F89F
S31508030620822007F50C73A3F509733222A3F88A20EF
S31508030630464B1B781A4607F50C73A3F50973A3F8FB
S31508030640962007F50C73A3F509730122A3F89A20DC
S3150803065007F50C73A3F509730122A3F89E2007F582
S315080306600C73A3F509730522A3F8A02007F50C73E9
S31508030670A3F5097341F28832A3F8A22007F50C7390
S31508030680A3F509732322A3F8AA20304B1B781A462D
S3150803069007F50C73A3F50973A3F8B62007F50C73CE
S315080306A0A3F509730122A3F8BE2007F50C73A3F576
S315080306B009730622A3F8C02007F50C73A3F509737B
S315080306C00722A3F8E02007F50C73A3F5097308229C
S315080306D0A3F8002107F50C73A3F509730922A3F8F8
S315080306E0202107F50C73A3F509730A22A3F8402101
S315080306F007F50C73A3F509730B22A3F8602107F515
S315080307000C73A3F509730C22A3F8802107F50C7360
S31508030710A3F509730D22A3F8A02107F50C73A3F516
S3150803072009730E22A3F8C02107F50C73A3F5097301
S315080307300F22A3F8E02107F50C73A3F509736322C7
S31508030740A3F800220023C7F82C3268E17E3601207D
S3150803075007F50C73A3F50972D7F82C325B0113441A
S315080307601B88D9B207F50C73A3F50B731A68D7F868
S315080307702C32134402330A461A7007F50C73A3F591
S315080307800972D7F82C325B0113440233198807F52B
S315080307900C73A3F50B731A68D7F82C3208335B006E
S315080307A013440A469A8007F50C73A3F50972D7F81A
S315080307B02C325B0113440433198807F50C73A3F52C
S315080307C00B731A68D7F82C3218335B0013440A469E
S315080307D0DA8007F50C73A3F50972D7F82C325B0197
S315080307E0134406331B88D9B207F50C73A3F50B73A9
S315080307F01A68D7F82C32134458330A461A7007F581
S315080308000C73A3F50972D7F82C325B01134408332A
S315080308101B88D9B207F50C73A3F50B731A68D7F8B7
S315080308202C32134469330A461A7007F50C73A3F579
S315080308300972D7F82C325B0113440A331B88D9B2E1
S3150803084007F50C73A3F50B731A68D7F82C32134400
S315080308507A330A461A7007F50C73A3F50972D7F8A3
S315080308602C325B0113440C331B88D9B207F50C737E
S31508030870A3F50B731A68D7F82C3213448B330A463D
S315080308801A7007F50C73A3F50972D7F82C325B01B6
S3150803089013440E331B88D9B207F50C73A3F50B73F0
S315080308A01A68D7F82C3213449C330A461A7007F58C
S315080308B00C73A3F50972D7F82C325B011344103372
S315080308C01B88D9B207F50C73A3F50B731A68D7F807
S315080308D02C321344AD330A461A7007F50C73A3F585
S315080308E00972D7F82C325B01134412331B88D9B229
S315080308F007F50C73A3F50B731A68D7F82C32134450
S31508030900BE330A461A7007F50C73A3F50972D7F8AE
S315080309102C325B01134414331B88D9B207F50C73C5
S31508030920A3F50B731A68D7F82C321344CF330A4648
S315080309301A7007F50C73A3F50972D7F82C325B0105
S31508030940134416331B88D9B207F50C73A3F50B7337
S315080309501A68D7F82C321344E0330A461A7007F597
S315080309600C73A3F50972D7F82C325B0113441833B9
S315080309701B88D9B207F50C73A3F50B731A68D7F856
S315080309802C321344F1330A461A7007F50C73A3F590
S315080309900972D7F82C325B0113441A331B88D9B270
S315080309A007F50C73A3F50B731A68D7F82C3213449F
S315080309B003F581730A461A7007F50C73A3F50972D2
S315080309C0D7F82C325B0113441C331B88D9B207F5BD
S315080309D00C73A3F50B731A68D7F82C32134403F276
